:0200000480007A
:10000000130540006B000500975101009381819614
:10001000F32610029396A601732600029315A600FC
:100020001316260037F1FF6F3301B1403301D14081
:100030003301C100F3261002638606001305000099
:100040006B00050067800000130101FD232681027B
:1000500013040103232EA4FC232CB4FC232AC4FC88
:100060008327C4FD83A707002326F4FE930744FDDE
:100070002322F4FE832744FE03C707008327C4FE20
:100080002380E7008327C4FE93871700032744FEDD
:10009000034717002380E7008327C4FE93872700C8
:1000A000032744FE034727002380E7008327C4FE7D
:1000B00093873700032744FE034737002380E70078
:1000C0008327C4FE938747002326F4FE232404FEDF
:1000D0006F004003832784FE032784FDB307F700E6
:1000E00003C707008327C4FE2380E7008327C4FEDD
:1000F000938717002326F4FE832784FE9387170037
:100100002324F4FE832744FD032784FEE344F7FC05
:100110008327C4FE2320F4FE832704FE93F73700D1
:10012000032704FEB307F7002320F4FE832704FE11
:100130002326F4FE8327C4FD0327C4FE23A0E70083
:10014000130000000324C1021301010367800000B3
:10015000130101FC232E8102130401042326A4FCB5
:100160002324B4FC8327C4FC83A707002326F4FEC2
:10017000832744FE2320F4FE8327C4FE03C7070021
:10018000832704FE2380E700832704FE938717005C
:100190000327C4FE034717002380E700832704FEDC
:1001A000938727000327C4FE034727002380E70027
:1001B000832704FE938737000327C4FE03473700D5
:1001C0002380E7008327C4FE938747002326F4FE9D
:1001D000232404FE6F004003832784FE032784FC4E
:1001E000B307F7000327C4FE034707002380E70097
:1001F0008327C4FE938717002326F4FE832784FEFB
:10020000938717002324F4FE032784FE832744FEEC
:10021000E344F7FC8327C4FE232EF4FC8327C4FDAC
:1002200093F737000327C4FDB307F700232EF4FC30
:100230008327C4FD2326F4FE8327C4FC0327C4FEC2
:1002400023A0E700130000000324C10313010104ED
:1002500067800000130101FF232611002324810081
:1002600013040101B707008113850704EF00404024
:10027000130000008320C100032481001301010149
:1002800067800000130101FE232E1100232C810042
:10029000130401022326A4FE2324B4FEB707008121
:1002A00013854705EF00C03C832784FE37270000F5
:1002B00023A2E70093070000138507008320C101F4
:1002C000032481011301010267800000130101FE74
:1002D000232E1100232C8100130401022326A4FEE7
:1002E000B707008113858706EF0080389307100059
:1002F000138507008320C10103248101130101023A
:1003000067800000130101FF2326110023248100D0
:1003100013040101B70700811385C707EF004035BB
:10032000130000008320C100032481001301010198
:1003300067800000130101FF2326110023248100A0
:1003400013040101B707008113850709EF0040324C
:10035000130000008320C100032481001301010168
:1003600067800000130101FD23261102232481026E
:1003700013040103232EA4FC232CB4FC232AC4FC65
:10038000B70700712326F4FE930750002324F4FEE0
:10039000130784FE9307C4FE13064000930507006D
:1003A00013850700EFF05FCA1307C4FD9307C4FE6F
:1003B000130640009305070013850700EFF0DFC820
:1003C0009307C4FE032644FD832584FD138507009F
:1003D000EFF09FC7B727008183A7C7BAE780070060
:1003E000B70700811385470AEF008028832744FD63
:1003F000138507008320C102032481021301010336
:1004000067800000130101FD23268102130401030C
:10041000232EA4FC8327C4FD63D807008327C4FDD3
:10042000B307F040232EF4FC0327C4FDB7370000C8
:100430009387078063D8E700B7370000938707806A
:10044000232EF4FCB727008183A707BB2326F4FEE5
:10045000B727008103A707BB8327C4FD3307F70035
:10046000B727008123A8E7BA8327C4FE13850700B6
:100470000324C1021301010367800000130101FE80
:10048000232E1100232C8100130401022326A4FE35
:10049000B70700811385870BEF00801D130500004F
:1004A000EF000016130000008320C1010324810126
:1004B0001301010267800000130101FE232E1100C9
:1004C000232C8100130401022326A4FE2324B4FE5E
:1004D0002322C4FEB70700811385470AEF004019A5
:1004E00093070000138507008320C10103248101C5
:1004F0001301010267800000130101FF2326110090
:100500002324810013040101B70700811385C70C60
:10051000EF000016130000008320C10003248100B7
:100520001301010167800000130101FF2326110060
:100530002324810013040101EF00000F930705003D
:10054000138507008320C1000324810013010101EA
:1005500067800000130101FF23261100232481007E
:1005600013040101B70700811385070FEF00401046
:10057000130000008320C100032481001301010146
:1005800067800000130101FF23261100232481004E
:1005900013040101B707008113854711EF00400DD7
:1005A000B727008183A787BC938617003727008170
:1005B0002324D7BC138507008320C10003248100B6
:1005C0001301010167800000130101FF23261100C0
:1005D0002324810013040101B70700811385071448
:1005E000EF000009130000008320C10003248100F4
:1005F00013010101678000006B10B50067800000E7
:100600006B000500678000006B40B500678000004C
:100610006B200500678000006B30000067800000E1
:1006200073251002678000007325000267800000B8
:10063000130540006B000500F32610029396F600A8
:10064000732600029315A6001316260037F1FF6FDC
:100650003301B1403301D1403301C100F326100210
:1006600063860600130500006B000500678000002C
:10067000130141FF232011002322B100834505000F
:1006800063880500EF00C001130515006FF01FFF20
:1006900083200100832541001301C1006780000011
:1006A000B702010023A0B20067800000130101FD22
:1006B000232611022324810213040103232EA4FC08
:1006C0000327C4FD9307F00063E4E702B717008136
:1006D0001387070C8327C4FD93972700B307F70000
:1006E00083A7070013850700EFF09FF86F0040070E
:1006F000930700022326F4FEA30504FE8327C4FE0D
:100700009387C7FF0327C4FDB357F70093F7F7009C
:100710002322F4FE832744FE63860700930710001C
:10072000A305F4FE8347B4FE63820702B717008176
:100730001387070C832744FE93972700B307F7001E
:1007400083A7070013850700EFF09FF28327C4FEFD
:100750009387C7FF2326F4FE8327C4FEE340F0FA05
:100760008320C1020324810213010103678000007A
:10077000130101FE232E1100232C8100130401021A
:100780002326A4FE2324B4FE0325C4FEEFF05FEE6F
:10079000032584FEEFF09FF1B70700811385471A08
:1007A000EFF01FED130000008320C101032481013D
:1007B0001301010267800000130101FE232E1100C6
:1007C000232C810013040102B727008183A747BEB1
:1007D00013850700EFF0DFE2B727008103A747BDCD
:1007E000B727008183A707BD13850700E70007002F
:1007F000EFF01FE32326A4FE8327C4FE63880700CF
:1008000013050000EFF0DFDF6F00C00013051000DC
:10081000EFF01FDF130000008320C10103248101DA
:100820001301010267800000130101FE232E110055
:10083000232C8100130401022326A4FE2324B4FEEA
:100840002322C4FE2320D4FEB7270081032744FEC1
:1008500023AAE7BCB7270081032704FE23A8E7BC2F
:10086000B7270081032784FE23A2E7BEB7070080D5
:100870009387877B938507000325C4FEEFF0DFD7BE
:10088000EFF09FF3130000008320C10103248101D6
:100890001301010267800000130101FE232E1100E5
:1008A000232C810013040102B727008183A787BD91
:1008B00013850700EFF0DFD4EFF01FD79307050093
:1008C0002326F4FEEFF0DFD5930705002324F4FE82
:1008D000B727008103A8C7BCB727008103A5C7BD00
:1008E000B727008183A707BE0326C4FE832684FEA4
:1008F0001307000093850700E7000800832784FEA4
:100900006386070013050000EFF09FCF130510006A
:10091000EFF01FCF130000008320C10103248101E9
:100920001301010267800000130101FE232E110054
:10093000232C8100130401022326A4FE2324B4FEE9
:100940002322C4FE8327C4FE03A787009307100059
:1009500063FAE700B70700811385871AEF00501D7F
:100960006F0080068327C4FE03A70700B727008116
:1009700023ACE7BC032784FEB727008123A6E7BC8E
:10098000B72700810327C4FE23A0E7BEB727008155
:10099000032744FE23AEE7BC8327C4FE03A747001A
:1009A0009307100063F0E7028327C4FE03A7470004
:1009B000B717008093878789938507001305070081
:1009C000EFF09FC3EFF05FED8320C10103248101AD
:1009D0001301010267800000130101FE232E1100A4
:1009E000232C810013040102B70700811385C7215E
:1009F000EFF01FC813054000EFF09FC0EFF0DFC21B
:100A00002326A4FE0327C4FEB7170081938607148C
:100A10008327C4FE93972700B387F60023A0E7003F
:100A200013051000EFF0DFBDB7170081938707149F
:100A300083A7070013850700EFF05FC7B7070081A2
:100A40001385C722EFF0DFC2B71700819387071421
:100A500083A7470013850700EFF05FC5B707008144
:100A60001385C722EFF0DFC0B71700819387071403
:100A700083A7870013850700EFF05FC3B7070081E6
:100A80001385C722EFF0DFBEB717008193870714E5
:100A900083A7C70013850700EFF05FC1B707008188
:100AA0001385C722EFF0DFBC130000008320C101D3
:100AB000032481011301010267800000130101FE7C
:100AC000232E1100232C810013040102EFF0DFB567
:100AD0002326A4FE8327C4FE93B72700A305F4FEB4
:100AE0008347B4FE13850700EFF09FB28347B4FE3F
:100AF000638407068327C4FE93B71700A304F4FE9C
:100B0000834794FE13850700EFF09FB0834794FE60
:100B100063820702B7270081138787BF8327C4FE3C
:100B200093972700B307F7001307A00023A0E7005F
:100B30006F000002B7270081138787BF8327C4FE99
:100B400093972700B307F7001307B00023A0E7002F
:100B5000EFF09FAC6F0040068327C4FE93B73700C9
:100B60002305F4FE8347A4FE13850700EFF05FAA78
:100B70008347A4FE63820702B7270081138787BFDC
:100B80008327C4FE93972700B307F7001307C0001D
:100B900023A0E7006F000002B7270081138787BFFB
:100BA0008327C4FE93972700B307F7001307D000ED
:100BB00023A0E700EFF05FA6EFF01FA6B7270081A4
:100BC000938787BF83A7070013850700EFF01FAE49
:100BD000B70700811385C722EFF09FA9B7270081CF
:100BE000938787BF83A7470013850700EFF01FACEB
:100BF000B70700811385C722EFF09FA7B7270081B1
:100C0000938787BF83A7870013850700EFF01FAA8C
:100C1000B70700811385C722EFF09FA5B727008192
:100C2000938787BF83A7C70013850700EFF01FA82E
:100C3000B70700811385C722EFF09FA313000000C0
:100C40008320C10103248101130101026780000098
:100C5000130101FE232E1100232C81001304010235
:100C6000EFF01F9C2326A4FEB7270081138787BEC1
:100C70008327C4FE93972700B307F7000327C4FE1A
:100C800023A0E7008327C4FE638607001305000046
:100C9000EFF01F97130000008320C101032481019E
:100CA0001301010267800000130101FE232E1100D1
:100CB000232C810013040102B7170080938707C516
:100CC0002326F4FE8325C4FE13054000EFF0DF92D7
:100CD000EFF01FF8B7270081938787BE83A707002F
:100CE00013850700EFF09F9CB70700811385C7228B
:100CF000EFF01F98B7270081938787BE83A747002F
:100D000013850700EFF09F9AB70700811385C7226C
:100D1000EFF01F96B7270081938787BE83A78700D0
:100D200013850700EFF09F98B70700811385C7224E
:100D3000EFF01F94B7270081938787BE83A7C70072
:100D400013850700EFF09F96B70700811385C72230
:100D5000EFF01F92130000008320C10103248101E2
:100D60001301010267800000130101FF2326110017
:100D70002324810013040101EFF01FC6B70700818F
:100D800013850723EFF0DF8E13054000EFF05F8738
:100D9000EFF0DFD213051000EFF09F86B707008158
:100DA00013854724EFF0DF8CEFF01FF013000000F5
:100DB0008320C1000324810013010101678000002A
:100DC000130101FC232E1102232C810213040104C0
:100DD0002326A4FC8327C4FC2326F4FEEFF05F84C3
:100DE0002324A4FEEFF05F842322A4FE8327C4FE05
:100DF00083A70701032784FE637EF7008327C4FED1
:100E000083A7C700032744FE6376F700930710000B
:100E10006F00800093070000A301F4FE834734FEB7
:100E200093F71700A301F4FE834734FE13850700F0
:100E3000EFF00FFE834734FE638607068327C4FE68
:100E400003A7C700832784FEB307F702032744FEE6
:100E5000B307F700232EF4FC8327C4FE03A7070083
:100E60008327C4FD93972700B307F70083A60700E5
:100E70008327C4FE03A747008327C4FD9397270059
:100E8000B307F70003A707008327C4FE03A6870064
:100E90008327C4FD93972700B307F6003387E60046
:100EA00023A0E700EFF04FF7130000008320C103F9
:100EB000032481031301010467800000130101FB77
:100EC00023261104232481041304010513051000B3
:100ED000EFF00FF3B707008113850729EFF04FF903
:100EE000EFF09FAFB70700811385072AEFF04FF8A7
:100EF00013054000EFF0CFF0EFF05FBC13051000DA
:100F0000EFF00FF0B70700811385472BEFF04FF696
:100F1000EFF09FD9B70700811385472CEFF04FF50D
:100F2000B707FFFF2326F4FE232404FE232204FE3A
:100F30006F0000088327C4FE032784FE23A0E70078
:100F40008327C4FE83A707002326F4FC8327C4FE5F
:100F500093850700B70700811385872DEFF05F8128
:100F6000832584FEB70700811385072EEFF05F808D
:100F70008325C4FCB70700811385472FEFF04FFF8F
:100F8000B707008113854730EFF08FEE832784FE8B
:100F9000938717002324F4FE8327C4FE938747001A
:100FA0002326F4FE832744FE938717002322F4FEB2
:100FB000032744FE93074000E3DEE7F6B70700810E
:100FC0001385C731EFF0CFEAB71700819387071970
:100FD000232CF4FAB71700819387071D232EF4FA08
:100FE000B7270081938787C02320F4FC9307400034
:100FF0002322F4FC930740002324F4FC93074000D1
:10100000232CF4FC93074000232AF4FC032784FDDF
:10101000832544FD930784FB93860700B717008060
:10102000138607DC13050700EFF01F80232004FE62
:101030006F000008232E04FC6F004005032744FCCA
:10104000832704FE3307F7028327C4FDB307F700A5
:101050002328F4FCB7270081138787C0832704FD6A
:1010600093972700B307F70083A7070013850700AE
:10107000EFF0CFE3B70700811385C733EFF04FDF01
:101080008327C4FD93871700232EF4FC032744FC19
:101090008327C4FDE3E4E7FAB7070081138507342B
:1010A000EFF00FDD832704FE938717002320F4FE63
:1010B000032784FC832704FEE3EEE7F69307000092
:1010C000138507008320C104032481041301010553
:1010D00067800000930505009306000013060000DA
:1010E000130500006F209076130101FF93050000A7
:1010F000232481002326110013040500EF20D07E55
:10110000B717008103A547028327C503638407003F
:10111000E780070013050400EFF04FB6130101FF4D
:1011200023248100B70700003704000013040400E3
:1011300093870700B387874023229100232611005D
:1011400093D42740638004029387C7FF33848700CA
:10115000832704009384F4FF1304C4FFE78007008F
:10116000E39804FE8320C10003248100832441000E
:101170001301010167800000130101FF2324810096
:1011800023202101370400003709000093070400E1
:10119000130909003309F940232611002322910085
:1011A000135929406300090213040400930400004A
:1011B000832704009384140013044400E78007008D
:1011C000E31899FE37040000370900009307040074
:1011D000130909003309F940135929406300090232
:1011E0001304040093040000832704009384140074
:1011F00013044400E7800700E31899FE8320C10030
:10120000032481008324410003290100130101010B
:10121000678000001303F00013070500637EC3021C
:101220009377F7006390070A63920508937606FFA9
:101230001376F600B386E6002320B7002322B7001A
:101240002324B7002326B70013070701E366D7FE60
:101250006314060067800000B306C340939626001F
:1012600097020000B38656006780C6002307B700C8
:10127000A306B7002306B700A305B7002305B700F0
:10128000A304B7002304B700A303B7002303B700E8
:10129000A302B7002302B700A301B7002301B700E0
:1012A000A300B7002300B7006780000093F5F50F97
:1012B00093968500B3E5D50093960501B3E5D50077
:1012C0006FF0DFF69396270097020000B386560072
:1012D00093820000E78006FA93800200938707FF5D
:1012E0003307F7403306F600E378C3F66FF0DFF319
:1012F000130101FC2324C1022326D1022328E10289
:10130000232AF102232C0103232E11031386050047
:101310008325850093068102232E11002326D10008
:10132000EF0000068320C101130101046780000063
:1013300037230081032383BB130101FC2324C10253
:101340002326D1022322B1022328E102232AF1021B
:10135000232C0103232E11038325830093064102CE
:101360001306050013050300232E11002326D100C8
:10137000EF0000018320C101130101046780000018
:10138000130101E12326111E2320211F2324811D87
:101390002320A11D138C050013090600232AD10068
:1013A0002324811E2322911E232E311D232C411D17
:1013B000232A511D2328611D2326711D2322911DDF
:1013C000232EB11B130D0500EF60C05B83270500C2
:1013D000138507002328F102EF8040752326A10220
:1013E0002328010E232A010E232C010E232E010E89
:1013F00063060D0003278D03E308070A8316CC005C
:1014000013970601939726011357070163CA070232
:101410003727000003264C0633E7E60013170701C1
:10142000B7E6FFFF135707419386F6FFB376D60062
:101430002316EC00131707012322DC0613570701BC
:10144000937687006388062E83260C016384062E1C
:101450001377A7019306A0006300D7309307C1104C
:10146000370700812322F10E9388070093078738FE
:1014700037070081232CF100130B09009307475015
:101480002324F10083470B002326010E2324010EA1
:1014900023200102232A0102232C0102232E010210
:1014A0002324010423260104232601006386072246
:1014B00013040B0093065002638AD730834714004D
:1014C00013041400E39A07FEB30464416306642125
:1014D0008326C10E8327810E23A06801B386960060
:1014E0009387170023A298002326D10E2324F10E00
:1014F000930670009388880063C2F62E0327C1000C
:1015000083470400330797002326E1006386071C06
:1015100083441400A303010C13041400930DF0FF83
:1015200093090000130A00001309A005930A900014
:10153000930BA002938C080013041400938704FEFD
:101540006364F9040327810193972700B387E700B9
:1015500083A707006780070093090000938604FDB6
:101560008344040093972900B387370193971700AA
:10157000B389F600938604FD13041400E3F2DAFE47
:10158000938704FEE370F9FC93880C0063860414CF
:1015900023069114A303010C930A1000930C10006E
:1015A000130BC11423280100930D00002324010212
:1015B00023220102232E0100937B2A0063840B0067
:1015C000938A2A0013794A088327C10E63160900FB
:1015D00033885941E34600718346710C638A0602E1
:1015E0008326810E1306710C23A0C8009387170071
:1015F000130610009386160023A2C8002326F10EBE
:101600002324D10E13067000938888006342D652BB
:10161000638C0B028326810E1306810C23A0C80065
:1016200093872700130620009386160023A2C80084
:101630002326F10E2324D10E130670009388880010
:101640006354D6006F00D07893060008E30ED93CAF
:10165000B38D9D41E34AB04993760A10E39806287A
:101660000327810EB387970123A068011307170092
:1016700023A298012326F10E2324E10E9306700085
:1016800063C8E65493888800137A4A0063060A0008
:10169000B3845941634E905463D4590193890A002D
:1016A0000327C100330737012326E100E398074EE3
:1016B000832701012324010E63880700832501018C
:1016C00013050D00EF30802D9308C110130B04009B
:1016D00083470B00E39E07DC8327C10E638407006A
:1016E0006F1050328357CC0093F7070463840700D0
:1016F0006F2000238320C11E0324811E0325C10007
:101700008324411E0329011E8329C11D032A811D33
:10171000832A411D032B011D832BC11C032C811C1B
:10172000832C411C032D011C832DC11B1301011FA0
:101730006780000093050C0013050D00EF20007B6F
:10174000630405006F20C01D0357CC009306A00062
:101750001377A701E314D7D00317EC00E34007D0B9
:10176000832641011306090093050C0013050D00A3
:10177000EF20C06B2326A1006FF0DFF713050D00EB
:10178000EF60402083274500138507002326F104DE
:10179000EF80C0399307050013050D0093840700FF
:1017A0002324F104EF60001E83278500232EF1021D
:1017B000638404006F10C012834404006FF0DFD70D
:1017C00083440400136A0A026FF01FD7B304644114
:1017D000E31064D1834704006FF05FD31306410E1A
:1017E00093050C0013050D00EFA0D077E31C05EE68
:1017F0009308C1106FF09FD093778A0093880C00F4
:10180000638407006F10C012832741011305010B89
:10181000232891019387770093F787FF83A507001B
:1018200003A6470093878700232AF100EF20D134D5
:101830008327010B832801012328F10E8327410B05
:10184000232AF10E8327810B232CF10E8327C10B52
:10185000232EF10E1305010F23281101EF60C00B99
:101860002326A10C93072000832801016314F500AF
:101870006F10C04F930710006314F5006F104064A1
:10188000930710066394F4006F20401C9307100424
:101890006394F4006F10101993FBF4FD9307F0FFAD
:1018A000232271056394FD006F20002893077004C4
:1018B0006394FB006F20001E0323C10F2324410308
:1018C000032E010F832E410F032F810F93670A1000
:1018D000635403006F20003E232C0104138A070089
:1018E00023280100930760046394FB006F10906944
:1018F00093075004232811056384FB006F10906048
:1019000013891D00930A010B930609001308C10DEA
:101910009307010D1307C10C1306200093850A00DD
:1019200013050D002328C10B2320C105232AD10B49
:101930002322D103232CE10B2320E103232E610A70
:10194000232E6100EF40D0530323C101032F010276
:10195000832E4102032E010483280105130B050089
:1019600033092501930C010A93850C0013850A00A5
:10197000232E11012328C10B232AD10B232CE10B89
:10198000232E610A2320010A2322010A2324010AAB
:101990002326010AEFF090708328C1011307090084
:1019A000630205020327C10D637E2701930600032E
:1019B00093071700232EF10C2300D7000327C10D36
:1019C000E36827FFB30767412320F1020327C10C17
:1019D00093077004232EE100032741046314F700EA
:1019E0006F10D04303274104930760046314F7008A
:1019F0006F10D0678327C1010327410493051004AA
:101A00009387F7FF2326F10C93F6F40F13060000DB
:101A10006318B7009386F60093F6F60F13061000CE
:101A2000230AD10C9306B00263DA07000327C10131
:101A3000930710009306D002B387E740A30AD10CA6
:101A40009306900063C4F6006F20C0281308310E7F
:101A5000130508001306A000130E300633E7C70273
:101A600093050500938607001305F5FF1307070389
:101A7000A38FE5FEB3C7C702E342DEFE93870703E9
:101A800013F6F70FA30FC5FE9387E5FF63E4070185
:101A90006F2040379306610D6F00800003C607007A
:101AA0002380C6009387170093861600E39807FFEC
:101AB0009307510EB387B7401307610DB307F700C3
:101AC0009306410DB387D740232CF102032701026F
:101AD0008326810393071000B30CD70063C4E7008B
:101AE0006F2040298327C102B38CFC008327810229
:101AF00093CAFCFF93DAFA4113FAF7BF136A0A108C
:101B0000B3FA5C012324010223220102232E0100E7
:101B100083278105639407006F1090379307D002E5
:101B2000A303F10C930D0000938A1A006FF0DFA855
:101B30001306410E93050C0013050D00EFA0904213
:101B4000E31805068327C10E9308C1106FF05FAC40
:101B5000832601030327C1021306700023A0D800C7
:101B60008326810EB307F70023A2E80093861600B0
:101B70002326F10E2324D10E938888006354D602C5
:101B80001306410E93050C0013050D00EFA0903DC8
:101B9000E31005028325C10C8327C10E8326810E25
:101BA0009308C11063D405006F1050580327010239
:101BB0009386160023A06801B307F70023A2E8006C
:101BC0002326F10E2324D10E13077000E35CD7AA5D
:101BD0001306410E93050C0013050D00EFA090387D
:101BE0006318057C8327C10E9308C1106FF0DFA92D
:101BF000930600010327810E63C496006F10905175
:101C0000B7060081938E464F13090001130A700036
:101C1000138B0E006F00C000938404FF6356990479
:101C2000938707011307170023A0680123A2280147
:101C30002326F10E2324E10E93888800E35EEAFC5C
:101C40001306410E93050C0013050D00EFA0903113
:101C500063100576938404FF8327C10E0327810E4A
:101C60009308C110E34E99FA930E0B00B3879700C7
:101C70001307170023A0D80123A298002326F10EF2
:101C80002324E10E93067000E3D8E6A01306410E6C
:101C900093050C0013050D00EFA0D02C631A0570FE
:101CA0008327C10E6FF05F9F13050D00EF20903664
:101CB0006FF0CFF40327410193880C00A303010CBC
:101CC0008327070013074700232AE1002306F114A6
:101CD000930A1000930C1000130BC1146FF09F8C2B
:101CE00083274101A303010C93880C0003AB070079
:101CF00013894700E30E0B5A9307F0FF6394FD002E
:101D00006F10001013860D009305000013050B00E3
:101D1000232A9101EF6040742328A1008328410108
:101D2000631405006F10D03183270101232A21019C
:101D300023280100B38C67418347710C93CAFCFFD1
:101D400093DAFA412324010223220102232E010007
:101D5000B3FA5C01930D0000E3800786938A1A00B2
:101D60006FF09F8583440400136A4A006FF0CFFC34
:101D70008326410193770A0293880C0003A706008B
:101D800093864600232AD100E39E073693770A0103
:101D9000638407006F10C00593770A04638407000B
:101DA0006F10C03F137A0A2063140A006F104004BA
:101DB0008327C100130B04002300F7006FF05F912D
:101DC000834404009307C006E384F44C136A0A01B9
:101DD0006FF08FF603274101B787FFFF93C7078393
:101DE0002314F10C93074700232AF100032907006D
:101DF000B70700819387473593880C00232AF102A7
:101E0000930C0000936B2A00930720009304800733
:101E1000A303010C1307F0FF6386ED2033679901DC
:101E200013FAFBF7631E071E63940D266390071CCD
:101E300093FC1B00130B011BE39C0C28938A0C00E2
:101E400063D4BC01938A0D008347710C23280100E1
:101E50002324010223220102232E0100E39007F034
:101E60006FF08FF58344040093078006E38AF44201
:101E7000136A0A046FF04FEC9307B0028344040026
:101E8000A303F10C6FF04FEB83440400136A0A08BC
:101E90006FF08FEA83440400130714006394740105
:101EA0006F105072938604FD13040700930D000019
:101EB00063E6DAE88344040093972D00B387B70103
:101EC00093971700B38DD700938604FD1304140075
:101ED000E3F2DAFE6FF08FE68327410183440400CA
:101EE00083A9070093874700232AF10063D609E4FA
:101EF000B3093041136A4A006FF00FE483440400D1
:101F0000136A1A006FF04FE38347710C8344040097
:101F1000639407E293070002A303F10C6FF0CFE193
:101F200093880C00136A0A0193770A02E38E070C68
:101F300083274101138B7700137B8BFF03290B0051
:101F4000832C4B0093078B00232AF100937BFABF6D
:101F5000930700006FF0DFEB93880C00936B0A018E
:101F600093F70B02E388070C83274101138B77005B
:101F7000137B8BFF93078B00232AF10003290B00AF
:101F8000832C4B00930710006FF09FE883440400FC
:101F9000136A8A006FF04FDA93880C00136A0A0103
:101FA00093770A02E380070C83274101138B7700A4
:101FB000137B8BFF83274B0003290B0013078B0038
:101FC000232AE100938C0700E3C6070C9307F0FF78
:101FD000930B0A006384FD02B3679901937BFAF7C0
:101FE000639E070063920D02138A0B00930D00009D
:101FF000930C0000130B011B6FF05FE4E3920C3AAB
:1020000093079000E3EE273913090903A307211B67
:10201000138A0B00930C1000130BF11A6FF01FE2E0
:10202000930B0A0013071000E38AE7FC1307200054
:10203000638CE706130B011B1397DC019377790080
:1020400013593900938707033369270193DC3C0058
:10205000A30FFBFE3367990113060B00130BFBFF65
:10206000E31C07FC93F61B00638A06069306000335
:102070006386D7061306E6FF9307011BA30FDBFE5B
:10208000B38CC740138A0B00130B06006FF01FDBE5
:10209000130710006394E7006F10D014130720009B
:1020A000930B0A00E398E7F883264103130B011B07
:1020B0009377F900B387F60003C707001359490067
:1020C0009397CC0133E9270193DC4C00A30FEBFE7F
:1020D000B3679901130BFBFFE39C07FC9307011BFC
:1020E000B38C6741138A0B006FF05FD593065006DF
:1020F00063DC962C8326010F9305010A1305010B5F
:102100002328D10A8326410F232211052320F1041D
:10211000232AD10A8326810F2320010A2322010AC0
:10212000232CD10A8326C10F2324010A2326010A66
:10213000232ED10AEFF080768327010483284104FF
:102140006318054A0327810EB70600819386463837
:1021500023A0D800938717009306100013071700D9
:1021600023A2D8002326F10E2324E10E930670004B
:1021700093888800E3C6E63A0327C10C8326010250
:10218000635CD772032701038326C102938888000A
:1021900023ACE8FE0327810EB387D70023AED8FE19
:1021A000130717002326F10E2324E10E9306700077
:1021B000E3C0E60C032701029304F7FF635690CCBB
:1021C000930600010327810EE3DC96361309000114
:1021D000930C70006F00C000938404FFE3529936A3
:1021E00083268100938707011307170023A0D800D7
:1021F00023A228012326F10E2324E10E93888800D0
:10220000E3DCECFC1306410E93050C0013050D00F6
:10221000EFA04055631E05188327C10E0327810ECA
:102220009308C1106FF05FFB33895941635220C39B
:10223000130600018326810E63542607130E000146
:10224000930B70006F00C000130909FF635A2E053D
:1022500003278100938707019386160023A0E800D7
:1022600023A2C8012326F10E2324D10E93888800CF
:10227000E3DCDBFC1306410E93050C0013050D0097
:10228000EFA0404E63160512130E0001130909FF5B
:102290008327C10E8326810E9308C110E34A2EFBCB
:1022A00003278100B38727019386160023A0E80047
:1022B00023A228012326F10E2324D10E1306700039
:1022C000938888006356D6B81306410E93050C0018
:1022D00013050D00EFA00049631C050C8327C10EF8
:1022E0009308C1106FF0CFB6130600018326810E4C
:1022F0006352B607930B0001130970006F00C00012
:10230000938D0DFF63D8BB050327810093870701D9
:102310009386160023A0E80023A278012326F10E5D
:102320002324D10E93888800E35CD9FC1306410E68
:1023300093050C0013050D00EFA0C042631A0506BB
:10234000938D0DFF8327C10E8326810E9308C11044
:10235000E3CCBBFB03278100B387B701938616004C
:1023600023A0E80023A2B8012326F10E2324D10ED6
:1023700013067000938888006350D6AE1306410E92
:1023800093050C0013050D00EFA0C03D631205027C
:102390008327C10E9308C1106FF00FAC1306410ED6
:1023A00093050C0013050D00EFA0C03B630205B0C0
:1023B000832B010163880BB293850B0013050D007D
:1023C000EF20C05D6FF00FB28326810E938C170053
:1023D000832701021306100023A0680193841600CE
:1023E000138988006356F6389307100023A2F8007B
:1023F0002326910F2324910E9307700063CE9774C8
:102400008327C1020327010393841400B38CFC00CB
:102410002322F9002320E9002326910F2324910E83
:10242000930770001309890063CA97748327010F0B
:10243000138614009305010A2328F10A8327410F0C
:102440001305010B232EC100232AF10A8327810FD4
:102450002320010A2322010A232CF10A8327C10F1A
:102460002324010A2326010A232EF10AEFF0004358
:102470000326C10183270102930889009306060001
:10248000938DF7FF630A053013071B00B38CBC0163
:102490002320E9002322B9012326910F2324C10E12
:1024A0009307700063CCC7509307090193862400FB
:1024B0001389080093880700032681031307410D41
:1024C0002320E900B30796012322C9002326F10E39
:1024D0002324D10E130770006358D79A6FF04FEF83
:1024E00037070081130600018326810E930E474FA4
:1024F000635C0609232081042322910413040D0048
:1025000093040C00130E000193027000130C0800DA
:10251000138D0E006F00C000130C0CFF635A8E0564
:10252000938707019386160023A0A80123A2C80160
:102530002326F10E2324D10E93888800E3DED2FCFB
:102540001306410E9385040013050400EFA08021BB
:102550006312057A130E0001130C0CFF8327C10EC2
:102560008326810E9308C11093027000E34A8EFB0C
:1025700013080C00930E0D00138C0400130D0400BF
:102580008324410403240104B387070193861600C2
:1025900023A0D80123A208012326F10E2324D10E63
:1025A00013067000938888006344D6006FF0CF82D2
:1025B0001306410E93050C0013050D00EFA0801AC1
:1025C000E31805DE8327C10E9308C1106FF0CF809A
:1025D0001306410E93050C0013050D00EFA08018A3
:1025E000E31805DC8327C10E9308C1106FF0CF8577
:1025F0008325C10C635CB0660327C10183260102F9
:102600009304070063C2E638635690028326810E66
:10261000B387970023A068019386160023A2980031
:102620002326F10E2324D10E130670009388880010
:10263000E342D63293C6F4FF0327C10193D6F64195
:10264000B3F4D400B3049740634490480327C10116
:1026500093760A40B30DEB00E398060C8324C10C7B
:102660000327010263C6E40093761A00E38806306C
:10267000832601030327C1021306700023A0D8009C
:102680008326810EB387E70023A2E8009386160015
:102690002326F10E2324D10E938888006354D6009C
:1026A0006F108017832601023307DB00B384964046
:1026B0003307B741138904006354970013090700D7
:1026C000635820030327810EB387270123A0B80195
:1026D0001307170023A228012326F10E2324E10E5D
:1026E000930670009388880063D4E6006F10801C06
:1026F0001347F9FF1357F7413377E900B384E440F8
:10270000634490006FE05FF8930600010327810E99
:1027100063D8966213090001930C70006F00C0002B
:10272000938404FF635E9960832681009387070189
:102730001307170023A0D80023A228012326F10E97
:102740002324E10E93888800E3DCECFC1306410EA1
:1027500093050C0013050D00EFA0C000E31A05C49B
:102760008327C10E0327810E9308C1106FF05FFB12
:1027700093771A00E39A07C623A2C8002326910F75
:102780002324910E9307700063CA97229386260034
:10279000938808016FF05FD2E350B0D313070001B4
:1027A0006344B7016F108061130B7000930406003F
:1027B0006F000001938D0DFF635EB71D93841400BD
:1027C00083278100938C0C012322E9002320F90048
:1027D0002326910F2324910E13098900E35C9BFCAF
:1027E0001306410E93050C0013050D00EF90907732
:1027F000E31005BC832CC10E8324810E1309C11084
:10280000130700016FF01FFB8326410193770A0134
:10281000138746006392071693770A046384076858
:1028200083274101930C0000232AE10003D907000C
:102830006FF0CFF18326410193F70B011387460018
:10284000639E070C93F70B04638E07608327410197
:10285000930C0000232AE10003D90700930710001E
:102860006FF00FDB8326410193770A01138746003F
:10287000639A070E93770A046386076083274101F2
:10288000232AE10003990700935CF94193870C0028
:1028900063DE07F2B3372001B30C9041B38CFC40E8
:1028A0009307D002A303F10C33092041930B0A00D4
:1028B000930710006FF00FD613771A006314070008
:1028C0006FE09FDC6FF01F8C93880C006FF04FED72
:1028D00093070003A307F11A130BF11A6FF00FD639
:1028E0008327C10383440400639407006FE0DFC4BF
:1028F00083C70700639407006FE01FC4136A0A4090
:102900006FE09FC38326C100130B040093D7F641E9
:102910002320D7002322F7006FE09FDB03A90600E6
:10292000930C0000232AE100930710006FF04FCEB4
:10293000032741018327070013074700232AE100EB
:1029400083A5070003A6470083A6870083A7C700C7
:102950002328B10E232AC10E232CD10E232EF10ED3
:102960006FE05FEF03A90600232AE100935CF941C1
:1029700093870C006FF04FE503A90600930C00004D
:10298000232AE1006FF08FDC93840600E34090C8B7
:102990006FF05FCA938614001307890083278100B4
:1029A000B38CBC012322B9012320F9002326910F07
:1029B0002324D10E9307700063DED7741306410EF3
:1029C00093050C0013050D00EF90D059E312059EFE
:1029D0008326810E832CC10E930841119386160025
:1029E0001309C1106FF05FAD93880C00930B0A00C0
:1029F0006FF00FD7B70700819387473593880C0096
:102A0000232AF10293770A02638807128327410180
:102A1000138B7700137B8BFF03290B00832C4B0058
:102A200093078B00232AF10093771A00638E070027
:102A3000B3679901638A0700930700032304F10C2D
:102A4000A304910C136A2A00937BFABF930720001A
:102A50006FF00FBCB70700819387873693880C000F
:102A6000232AF1026FF01FFA93880C006FF0CFCB8E
:102A70001306410E93050C0013050D00EF90904EC8
:102A8000E31805928327C10E9308C1106FF08FF2EF
:102A900083441400136A0A02130414006FE0DFA9D0
:102AA00083441400136A0A20130414006FE0DFA8A3
:102AB00093076000938C0D0063EEB76B37070081BE
:102AC000938A0C00232A2101130BC7376FE09FADB7
:102AD000130600018326810E63549640930C000177
:102AE000930D70006F00C000938404FF63DA9C3E76
:102AF00003278100938707019386160023A0E8002F
:102B000023A298012326F10E2324D10E9388880056
:102B1000E3DCDDFC1306410E93050C0013050D00EC
:102B2000EF905044E31605888327C10E8326810E5B
:102B30009308C1106FF05FFB8326410193770A0170
:102B4000138746006380071C03A90600930C00004E
:102B5000232AE1006FF05FED1306410E93050C0090
:102B600013050D00EF901040E3140584832CC10E73
:102B70008324810E1309C1106FF09F881306410E44
:102B800093050C0013050D00EF90D03DE312058274
:102B9000832CC10E8324810E1309C1106FF01F898D
:102BA000130B011B9307000023288100232E9100A3
:102BB00013040B0023223103130B0C0093040900B0
:102BC00093890C0013FA0B40832CC103930AF00F76
:102BD000138C0800138907006F0040021306A00041
:102BE000930600001385040093850900EFD0807CD4
:102BF000E38A092A93040500938905001306A000BF
:102C0000930600001385040093850900EFD0D03DA2
:102C100013050503A30FA4FE130919001304F4FF01
:102C2000E30E0AFA83C60C00E31AD9FAE30859FB4B
:102C30006392094A9307900063EE974893080C004B
:102C40009307011B130C0B00130B0400232E91039D
:102C50008324C1018329410203240101232021038C
:102C6000B38C6741138A0B006FF04F9D8326810E52
:102C7000370600811306463823A0C8009387170043
:102C8000130610009386160023A2C8002326F10E17
:102C90002324D10E13067000938888006344D6481D
:102CA000638405006FE0DFEA0327010293761A00D0
:102CB000B3E6E600639406006FE01F9D83260103E0
:102CC0000327C1021306700023A0D8008326810EBB
:102CD000B307F70023A2E800938616002326F10E1F
:102CE0002324D10E6354D6006FE09FE993888800B7
:102CF0006FE0DFEB832B0101130D0400138C040044
:102D00006FF04FEB93770A04638007148327410128
:102D1000930C0000232AE10003D907006FF0DFD0F5
:102D20001306410E93050C0013050D00EF90902340
:102D3000631005E88327C10E9308C1106FF0CFC35D
:102D400083268100B387970023A2980023A0D80090
:102D5000130717002326F10E2324E10E93067000BB
:102D600063C4E6006FE01F926FE09FE68327010FC8
:102D70009305010A1305010B2328F10A8327410F4C
:102D80002320010A2322010A232AF10A8327810F23
:102D90002324010A2326010A232CF10A8327C10FC9
:102DA000232EF10AEFE0905083280101E34005262D
:102DB0008347710C130770046358973837070081F5
:102DC000130B87342328010023240102232201024C
:102DD000232E0100137AFAF7930A3000930C300087
:102DE000930D0000638407006FE05FF76FE0CFFC96
:102DF0008327C100130B04002320F7006FE05F8DD1
:102E000013050B0023209105EF6050528347710C8E
:102E1000934AF5FF93DAFA41232A2101232801007E
:102E20002324010223220102232E0100832801040E
:102E3000930C0500B37A5501930D000063840700DD
:102E40006FE0DFF16FE04FF793770A206382073A74
:102E500083274101930C0000232AE10003C90700E6
:102E60006FF09FBC93F70B206388073683274101DF
:102E7000930C0000232AE10003C907009307100008
:102E80006FE01FF993770A20638C07328327410193
:102E9000232AE10003890700935CF94193870C0022
:102EA0006FF08F9293770A20638207308327410166
:102EB000930C0000232AE10003C907006FF00F897B
:102EC0008327C10F63CA07348347710C130770044B
:102ED000E35C971C37070081130B07356FF09FEEFB
:102EE00003278100B38797009386160023A0E8008C
:102EF00023A298002326F10E2324D10E130670007E
:102F0000938888006354D6F41306410E93050C0091
:102F100013050D00EF901005631C05C88327C10E33
:102F20009308C1106FF08FF203270102832C410236
:102F3000232E410123208104232231052322510322
:102F40008329810223246103B30BEB000324C10313
:102F5000032A8104832AC104930470001309000129
:102F6000130B0C0063880C08639809081304F4FF22
:102F7000938CFCFF0327810EB387470123A05801E0
:102F80001307170023A248012326F10E2324E10E84
:102F90009388880063CEE40E834604003386BB41E9
:102FA000138C06006354D600130C0600635680038E
:102FB0008326810EB387870123A0B801938616006C
:102FC00023A288012326F10E2324D10E63C2D40E3E
:102FD00083460400938888001346FCFF1356F6418D
:102FE0003377CC00338CE640634C8001B38DDD0039
:102FF000E39C0CF6638A095E9389F9FF6FF09FF7F3
:103000008326810E634889016F008005130C0CFF35
:10301000635889050327810093870701938616006B
:1030200023A0E80023A228012326F10E2324D10E99
:1030300093888800E3DCD4FC1306410E93050B0053
:1030400013050D00EF90007263140566130C0CFF5E
:103050008327C10E8326810E9308C110E34C89FBA0
:1030600003278100B38787019386160023A0E80019
:1030700023A288012326F10E2324D10E63C0D46637
:103080008346040093888800B38DDD006FF05FF6FF
:103090001306410E93050B0013050D00EF90806C95
:1030A000631805608327C10E9308C1106FF0DFEE2F
:1030B0001306410E93050B0013050D00EF90806A77
:1030C0006318055E834604008327C10E9308C11070
:1030D0006FF09FF0832781048325C104130900004A
:1030E0003304F4401386070013050400EF60D02C6E
:1030F00083C51C001306A000930600003338B000FF
:103100001385040093850900B38C0C01EFD0802A4D
:103110006FF05FAE938616009308870013090700CF
:103120006FF08FB91306410E93050C0013050D00C7
:10313000EF904063631E05A68325C10C8327C10E53
:103140009308C1106FF0DFB537070081130B4734C8
:103150006FF05FC71306410E93050C0013050D00B9
:10316000EF904060631605A48327C10E9308C11039
:103170006FF04FCC930C60006FF05F9483260102D8
:103180003307DB00B38496403308B741138904004A
:10319000635098D6130908006FF08FD58327C100BC
:1031A000130B04002310F7006FE08FD28327410137
:1031B000930C0000232AE10003A907006FE01FD948
:1031C00083274101232AE10003A90700935CF94109
:1031D00093870C006FE05FDF83274101930C0000B1
:1031E000232AE10003A90700930710006FE05FC2E4
:1031F00083274101930C0000232AE10003A9070063
:103200006FF09F821306410E93050C0013050D000D
:10321000EF9040556FE00FCD9307D002A303F10C60
:103220006FF0DFCA930700032304F10C93078005B6
:1032300013672A00A304F10C2324E102930730064C
:1032400023280100130BC114E3C4B7030323C10FE8
:1032500093FBF4FD23227105232C0104032E010F9F
:10326000832E410F032F810F136A2A10634E0344EC
:1032700093071006E38EF40A930710046384F400A6
:103280006FE04FE6930A010B13850A00232A11050C
:103290002328C10B232AD10B232CE10B232E610AF7
:1032A000EF10C12C1306C10CEF60803613860500A9
:1032B0009305050013850A00EF10010C8327010B0D
:1032C000930C010A130901092328F1088327410BF4
:1032D0001306010893050900232AF1088327810BAF
:1032E00013850C002320C104232CF1088327C10B74
:1032F0002320010823220108232EF108B707FC3FF1
:103300002326F10823240108EFE0900E0328010A88
:10331000032E410A832E810A032FC10A93850C00D4
:1033200013850A002328010B23280105232AC10B3A
:103330002322C103232CD10B2320D103232EE10B05
:10334000232EE1012320010A2322010A2324010A5A
:103350002326010AEFE08054032FC101832E0102CE
:10336000032E410203280105832841056316050049
:10337000930710002326F10CB70700819387873647
:103380002322F1029386FDFF232E4105232291067D
:103390002326B107232AA107232C81072320810696
:1033A0002324310723281107130C0B00938B0600ED
:1033B000232E6107130D0800930D0E0093840E0059
:1033C000130A0F006F00800493850C0013850A0018
:1033D0002320C102232EF101232CF10B232EC10A3D
:1033E0002328610B232A310B2320010A2322010AFF
:1033F0002324010A2326010AEFE0404A832FC1015A
:1034000003260102938BFBFF6302050EB7070340FF
:103410001306090093850C0013850A00232EF1087A
:103420002320A10B2322B10B2324910A2326410B35
:1034300023280108232A0108232C0108EFE0407B00
:1034400013850A00EF00114D9305050013040500D4
:1034500013850A008329010B8324410B032B810B65
:10346000032AC10BEF00515C0327010B0326010463
:10347000930509002320E1080327410B13850C0065
:10348000232831092322E1080327810B232A9108ED
:10349000232C61092324E1080327C10B232E4109B2
:1034A0002326E108EFF0007583274102032B010A70
:1034B0008329410A3387870003470700832F810A46
:1034C0000326C10A232A81052300EC002328710565
:1034D0009307F0FF130C1C00130D0B00938D0900D4
:1034E00093840F00130A0600E390FBEE8328010784
:1034F00093030B00938209003709FE3F93850C006C
:1035000013850A0023201103232E8100032AC105FD
:1035100083244106032401062328710A232271060D
:10352000232A510A23205106232CF10B232EF105C7
:10353000232EC10A2320C1042320010A2322010AC9
:103540002324010A2326210BEFE00042930B0C00F9
:10355000832DC106032D4107032C8107032BC107CF
:1035600083298106832801026342A0488323410600
:1035700083220106832FC1050326010493850C00D5
:1035800013850A002328710A232A510A232CF10BE0
:10359000232EC10A2320010A2322010A2324010A1F
:1035A0002326210BEFE0802F8328010263180500FA
:1035B0008327C10193FC1700639A0C4283270105FE
:1035C0001306000393861700B386DB0063C8070069
:1035D000938B1B00A38FCBFEE39C76FFB3876B41DD
:1035E0002320F1026FE08FBE03270102130C0B00B2
:1035F000032B8102232E8102032AC101B306EB00B3
:103600000324010483294104832A410263E4B601AF
:103610006FF0CF84938D06006FF04F840327C101B4
:103620009307D0FF6344F70063DAED009384E4FF6F
:1036300093F7F4FD2322F1046FE0CFBB832701024F
:103640000327C1016340F72A83278102930C0700F7
:1036500093F71700638607008327C102B30CF700B6
:103660008327810293F70740638607008327C10100
:103670006342F05C93CAFCFF93DAFA41B3FA5C014F
:103680009304700623240102232201026FE04FC835
:103690008347710C930D0000638407006FE00FEC0B
:1036A0006FD09FF19307900063E697D46FF00FD926
:1036B000832B0101130C0B006FE0DFCF23244103A8
:1036C00023280100130A0900B707008033C36700ED
:1036D0009307D002232CF1046FF09FB91306410E1B
:1036E00093050B0013050D00EF90C007E31205FCD6
:1036F000834604008327C10E9308C110B38DDD00FB
:103700006FF01F8F930A010B9307010D1308C10D72
:103710001307C10C93860D001306200093850A0041
:1037200013050D002328C10B2320C105232AD10B2B
:103730002322D103232CE10B2320E103232E610A52
:10374000232E6100EF20D073930770040323C1017F
:10375000032F0102832E4102032E01048328010559
:10376000130B05006390FB088327810293F7170072
:103770006396072E930770040327C10D2322F104DB
:103780006FE04FA4930A010B1308C10D9307010DBD
:103790001307C10C93860D001306300093850A00B1
:1037A00013050D00232811052328C10B2320C10573
:1037B000232AD10B2322D103232CE10B2320E10365
:1037C000232E610A232E6100EF20906B0323C10199
:1037D000032F0102832E4102032E010483280105D9
:1037E000130B0500930760043309BB01639EFB269E
:1037F00083460B00930700036386F650930C010A7F
:103800008327C10C3309F9006FE00F969307D002AC
:10381000A303F10C6FF00FDA1306410E93050C00B1
:1038200013050D00EF801074630405006FE05FB8AE
:103830008324C10C8327C10E9308C1106FE09FE65B
:103840008347710C232A2101232401022322010230
:10385000232E0100938A0D00938C0D00930D000020
:10386000638407006FE08FCF6FD01FD5832781025D
:103870000327C10193F71700B3E7B7016356E05080
:1038800063900744832CC10193046006832781025F
:1038900093F707406392073A93CAFCFF93DAFA4121
:1038A000B3FA5C016FF01FDE37070081130BC734DA
:1038B0006FF04FD11306410E93050C0013050D0058
:1038C000EF80506A630405006FE09FAE8324C10C53
:1038D000032701028327C10E9308C110B304974048
:1038E0006FE01FE1832701020327C10293047006E2
:1038F000B38CE7008327C101E34AF0F8B38CFC40A6
:10390000938C1C0093CAFCFF93DAFA41B3FA5C0172
:103910006FF05FD7B7060081938E464F6FE00FB50B
:103920009307F0FF2326F1006FD0DFDC130600FFC2
:10393000B304B04063D2C50613090001930C7000B4
:103940006F00C000938404FF63589904032781002B
:10395000938707019386160023A0E80023A228017D
:103960002326F10E2324D10E93888800E3DCDCFCAF
:103970001306410E93050C0013050D00EF80905EB9
:10398000630405006FE0DFA28327C10E8326810E4A
:103990009308C1106FF01FFB03278100B3879700C6
:1039A0009386160023A0E80023A298002326F10E98
:1039B0002324D10E13067000635AD6B21306410EAB
:1039C00093050C0013050D00EF80D059630405002A
:1039D0006FE01F9E8327C10E8326810E9308C110BE
:1039E0006FE0CF9C930B0A006FE00FE28327410545
:1039F00093860B00232EF10C8327410203C6FBFFA5
:103A000083C5F7006310B60213050003A38FA6FE5B
:103A10008326C10D9387F6FF232EF10C03C6F6FF14
:103A2000E386C5FE930516001305900393F5F50F85
:103A30006306A600A38FB6FE6FF05FBA832741022C
:103A400083C5A700A38FB6FE6FF05FB9930700038D
:103A50002304F10C930780076FF08FFD9307700428
:103A60003309BB012322F104930C010A6FD0DFEF6D
:103A700093851D0013050D0023281101EF40001B45
:103A800083280101130B0500630005362328A100DC
:103A90006FF0CFFB63940D00930D10000323C10F53
:103AA000032E010F832E410F032F810F13690A107C
:103AB000E34603C0930A010B1308C10D9307010DE0
:103AC0001307C10C93860D001306200093850A008E
:103AD00013050D00232211052328C10B2320C10546
:103AE000232AD10B2322D103232CE10B2320E10332
:103AF000232E610A232E6100EF2090380323C10199
:103B000023244103032F0102832E4102032E0104CB
:103B100083284104130B0500130A0900232C010418
:103B2000232801006FF05FC4930D60006FD0DFD8D1
:103B3000930A010B13850A00232A11052328C10BC0
:103B4000232AD10B232CE10B232E610AEF00112233
:103B50001306C10CEF50D02B13860500930505000A
:103B600013850A00EF0051018327010B930C010A12
:103B7000130901092328F1088327410B13060108C3
:103B800093050900232AF1088327810B13850C0074
:103B90002320C104232CF1088327C10B2320010813
:103BA00023220108232EF108B707FC3F2326F10842
:103BB00023240108EFE0C0030328010A032E410A71
:103BC000832E810A032FC10A93850C0013850A00F6
:103BD0002328010B23280105232AC10B2322C1031B
:103BE000232CD10B2320D103232EE10B232EE10123
:103BF0002320010A2322010A2324010A2326010A81
:103C0000EFD0D049032FC101832E0102032E4102C0
:103C1000032801058328410563160500930710005A
:103C20002326F10CB7070081938747352322F10241
:103C30006FF04FF5930470060326C1039306F00F4F
:103C400083470600638AD71A0327C10113050000C2
:103C50009305000063DEE7003307F7408347160053
:103C6000638407049385150013061600E394D7FEBA
:103C7000232EC102232EE1002322B1022324A1021C
:103C80000327810283274102B387E70003278104CA
:103C9000B387E702B38C970193CAFCFF93DAFA412A
:103CA000B3FA5C016FD0DFE6834706001305150009
:103CB0006FF0DFFB23280100138A07006FF0DFA0FD
:103CC0008327C10293046006B30CF700B38CBC01D8
:103CD0006FF0DFBB9306610D6318060093060003C7
:103CE000230BD10C9306710D1307011B9387070358
:103CF0003386E6402380F6009307D60D232CF1028D
:103D00006FD0DFDC930C010A93850C0013850A0049
:103D1000232811052328C10B2320C105232AD10BF9
:103D20002322D103232CE10B2320E103232E610A5C
:103D3000232E61002320010A2322010A2324010AE1
:103D40002326010AEFD090350323C101032F01027E
:103D5000832E4102032E010483280105E30205AAF4
:103D600093071000B387B7412326F10C3309F900FC
:103D70006FD09FBF8327810293F7170063940700DA
:103D80006FD0DFD66FD01FD6639A0700930A10005A
:103D900093046006930C10006FF0DF8E8327C1023E
:103DA00093046006938C1700B38CBC0193CAFCFF8C
:103DB00093DAFA41B3FA5C016FF0DF8C13870800E5
:103DC0006FE0DFBD8327410183AD07009387470084
:103DD00063D40D00930DF0FF83441400232AF100F7
:103DE000130407006FD04FF58357CC0093E7070407
:103DF0002316FC006FD01F8F23240102232201020F
:103E00006FF01FE893072000232CF1026FD01FCC26
:103E10003727008193070500032587BB930606001B
:103E200013860500938507006FD08FD583D7C50013
:103E300003AE450603D3E50083A8C50103A84502E8
:103E4000130101B893F7D7FF13070040232C8146D5
:103E5000231AF100138405009307010793058100DD
:103E6000232A914623282147232E114613090500B2
:103E70002326C107231B61002322110323260103EC
:103E80002324F100232CF1002328E100232EE1005C
:103E900023200102EFD0CFCE93040500635C05021E
:103EA0008357410193F70704638807008357C400D1
:103EB00093E707042316F4008320C14703248147B6
:103EC0000329014713850400832441471301014856
:103ED000678000009305810013050900EF00C058BA
:103EE000E30005FC9304F0FF6FF09FFBB727008110
:103EF00083A787BB130101FF2324810023229100A4
:103F0000232611009304050013840500638607002F
:103F100003A787036300070E0317C4009317070165
:103F20009376870093D707016380060483260401F4
:103F30006380060613F6170063040608032644018F
:103F400023240400130500003306C040232CC400C2
:103F5000638606088320C100032481008324410076
:103F6000130101016780000093F607016384060CCA
:103F700093F74700639607088326040113678700B9
:103F8000931707012316E40093D70701E39406FA79
:103F900013F6072893050020E30EB6F893050400F6
:103FA00013850400EF3090360317C4008326040104
:103FB0009317070193D7070113F61700E31006F8CC
:103FC00013F62700930500006314060083254401BF
:103FD0002324B40013050000E39E06F693F70708B8
:103FE000E38A07F6136707042316E4001305F0FFBE
:103FF0006FF05FF613850700EF00D0016FF0DFF17F
:1040000083250403638E0500930704046388F50089
:1040100013850400EF0090180317C400232804023E
:10402000832604011377B7FD232204002320D40044
:104030006FF0DFF49307900023A0F40013670704E8
:104040002316E4001305F0FF6FF0DFF0B7170081CF
:1040500003A7470283278714638C070403A747003D
:104060001308F001634EE8061318270063060502E3
:10407000338307012324C30883A88718130610007D
:104080003316E600B3E8C80023A417192324D3107D
:10409000930620006304D5021307170023A2E7004C
:1040A000B387070123A4B700130500006780000051
:1040B0009307C7142324F7146FF05FFA83A6C71879
:1040C0001307170023A2E70033E6C60023A6C7188C
:1040D000B387070123A4B700130500006780000021
:1040E0001305F0FF67800000130101FDB717008181
:1040F000232C410103AA4702232021032326110276
:1041000003298A142324810223229102232E3101C0
:10411000232A5101232861012326710123248101CF
:1041200063000904130B0500938B0500930A10002C
:104130009309F0FF832449001384F4FF63420402CF
:1041400093942400B304990063840B0483A7441060
:10415000638077051304F4FF9384C4FFE31634FFF0
:104160008320C10203248102832441020329010226
:104170008329C101032A8101832A4101032B010103
:10418000832BC100032C8100130101036780000011
:104190008327490083A644009387F7FF638E870433
:1041A00023A20400E38806FA8327891833978A003C
:1041B000032C4900B377F70063920702E7800600FB
:1041C0000327490083278A1463148701E304F9F85D
:1041D000E38807F8138907006FF0DFF58327C91814
:1041E00083A544083377F700631C070013050B0011
:1041F000E78006006FF0DFFC232289006FF09FFA52
:1042000013850500E78006006FF09FFB8397C500CC
:10421000130101FE232C810023263101232E1100DE
:10422000232A91002328210193F687001384050097
:1042300093090500639A06103717000013070780DB
:1042400083A64500B3E7E7002396F5006354D01832
:1042500003278402630A070C83A4090093960701CD
:1042600023A00900139637018325C40193D60601C4
:104270006348061693061000130600001385090014
:10428000E70007009307F0FF630CF5188356C4009E
:10429000032784028325C40193F64600638E06003B
:1042A00083264400832704033305D5406386070033
:1042B0008327C4033305F540130605009306000069
:1042C00013850900E70007009307F0FF631EF51050
:1042D00003A709008317C400630807169306D001DB
:1042E0006306D700930660016314D70C832604018C
:1042F00037F7FFFF1307F77FB3F7E7002316F40044
:10430000232204002320D4008325040323A0990042
:10431000638C0500930704046386F5001385090088
:10432000EF00C06723280402130500008320C101A9
:104330000324810183244101032901018329C10050
:10434000130101026780000003A90501E30E09FCC7
:1043500083A405001397070113570701137737004C
:1043600023A02501B38424419307000063140700B0
:1043700083A745012324F400634890006FF0DFFA1F
:104380003309A900E35290FA832744028325C4012C
:10439000938604001306090013850900E7800700CF
:1043A000B384A440E34EA0FC8357C4001305F0FF80
:1043B00093E707048320C1012316F400032481013D
:1043C00083244101032901018329C1001301010252
:1043D0006780000003A7C503E34CE0E66FF0DFF45D
:1043E000032504056FF05FEB8357C40037F7FFFF29
:1043F0001307F77FB3F7E7008326040193970701BC
:1044000093D707412316F400232204002320D4006D
:1044100013973701E35A07EE2328A4046FF0DFEE69
:1044200083A70900E38407E61307D0016388E70246
:10443000130760016384E7028357C40093E707040E
:104440002316F4006FF09FEE37F7FFFF1307F77F97
:1044500083260401B3F7E7006FF0DFFA23A0990089
:10446000130500006FF09FEC130101FE232C810067
:10447000232E11001304050063060500832785031E
:10448000638007028397C500639607028320C101FA
:10449000032481011305000013010102678000005D
:1044A0002326B100EF0000378325C1008397C500A4
:1044B000E38E07FC13050400032481018320C1015E
:1044C000130101026FF09FD49305050063080500F6
:1044D000B727008103A587BB6FF01FF9B7170081CD
:1044E00003A54702B7450080938585466F00900677
:1044F0001305000067800000B7E50080938545C57F
:104500006F005005130101FEB7470080232E1100F4
:10451000232C8100232A9100232821012326310105
:10452000232441012322510123206101032445005A
:104530009387874F232EF5021307C52E930730006C
:104540002324E52E2322F52E2320052E9307400059
:10455000130905002326F4001306800093050000CC
:104560002322040623200400232204002324040021
:1045700023280400232A0400232C04001305C40567
:10458000EFC05FC9379B008083248900B7AA0080F1
:1045900037AA0080B7A90080130B4B7A938A8A80D0
:1045A000130A0A899389898FB707010023206403BE
:1045B000232254032324440323263403232E84007C
:1045C0009387970023A6F40013068000930500004C
:1045D00023A2040623A0040023A2040023A40400B1
:1045E00023A8040023AA040023AC04001385C405F7
:1045F000EFC05FC20324C900B707020023A0640311
:1046000023A2540323A4440323A6340323AE94001B
:10461000938727012326F400232204062320040085
:10462000232204002324040023280400232A040056
:10463000232C04001305C405130680009305000015
:10464000EFC05FBD8320C1012320640323225403F4
:104650002324440323263403232E840003248101CE
:1046600093071000232CF90283244101032901013F
:104670008329C100032A8100832A4100032B010002
:10468000130101026780000013050000678000002D
:10469000130101FF23229100130680069384F5FF86
:1046A000B384C4022320210113890500232481003F
:1046B0002326110093854407EF304057130405006B
:1046C000630005021305C5002320040023222401F2
:1046D0002324A4001386840693050000EFC09FB333
:1046E0008320C100130504000324810083244100BA
:1046F000032901001301010167800000130101FE7D
:10470000B71700812328210103A94702232631017D
:10471000232E110083278903232C8100232A910053
:10472000930905006386070A1309092E9304F0FF15
:1047300083274900032489009387F7FF63D8070084
:104740006F00000813048406638C97060317C400E7
:104750009387F7FFE31807FEB707FFFF938717005C
:10476000232204062320040023220400232404001F
:104770002326F40023280400232A0400232C040009
:1047800013068000930500001305C405EFC09FA821
:1047900023280402232A04022322040423240404D9
:1047A0008320C101130504000324810183244101F6
:1047B000032901018329C100130101026780000060
:1047C00003240900630C0400130904006FF05FF672
:1047D00013050900EFF01FD36FF01FF5930540009C
:1047E00013850900EFF0DFEA2320A9001304050078
:1047F000E31C05FC9307C00023A0F9006FF05FFAEB
:10480000B717008103A54702B7E50080938545C52A
:104810006F0040548327850363840700678000008E
:104820006FF05FCE67800000678000006780000047
:1048300067800000B727008103A587BBB7450080CC
:104840009385054F6F00C046B727008103A587BB3E
:10485000B7450080938585686F008045130101FE90
:1048600023263101B7190081232C8100232A9100CE
:104870002328210123244101232E1100138A05003E
:10488000130905009389497AEF30504A03A789003C
:10489000B71700001384F7FE832447003304444114
:1048A00093F4C4FF330494001354C4001304F4FFBE
:1048B0001314C400634EF4009305000013050900AF
:1048C000EF40104F83A78900B38797006308F50274
:1048D00013050900EF30D0458320C1010324810175
:1048E00083244101032901018329C100032A810096
:1048F000130500001301010267800000B30580402A
:1049000013050900EF40D04A9307F0FF630AF5044E
:10491000B7270081938787C403A7070083A6890070
:10492000B384844093E414003304874013050900E2
:1049300023A2960023A08700EF30903F8320C1017F
:104940000324810183244101032901018329C1003A
:10495000032A810013051000130101026780000083
:104960009305000013050900EF40904403A7890058
:104970009306F000B307E540E3DCF6F4B7260081C8
:1049800083A6C6BB93E717002322F7003305D54063
:10499000B726008123A4A6C46FF09FF3638A051293
:1049A000130101FF232481002322910013840500B9
:1049B0009304050023261100EF3050370328C4FF6D
:1049C000130784FFB71500819377E8FF3306F700DC
:1049D0009385457A8326460003A5850093F6C6FF96
:1049E000630AC51A2322D600137818003305D600AF
:1049F0006310080A032384FF03284500371500814C
:104A000033076740832887001305C57AB38767009B
:104A1000137818006380A8140323C70023A6680036
:104A2000232413016304081E93E617002322D700F2
:104A30002320F6009306F01F63E8F60A93F687FF3B
:104A40009386860003A54500B386D50003A606001D
:104A500013D8570093071000B3970701B3E7A700D7
:104A6000138586FF2326A7002324C70023A2F50071
:104A700023A0E6002326E600032481008320C10052
:104A80001385040083244100130101016F30502A73
:104A90000325450013751500631E050237150081B7
:104AA000B387D7001305C57A8326860093E81700DD
:104AB0003308F7006388A6160326C60023A6C6009F
:104AC0002324D600232217012320F8006FF09FF63D
:104AD0006780000093E61700232ED4FE2320F60003
:104AE0009306F01FE3FCF6F493D6970013064000FC
:104AF000636CD60E93D667001388960313868603DD
:104B0000131838003388050183260800130888FF2E
:104B10006308D81203A646001376C6FF63F6C700E3
:104B200083A68600E318D8FE03A8C6002326070143
:104B30002324D700032481008320C1002324E8001C
:104B4000138504008324410023A6E600130101011C
:104B50006F30101E631608148325C60003268600D6
:104B6000B387F600032481002326B60023A4C500E2
:104B700093E617008320C1002322D7001385040089
:104B80003307F700832441002320F70013010101BC
:104B90006F30101A13781800B387D700631008021B
:104BA000032584FF3307A7408326C7000326870019
:104BB000B387A7002326D60023A4C600B72600810A
:104BC00013E6170083A606BC2322C70023A4E50032
:104BD000E3E4D7EAB727008183A507C8138504005B
:104BE000EFF0DFC76FF05FE9130640016374D60290
:104BF000130640056364D60693D6C7001388F606ED
:104C00001386E606131838006FF0DFEFB387D7007E
:104C10006FF09FE91388C6051386B6051318380090
:104C20006FF05FEE23AAE50023A8E5002326A70086
:104C30002324A700232217012320F8006FF0DFE3CD
:104C400003A5450013562640930710003396C7006E
:104C50003366A60023A2C5006FF05FED1306401572
:104C6000636CD60093D6F700138886071386760701
:104C7000131838006FF01FE913064055636CD60017
:104C800093D627011388D6071386C6071318380052
:104C90006FF05FE71308803F1306E0076FF09FE6B1
:104CA00093E617002322D7002320F6006FF0DFDC05
:104CB000130101FE23282101232631012324410170
:104CC0002322510123206101232E1100232C810076
:104CD000232A9100138B0500930A052E130A000066
:104CE000930910001309F0FF83A44A0003A48A006B
:104CF0009384F4FF63C604028357C4009384F4FFD3
:104D000063FCF9008317E4001305040063862701A0
:104D1000E7000B00336AAA0013048406E39E24FD17
:104D200083AA0A00E3920AFC8320C10103248101C3
:104D300083244101032901018329C100832A410001
:104D4000032B010013050A00032A8100130101024D
:104D500067800000130101FD23202103232E310170
:104D6000232C4101232A51012328610123267101AB
:104D7000232611022324810223229102930A050093
:104D8000938B0500130B052E130A000093091000E6
:104D90001309F0FF83244B0003248B009384F4FF5A
:104DA00063C804028357C4009384F4FF63FEF900D0
:104DB0008317E4009305040013850A006386270126
:104DC000E7800B00336AAA0013048406E39C24FDE9
:104DD000032B0B00E3100BFC8320C1020324810290
:104DE00083244102032901028329C101832A41014D
:104DF000032B0101832BC10013050A00032A810143
:104E0000130101036780000093064500930700002B
:104E10001305A5013788FFFF6F00C00193971700A6
:104E20002390E600939707019386260093D7070106
:104E3000630ED50203D7060013761700630406003D
:104E400093E717001357170013F62700B365070100
:104E5000E30606FC939717002390B600939707018B
:104E60009386260093D70701E316D5FC67800000E0
:104E70009306850113070000130525006F00C0018C
:104E8000131717002390F600131707019386E6FF08
:104E9000135707016304D50483D70600139607014F
:104EA00013560641939717006354060013671700C3
:104EB0009397070193D707011376270093E517000F
:104EC000E30006FC131717002390B6001317070121
:104ED0009386E6FF13570701E310D5FC67800000B7
:104EE000130101FE370E0100231D0100231E0100E6
:104EF000938585019307C10113088100130EFEFFFE
:104F000003D705009387E7FF9385E5FF6318070242
:104F1000239F07FEE39607FF130646009306E10171
:104F200003D707009387270013062600231FE6FEFA
:104F3000E398D7FE13010102678000003307A70240
:104F400083D8270003D30700B376C701B3861601C1
:104F50001357070193D8060133076700330717017A
:104F6000935807012391D7002390E700239F17FF51
:104F7000E39807F96FF05FFA1307250183570500DF
:104F80001305250063980700E31AE5FE13050000EA
:104F9000678000001305100067800000130101FF07
:104FA000232291008354250123248100232611000C
:104FB00093C7F4FF13971701130405006316070046
:104FC000EFF09FFB63180500B787FFFFB3C4F40041
:104FD000231994008320C10003248100832441000D
:104FE0001301010167800000130101FF23248100E8
:104FF00003542501232611009347F4FF139717014B
:10500000631A0700EFF05FF7930705001305000030
:10501000639407001355F4008320C100032481002A
:10502000130101016780000083572501130101FD71
:105030002324810293D7F700232291022326110211
:1050400023202103232E3101B307F0402390F500E4
:1050500083572501378700001307F7FFB377F70061
:105060002391F50093040500130405016382E7040E
:1050700093876500239205001305E5FF035704009D
:105080001304E4FF93872700239FE7FEE31885FEC0
:10509000239C05008320C102032481028324410252
:1050A000032901028329C101130101036780000064
:1050B000035725011389450033F7E700631CF70206
:1050C0002326B100EFF05FEB8325C10063040502E6
:1050D00093876500239205001385C4FF03570400DE
:1050E0001304E4FF93872700239FE7FEE31885FE60
:1050F0006FF05FFA9389A50113092900231F09FEA8
:10510000E39C29FF8320C1020324810283244102FE
:10511000032901028329C1011301010367800000F3
:1051200083572501130101FB2324810493C7F7FF53
:1051300023229104232611041397170193040500D9
:105140001384050063160700EFF01FE363120508E0
:105150008357240193C7F7FF1397170163040706CA
:105160009305810013850400EFF01FEC93054102C5
:1051700013050400EFF05FEB8355810003554102F6
:10518000630CB5049307A100130761021306010223
:1051900083D6070093872700639A06088356070083
:1051A0001307270063940608E394C7FE1305000065
:1051B0008320C104032481048324410413010105D5
:1051C0006780000013050400EFF01FDBE30A05F819
:1051D0001305E0FF6FF0DFFD133515000356A10046
:1051E000835661023305A0401307A10093076102B3
:1051F000137525001305F5FF9305C1039387270059
:1052000013072700631ED600E382B7FA0356070090
:1052100083D607001307270093872700E306D6FEEF
:10522000E3E8C6F83305A0406FF09FF813051000BF
:10523000E38005F81305F0FF6FF09FF7130101FFFE
:1052400023261100EFF05FD38320C1001335150032
:105250001301010167800000130101FE232C81006E
:10526000232A9100232E1100232821012326310116
:10527000938405001304050063C4050A9307F00036
:105280001386050013054500930684019305F0007D
:1052900063D497029307050003D72700938727005D
:1052A000239FE7FEE39AD7FE231C0400130606FFA4
:1052B000E3C2C5FE93F4F4009307700063D897022D
:1052C0001307840193052400930700008356070009
:1052D0001307E7FF13968600B3E7C7002311F70013
:1052E00093D78600E314B7FE938484FF638A040097
:1052F0009384F4FF13050400EFF09FB7E39A04FED4
:10530000130500008320C10103248101832441018E
:10531000032901018329C1001301010267800000F4
:10532000930710FF3309B04063DCF5129305850144
:1053300093090000930645001306F000035784010B
:1053400093870500B3E9E90003D7E7FF9387E7FFF9
:105350002391E700E39AD7FE23120400130909FF03
:10536000E34E26FD930700FF130710FFB387974016
:105370001309000063C4E40A3309F90093077000BD
:1053800063D627059399090193D90941834784017D
:105390009305A401B3E9F9009399090193D909018F
:1053A0009307000003D60600938626001357860055
:1053B00033E7E7009317860093970701239FE6FEE4
:1053C00093D70701E390B6FE130989FF630C090622
:1053D000835784011309F9FF1305040093F717009D
:1053E000B3E93701EFF05FA2E31409FE93970901D7
:1053F00093D70741639007041395090113550501DD
:105400008320C10103248101832441010329010177
:105410008329C100130101026780000013F907FF0F
:10542000330920413309F90093077000E3D027FBCB
:105430006FF05FF5930910001395090113550501ED
:105440006FF01FFC1385090063980900131505010F
:10545000135505016FF01FEB130510006FF01FFFD0
:10546000930790FF93090000E3D4F5F693064400F8
:105470006FF0DFF183574500130101FF23229100F4
:1054800023261100232481002320210193040500F9
:10549000639C070C03576500130400009317070172
:1054A00093D7074163C4070A9306A5011306000AB0
:1054B00063180702938764006F00800003D707001A
:1054C00093872700239EE7FEE39AF6FE239C0400C1
:1054D00013040401630CC40603D76400E30C07FC47
:1054E000937707F063900704138584019385240064
:1054F0009307000013070500835607001307E7FF13
:1055000013968600B3E7C7002311F70093D78600F0
:10551000E394E5FE03D7640013048400937707F057
:10552000E38807FC1309000A6F004001130414000C
:10553000EFF01F94634C890003D764001317070131
:105540001357074113850400E35207FE8320C1006F
:105550001305040003248100832441000329010072
:10556000130101016780000013F707F01304000026
:10557000631007041309F0F66F0040011304F4FFF1
:10558000EFF09F88E30424FD83D7440013850400D3
:10559000E39607FE8320C100130504000324810065
:1055A00083244100032901001301010167800000E9
:1055B000930645009305A501130700006F008000C6
:1055C00083D7060013D687003367C70093978700F9
:1055D0002390E600139707019386260013570701CF
:1055E000E390B6FE83D74400130480FF6FF09FF86A
:1055F000130101FE232C8100232A9100232821017D
:10560000232631012324410123225101138906005D
:1056100093840700232E11001304050093890500CD
:10562000130A0600930A0700EFF0DFE4930700096E
:105630003309A94063DCA716B78700009387E7FF0B
:1056400063DA271F63840A1C03A5440083A70400B0
:10565000630AF5061387A401938744031307270001
:10566000231F07FEE31CF7FE93078003630CF5324C
:1056700063D0A71693070004630CF52E9307100759
:105680006318F534B78700409387F7FF1307A0002E
:1056900023AAF400B787FFFF23A4E400239CF400AF
:1056A00023A6E4009307A0003787000093878700B4
:1056B00093971700B387F4002395E70023A0A40075
:1056C0006358201B83A5840083D744011308F00886
:1056D000139615003306C40003570600B376F7008F
:1056E000634AA8021308B0006346B8029307060095
:1056F0009305840103D727006304070093E616008F
:105700002391070093872700E396F5FE03570600D1
:1057100083D7440193C7F7FFB3F7E7002310F600E0
:1057200083D7640133F7D700630007046384D71A73
:1057300013862403930684019384C4011307000095
:105740008357060083D506009386E6FF1306E6FF1F
:10575000B387B700B387E70013D707012391F6009B
:1057600013771700E31E96FC6358201983574400F3
:10577000639E0712B7870000231C04009387E7FF8E
:1057800063C82709231124018320C1010324810157
:1057900083244101032901018329C100032A8100D7
:1057A000832A410013010102678000006354090E3F
:1057B000930700F7635CF908930724001304A4011E
:1057C00093872700239F07FEE39C87FE6FF0DFFB94
:1057D000930780016308F51693075003631AF51EBB
:1057E00037170000B7070004930660009387F77F20
:1057F0001307078023AAF40023A4D400239CE40009
:1058000023A6D400930760006FF05FEA231C040016
:10581000B787FFFF93C7F7FF2311F40093074400F6
:10582000130484012390070093872700E31CF4FEF0
:105830006FF09FF5930724001304A40193872700BA
:10584000239F07FEE39C87FE6FF01FF4930509007A
:1058500013050400EFF05FA0630405009309100036
:10586000638C0A0C03A5440083A70400E314F5DE4F
:10587000930700096304F50A8357840113050400A4
:1058800093F71700B3E9F900EFF00FD803A5440030
:105890006FF05FE3E3800AEE03A5440083A70400F2
:1058A000E31AF5DAE34020E36FF09FFC13050400F0
:1058B000EFF08FD5B787000013091900231C0400EF
:1058C0009387E7FFE3C627F5E35E09EA23110400A7
:1058D0006FF09FEB6394090C83A7C40003D7840186
:1058E00093971700B307F40083D70700B3F7E700D7
:1058F000E39007E4E34C20E7930700096306F50013
:1059000013050400EFF0CFD683574400E39007FA65
:10591000231C0400E34C09FA6FF0DFE603A68400C1
:1059200083D74401131616003306C400035706003C
:10593000B3F6E7006FF01FDE231C04002311040000
:105940006FF09FE4B70780009387F70F13074000BD
:1059500023AAF4009307001023A4E400239CF4007E
:1059600023A6E40093074000130700106FF01FD434
:105970009307700023A4F400B70701809387F7FF13
:1059800023AAF40093071000239CF40093076000FF
:1059900023A6F400130710006FF05FD1E30A0AD8C2
:1059A0006FF09FDCB70780009387F70F1307600045
:1059B00023AAF4009307001023A4E400239CF4001E
:1059C00023A6E40093076000130700106FF01FCEBA
:1059D0009307C00023A4F400B70701809387F7FF63
:1059E00023AAF40093071000239CF4009307B0004F
:1059F00023A6F400130710006FF05FCB130101FD25
:105A000023229102232E310193840500835925001E
:105A1000232611022324810223202103232C410168
:105A200013090600232A510123286101232671014D
:105A300023248101232291012320A101130A0500BF
:105A4000EFF05FA303D4240093070500138504003F
:105A5000B389F940930A4903EFF0DFA13304A4406E
:105A60001307E90493870A0093872700239F07FE03
:105A7000E39CE7FE634A3409930B4A00138B44000E
:105A80009389F9FF930CAA01138C240013070B00D0
:105A900093870B0003D607008356070093872700E0
:105AA00013072700631AD60AE39697FF13068A01A5
:105AB000138784019306000083570700835506006F
:105AC0001307E7FFB387D740B387B74093D60701E3
:105AD0002311F70093F616001306E6FFE31EECFC15
:105AE000130D100013850A00EFF08FB88357C90417
:105AF0001304F4FF13850400336DFD002316A9057C
:105B0000EFF00FB7E31434F9930604000324810285
:105B10008320C1028329C101032A8101832A410113
:105B2000032B0101832BC100032C8100832C410036
:105B3000032D0100930709001385040003290102C6
:105B400083244102130700001306000093050000A0
:105B5000130101036FF0DFA9130D0000E3E4C6F8A1
:105B60006FF0DFF403570500835725006306070035
:105B700037870000B3E7E7002399F50003572500B6
:105B8000B78700009387F7FF6304F7029307650068
:105B9000938505011305850103D707009387270027
:105BA0009385E5FF2391E500E398A7FE6780000059
:105BB000930765001305A50103D707009387270006
:105BC000631A0702E39AA7FE13872501938705004E
:105BD00093872700239F07FEE31CF7FE83D7250149
:105BE000378700001307F7FFB3E7E7002399F500B5
:105BF00067800000138705019387050093872700BE
:105C0000239F07FEE31CF7FEB7C7FF7F23A8F5001D
:105C100067800000130101F723286107035B25015A
:105C2000B78700009387F7FF232C410733FA6701FA
:105C3000131A0A0123248108232291082320210911
:105C4000232E310723261108232A51072326710703
:105C50002324810723229107135A0A019304050084
:105C60001389050013040600938906006312FA10D5
:105C7000EFF08FB0631A0528835A2901B3775A01D0
:105C80006382472B13850400EFF04FDB630E052E74
:105C9000B70500819385C55313050900EFF04FC880
:105CA00063060536835A2901B78700009387F7FFFB
:105CB000B3FA5701939A0A0193DA0A016394FA2C12
:105CC00013050900EFF08FD76310053283D7240145
:105CD000B3F7FA006398570B13850400EFF00FD663
:105CE0006318050013050900EFF04FD5630C050894
:105CF00013850400EFF04FAF93040500130509006E
:105D0000EFF08FAEB384A440B33490009394F400CA
:105D10002319940013072401930704009387270095
:105D2000239F07FEE31CF7FE8357240137870000FB
:105D30001307F7FFB3E7E7002319F4008320C10836
:105D40000324810883244108032901088329C1070A
:105D5000032A8107832A4107032B0107832BC106EE
:105D6000032C8106832C4106130101096780000082
:105D700083DA250133F7570113170701135707017A
:105D8000630AF704138504009305C100EFF0CFA95F
:105D90001305090093058102EFF00FA98354E10078
:105DA0000359A102639C0404930701019306410275
:105DB0006388D72003D7070093872700E30A07FEED
:105DC0001305C100EFF00FEB0357A102B304A0408D
:105DD0006F00000313850500EFF00F9AE30605EC52
:105DE00013074901835709001309290013042400EC
:105DF000231FF4FEE318E9FE6FF05FF413070900B8
:105E0000930A09009307C102930601046312070273
:105E10006382F61C03D7070093872700E30A07FE77
:105E200013058102EFF00FE50357A102B30AA94061
:105E300083578102138C8903239BE902239AF90279
:105E40001387E90493070C0023900700938727002A
:105E5000E31CF7FE138AC904930B000013094102E7
:105E6000930C0101130B6104035509001309E9FFA9
:105E70006318050C03D7C90493070A00B3EBEB00C2
:105E800003D7E7FF9387E7FF2391E700E39A87FFB4
:105E9000239C0902E31A99FD1387490393078102A2
:105EA0009305210403560700938727001307270053
:105EB000239FC7FEE398F5FEB7C6FFFFB3845401E6
:105EC0009386260093850B001305810293870900B2
:105ED00013070004B386D40013060000EFF04FF15F
:105EE000035781028357C100930504001305810203
:105EF000B387E740B337F000B307F0402314F10253
:105F0000EFF05FC66FF09FE31387440183D704006F
:105F10009384240013042400231FF4FEE398E4FE7A
:105F20006FF0DFE113050900EFF00F85E31A05EAD2
:105F300013850400EFF08FB0E30805D66FF05FD54E
:105F40001306410493058102EFE09FF993050A00CF
:105F5000130600001307C10503D805008357070087
:105F60009385E5FF1307E7FFB3870701B387C700F2
:105F700013D607012391F50013761600E31E67FD83
:105F80006FF05FEF03DB2401B78700009387F7FF13
:105F900033FB6701131B0B01135B0B01E314FBDEE7
:105FA00013850400EFF08FA9E31405D4835729016A
:105FB00093C7F7FF13971701E31607DC6FF09FD223
:105FC0009307440113042400231F04FEE39C87FE6F
:105FD0006FF0DFD69307440113042400231F04FE4F
:105FE000E31CF4FE6FF09FD5B70500819385C55380
:105FF00013850400EFF0CF92630A050083D72401D4
:10600000B3F7FA00E38E57F96FF05FFA1307040154
:106010009307040093872700239F07FEE39CE7FE76
:10602000B7C7FF7F2328F4006FF05FD183572501A6
:10603000130101F52324810A93C7F7FF2322910A54
:106040002320210B232E31092326110A232C410959
:10605000232A510923286109232671092324810950
:10606000232291092320A109232EB1071397170199
:1060700013090500938905001304060093840600A4
:1060800063160700EFE05FEF6318053883D7290137
:1060900093C7F7FF13971701630E0708370A0081AC
:1060A0009305CA5313050900EFF08F8763040510A9
:1060B000035A290103D72901B78700009387F7FF07
:1060C00033FA4701B3FAE700631AFA081305090027
:1060D000EFF0CF966308051063984A011385090015
:1060E000EFF0CF956310050E9307440113042400CD
:1060F000231F04FEE31CF4FE8320C10A0324810A4B
:106100008324410A0329010A8329C109032A810939
:10611000832A4109032B0109832BC108032C810821
:10612000832C4108032D0108832DC1071301010BA6
:106130006780000013850900EFE01FE4E30005F627
:106140001387490183D70900938929001304240088
:10615000231FF4FEE398E9FE6FF01FFA6386FA0846
:10616000130509009305C101EFE01FEC93058103BE
:1061700013850900EFE05FEB835BA1030359E101A5
:1061800063920B0C9307C103930D0105638EFD34DD
:1061900003D7070093872700E30A07FE130581034F
:1061A000EFF04FADB307A0400356E1012326F10005
:1061B0006F00C0099305CA5313850900EFE05FF62D
:1061C000E31805EE130704019307040093872700E3
:1061D000239F07FEE39CE7FEB7C7FF7F2328F40059
:1061E0006FF09FF1E39E4AF713850900EFF00F85EA
:1061F000E30805F613050900EFE01FDF930405002F
:1062000013850900EFE05FDEB387A440B337F000E9
:106210009397F7002319F400130724019307040050
:1062200093872700239F07FEE39CE7FE8357240103
:10623000378700001307F7FFB3E7E7002319F400DF
:106240006FF09FEB2326710113060900232421011F
:106250009307010293064103631206026380F62A44
:1062600003D7070093872700E30A07FE1305C10140
:10627000EFF04FA0B307A9402324F10003278103C7
:10628000138D840393070D0023AAE4021389E40409
:1062900093872700239F07FEE31CF9FE1305810364
:1062A000EFE09FB6035C2102370A0100930D010560
:1062B000931A0C01B38A8A41130BA103130AFAFF44
:1062C000930CE106930961058357C1030357E1036A
:1062D000930B0A0093970701B387E70063E8FA007E
:1062E000B3D78703939B070193DB0B01130641058B
:1062F0009305C10113850B00EFE09FBE1307C10397
:106300009307810583D5070003560700938727006D
:10631000130727006390C512E39697FF93070000C9
:106320009305C10613860D000357060003D8050028
:106330001306E6FF3307F74033070741935707017A
:106340002311E60093F717009385E5FFE31E66FD32
:1063500023107D019307C10303D7270093872700EC
:10636000239FE7FEE39AB7FF23180104130D2D00C6
:10637000E31CA9F5930500009307C10393062105CB
:1063800003D7070093872700B3E5E500E39AD7FE1C
:106390009397050193D70741638407009305100085
:1063A0009395050193D50501138744039307810352
:1063B000035607009387270013072700239FC7FE74
:1063C000E398F6FE8327C10003278100B74600004B
:1063D0009386F6FFB38BE740130581039387040090
:1063E00013070004B386DB0013060000EFF04FA094
:1063F000035781038357C1019305040013058103EB
:10640000B387E740B337F000B307F040231CF10235
:10641000EFF04FF56FF05FCE130749018357090086
:106420001309290013042400231FF4FEE318E9FED6
:106430006FF09FCCE374B6EE9387FBFF9398070150
:1064400093D8080193070000930541031306C10682
:106450000357060003D805001306E6FF3307F7408D
:1064600033070741935707012311E60093F71700FD
:106470009385E5FFE31E36FD1307C10393078105EE
:1064800083D50700035607009387270013072700CB
:106490006398C500E39697FF938B08006FF01FE8A1
:1064A000E37CB6FE9387EBFF939B070193DB0B0125
:1064B00013060000930541031307C1068357070025
:1064C00003D805001307E7FFB387C740B387074129
:1064D00013D607012311F700137616009385E5FF05
:1064E000E31E37FD6FF09FE393074401130424007C
:1064F000231F04FEE39C87FE6FF01FC00357C101FA
:10650000835781036304F700378600002319C40012
:10651000130724019307040093872700239F07FE96
:10652000E31CF7FE83572401378700001307F7FFAA
:10653000B3E7E7002319F4006FF01FBC130101FD5E
:1065400023248102232611021384050093074100AE
:106550001307E10193872700239F07FEE39CE7FED3
:106560000356E5009317060193D7074163CA070650
:10657000B78700009387F7FF231201003376F600F8
:10658000630CF6069307E5002313C1001307A1006F
:1065900083D6E7FF9387E7FF13072700231FD7FE64
:1065A000E318F5FE631206022314010093050400AC
:1065B00013054100EFF00FDB8320C10203248102A9
:1065C0001301010367800000930710009305F0FF9B
:1065D000130541002314F100EFE01FC86FF01FFD09
:1065E0009307F0FF2312F100B78700009387F7FFAE
:1065F0003376F600E318F6F8930705009306E500F6
:1066000003D7070093872700631C0704E39AD7FE8C
:10661000130744019307040093872700239F07FE75
:10662000E31CF7FE13072401930704009387270058
:10663000239F07FEE31CF7FE8357240137870000E2
:106640001307F7FFB3E7E7002319F4008317E5000A
:10665000E3D407F613050400EFE05F946FF0DFF575
:10666000130704019307040093872700239F07FE65
:10667000E31CF7FEB7C7FF7F2328F4006FF0DFF3BA
:1066800083A8C500130101E183AE050003AE4500F8
:1066900003A38500232E1103832505049308F0FF2F
:1066A00023201117930800092324811E232C411D48
:1066B0002326111E2322911E2320211F232E311D4C
:1066C000232A511D2328611D2326711D2324811D8A
:1066D0002322911D2320A11D232EB11B2328D1038A
:1066E000232AC103232C6102232211172320C10076
:1066F0002324D1002326E100232C0101130A0500E5
:1067000013840700638005020327450493071000E4
:10671000B397E70023A2E50023A4F500EF10106C67
:1067200023200A0493090106938509001305010338
:10673000EFF0DFE013850900EFE01F8B0327010076
:106740003335A0002320A40093073000E302F714A0
:10675000930740012322F100E318075E83572107C6
:106760000327411693C7F7FF232AE1001397170168
:106770006318070013850900EFE01F80E31405404C
:10678000930700092322F1161307C1079387090015
:106790001306410783D607009387270013072700B6
:1067A000231FD7FEE398C7FE0356E1082328010004
:1067B0009317060193D7074163DE070013161601EE
:1067C000B7070100135616019387F7FF2317C10877
:1067D0002328F100370B0081930DCB53138C4D010F
:1067E000930600009307810913070C00130DC10ADB
:1067F0006F0080008356070093872700239FD7FEF2
:1068000013072700E398A7FF63080614B787000063
:106810009387F7FFE306F6568317C108E3D8075AB4
:106820009305C10713050C00EFE09F8F6302051469
:10683000E34C050C8357E108E39C07628317C1080A
:10684000930400001309011663C4070213848D1119
:106850001306C107930609009305060013050400FB
:10686000EFF04FBB8317C1089384F4FFE3D207FE18
:106870001304010D930B810E130704009307C10746
:106880001306010983D60700938727001307270003
:10689000231FD7FEE398C7FE9306000093078109E4
:1068A00013070C006F0080008356070093872700B2
:1068B000239FD7FE13072700E398A7FF938C8D0231
:1068C000138DCD12B7FAFFFF938D8D116F00C000AD
:1068D000130D4D01938C4C019305040013050C001E
:1068E000EFE01F84930705009305040013050D00D6
:1068F0006356F004EFE0DF8293070500930609007A
:10690000130604009305040013850C0063C00702FE
:10691000EFF04FB0130681099306090093050600B6
:1069200013850C00EFF00FAFB384540193D7FA0135
:10693000B387570193DA1740E39CBCF9130681092A
:106940009306090093050C0013050600EFF00FEE07
:10695000930A41126F0000039307C1079306E108F1
:1069600003D7070093872700E31C07EAE39AD7FEC3
:1069700093040000930A4112130901161304010D38
:10698000930B810E9305040013058109EFE0CFE915
:10699000130781099307040083D607009387270014
:1069A00013072700231FD7FEE39877FF9305040002
:1069B0001305C1072318010AEFE00FE79307C1078A
:1069C000035704001304240093872700239FE7FE46
:1069D000E31874FF13058109130609009305C10725
:1069E000231A0108EFF08F810355C11A6314051CA7
:1069F000930C41091304E107130C610B9305CB536E
:106A00001305C107EFE0CFF16306051A1307000075
:106A100093860C006F00C001131717002390F60037
:106A2000131707019386E6FF135707016384860453
:106A300083D7060013960701135606419397170054
:106A400063540600136717009397070193D7070154
:106A50001376270093E51700E30006FC13171700D1
:106A60002390B600131707019386E6FF135707011B
:106A7000E39086FC1307410B9307C10783D60700F9
:106A80009387270013072700231FD7FEE39897FF5C
:106A90002316010C130700009306C10C6F00C00100
:106AA000131717002390F600131707019386E6FFCC
:106AB000135707016384860583D7060013960701E1
:106AC0001356064193971700635406001367170087
:106AD0009397070193D707011376270093E51700D3
:106AE000E30006FC131717002390B60013170701E5
:106AF0009386E6FF13570701E39086FD1307000016
:106B00009306C10C6F00C001131717002390F60005
:106B1000131707019386E6FF135707016384860561
:106B200083D7060013960701135606419397170063
:106B300063540600136717009397070193D7070163
:106B40001376270093E51700E30006FC13171700E0
:106B50002390B600131707019386E6FF135707012A
:106B6000E39086FD1306000093860C001307C10C0A
:106B700083D50600835707009386E6FF1307E7FFD8
:106B8000B387B700B387C70013D607012391F60078
:106B900013761600E31E87FD13058109130609000D
:106BA0009305C107EFE09FE50355C11A9384F4FFF5
:106BB000E30605E483270101832601001307300063
:106BC000B337F000B307F04093F7D700938707027D
:106BD0002302F112832741006394E600B3879700F4
:106BE0001307A002138407006354F7001304A002E4
:106BF0001307A0006302E54E130505031307E00227
:106C0000A302A1122303E112E3C2071E930771122C
:106C10002328F100130C0000232E910093040C0094
:106C2000130C090003290101930C410B930D410939
:106C3000930BE107130D610B1307000013860D0082
:106C40006F00C001131717002310F6001317070178
:106C50001306E6FF13570701630476058357060002
:106C60009395070193D505419397170063D40500C9
:106C7000136717009397070193D7070193752700B0
:106C800013E51700E38005FC131717002310A60077
:106C9000131707011306E6FF13570701E31076FDEC
:106CA00013870C009307C10703D6070093872700BB
:106CB00013072700231FC7FEE398B7FF2316010C15
:106CC000130700001306C10C6F00C0011317170053
:106CD0002310F600131707011306E6FF13570701E9
:106CE0006304A605835706009395070193D50541D4
:106CF0009397170063D40500136717009397070154
:106D000093D707019375270013E51700E38005FC6F
:106D1000131717002310A600131707011306E6FF29
:106D200013570701E310A6FD130700001306C10C5B
:106D30006F00C001131717002310F6001317070187
:106D40001306E6FF135707016304A60583570600E1
:106D50009395070193D505419397170063D40500D8
:106D6000136717009397070193D7070193752700BF
:106D700013E51700E38005FC131717002310A60086
:106D8000131707011306E6FF13570701E310A6FDCB
:106D90009305000013860D001307C10C0355060070
:106DA000835707001306E6FF1307E7FFB387A70023
:106DB000B387B70093D507012311F60093F51500AB
:106DC000E31EA7FD13060C009305C10713058109F7
:106DD000EFE0DFC28357C11A330799009384140090
:106DE000138607032300C700E35894E41345F4FF18
:106DF000032701011355F5413375A4008324C10114
:106E00001309150033092701330CA70013074000AD
:106E1000635EF70413075000E380E7008347E9FF50
:106E20001307E9FF93F7F707634404789306E0023A
:106E30001306800393050003638ED7006352F67830
:106E40008347F7FF2300B7001307F7FF93F7F70710
:106E50006FF09FFE8347F7FF93068003E3F4F6008D
:106E60009307100393841400A30FF7FEB705008166
:106E7000138604009385855313050C00EF20D00A78
:106E800083572107032741012328911693C7F7FF52
:106E90002322E11613971701631E070013850900CB
:106EA000EFE0CFB96310052213850900EFE0CF8C26
:106EB000631A05208326C1000347411293871400FB
:106EC00023A0F60093870A00630A07029306E002F4
:106ED000630CD71C03C7170093871700E31A07FE3C
:106EE0009306500463E6FA006F004001638857017F
:106EF00003C7F7FF9387F7FFE31AD7FE2380070046
:106F000093870A00930600021306D00203C7070006
:106F10006304D7006316C700938717006FF01FFF45
:106F200013840A006F00C00003C707001384060023
:106F30002300E4009306140093871700E31607FE6E
:106F400083260100930720000347F4FF6386F612AF
:106F5000832741009386070063D49700938604003B
:106F6000930700036316F702B307544163D2F60296
:106F7000130600036F00800063DCE6008347E4FF34
:106F8000A30F04FE1304F4FF33075441E386C7FE46
:106F900003270100930730006302F70A832781006B
:106FA00023220A04938697009307700163F2D70C9B
:106FB00013071000930740009397170013864701AB
:106FC0009305070013071700E3F8C6FE2322BA044F
:106FD00013050A00EF1000562320AA0493850A0027
:106FE00093040500EF20902983278101638807001F
:106FF000330454413384840023A087008320C11EBE
:107000000324811E0329011E8329C11D032A811D1A
:10701000832A411D032B011D832BC11C032C811CC2
:10702000832C411C032D011C832DC11B13850400DF
:107030008324411E1301011F678000008327410044
:10704000B384970063C804508327C10003278100DD
:1070500083A70700B307F7002324F10083278100EB
:1070600023220A049386370093077001E3E2D7F4E2
:10707000930500006FF0DFF593070003E310F7F2CC
:10708000B307544193061000E3C4F6EE6FF01FF10E
:1070900083248100232291009307A00263D097EC00
:1070A0002322F1006FF08FEB03C70700E30A07E22A
:1070B00003C7170093871700A38FE7FEE31A07FEA5
:1070C0006FF01FE20327C100B72700009387F77016
:1070D0002320F7006FF0DFE213071003A302E11291
:1070E0001307E0022303E11293841400635CF02A87
:1070F00093070003A303F112930781121304F4FF13
:107100002328F1006FF01FB1930C410B13870C0083
:107110009307C1071306010983D607009387270049
:1071200013072700231FD7FEE398C7FEB7470000C9
:107130009387E7082313F10CB78700009387F7FFC5
:10714000232EF100B7C7FFFF930A41121304010D6C
:10715000130E000113838D0C938727002324410312
:107160002322510393040000938A0C001309011693
:10717000930C0400930BA10A2320F102130A0E00C2
:1071800013040300930609001306810993850A007E
:1071900013050400EFE09FE91307C1049307810979
:1071A00083D607009387270013072700231FD7FEE6
:1071B000E398A7FF8327C1018355E10533F6F50066
:1071C000832701023305F6006350A03A1306000935
:1071D0003306A64013870C009307C10483D607002B
:1071E0009387270013072700231FD7FEE39837FF55
:1071F0006354C0069307F00013870C0063DCC702DA
:10720000130606FF93564600138716001317170040
:107210003387EC0093870C0093872700239F07FE9A
:10722000E39CE7FE130600083306A640939646004B
:107230003306D640131616003386CD008357070059
:1072400083560623B3F7D7002310F7009395050163
:1072500093D5054163C005169307810913870C0078
:1072600003D60700835607009387270013072700DC
:107270006314D602E396FBFE13870A009307810985
:1072800083D607009387270013072700231FD7FE05
:10729000E398A7FFB3844401130444019387CD12FC
:1072A000135A1A00E310F4EE8357610C0357E108F8
:1072B00013840C00032A8102B387E70037C7FFFF5E
:1072C000938C0A00130727F7832A4102B387E7004C
:1072D0002313F10C1307C10793870C001306810CCD
:1072E00083D607009387270013072700231FD7FEA5
:1072F000E398C7FE13070000930781096F00800021
:1073000003570C0093872700239FE7FE130C2C00E4
:10731000E398A7FF138D8D02371C0000938D8D110C
:107320006F000001135C1C006300BD29130D4D01AB
:1073300093850C0013850D00EFD09FDE93070500A9
:1073400093850C0013050D006340F026EFD05FDD40
:10735000E34AA0FC9306090013860C0093850C00F9
:1073600013050D00EFE09FCC130681099306090079
:107370009305060013050D00EFE0DF89B384840157
:107380006FF05FFA930A4112B7050081938545516A
:1073900013850A00B7240000EF2000399384F470AD
:1073A0006FF01FAE130C7112E39207AC232881011A
:1073B0006FF05F869307C10413870C006F00C00055
:1073C0009306E105E38AF6E803D607008356070033
:1073D0009387270013072700E304D6FE8357210E67
:1073E0000327C101B377F700639EE70013850C0004
:1073F000EFD09FB8E31205E613850C00EFD01FE431
:10740000E31C05E49305C10E13050C00EFD0DFC1AA
:107410009305811013850C00EFD01FC10356C10ED8
:107420000355A1108358E10E1346F6FF131606010B
:10743000135606012316C10EB385A8409306050016
:10744000635EB00683264102130781109307011281
:10745000835507001307270093862600239FB6FE57
:10746000E318F7FE231E0112130781109306C10EC5
:107470006F00800003D6060013072700231FC7FEF6
:1074800093862600E318F7FE83274102231001129A
:107490001307C10E1306C11383D607009387270075
:1074A00013072700231FD7FEE398C7FE8356A110BA
:1074B000B305154123120110138506006386052CC0
:1074C0002326D1029307F0F663C8F5061305C10E13
:1074D000EFD09FD88326C1029305050093070112C0
:1074E000130541100356C10E03578110630AE62E9F
:1074F000130700001306070003D707000358050011
:107500009387E7FF3307C740330707411356070147
:107510002391E7001307A110137616001305E5FF6A
:10752000E39CE7FC1306100093070900130700040F
:1075300013058110EFE0CF8B93850C0013058110AC
:10754000EFE04FE26FF05FD1832781009384F7FF74
:107550006FF05FB48327C1002302011213840A0075
:1075600023A007006FF09FAF93870C001307410E15
:1075700093872700239F07FEE39CE7FE6FF01FCD54
:1075800083270101930A4112638A0706B705008128
:107590009385C55113850A00B7240000EF20C01859
:1075A0009384F4706FF0DF8D930B810E6FF08FBDBD
:1075B00093071003230FF9FE938414006FF01F8BC1
:1075C000938717002300F7006FF05F8A930A411238
:1075D000B70500819385455313850A00B724000041
:1075E000EF2080149384F4706FF09F898357C11A41
:1075F000130C6112130971126FF05F81B7050081DE
:107600009385855213850A00B7240000EF20C0112E
:107610009384F4706FF0DF86930581091305C10729
:10762000EFE04FD49305CB5313058109EFD05FAF43
:10763000631605FEE34C04828347E9FF138727FDA9
:10764000133717001347F7FF3307EC000347070012
:1076500013771700E30C07801307E9FF93F7F70789
:107660006FF0CFFC93871700A30FF7FE6FF01F801A
:107670001304010D930504001305C107B74C000066
:10768000EFD09F9A93040000930B810E1309C10C55
:10769000930A210D938CECFF8357810E93F77700AB
:1076A000639A070C1307410B9307040083D6070066
:1076B0009387270013072700231FD7FEE39877FF40
:1076C0001305410B2316010CEFD00FF41305410BEA
:1076D000EFD08FF3130600009306090013870B0009
:1076E00083D50600835707009386E6FF1307E7FF5D
:1076F000B387B700B387C70013D607012391F600FD
:1077000013761600E31E57FD8357610B0357810B59
:1077100093873700231BF10A630007021305410B0F
:10772000EFD08FEE8357610B0357810B93871700C0
:10773000231BF10AE31407FE8357C10C639C070265
:107740008357610B63E8FC02130704009307410BA6
:1077500083D607009387270013072700231FD7FE30
:10776000E39827FF2314010E9384F4FF930750FD41
:10777000E394F4F29305C10713050400EFE08FBE14
:10778000130901166FF04F8F1307C1109307010FF4
:1077900083D80700035607009387270013072700A5
:1077A0006398C80213066110E394C7FE0357C10E25
:1077B000835781106302F70693870C001307410E6D
:1077C00093872700239F07FEE39CE7FE6FF0DFA867
:1077D0006366160D93070112130541106FF09FD0D9
:1077E000130700001303E10E03D80700035605003A
:1077F0009387E7FF1305E5FF330606013307E6002D
:10780000135607012391E70013771600E31E65FC6A
:10781000130600006FF05FD113870600639206061F
:107820008317E11063CE0704930601126F00000274
:107830002390F60013171700131707019386E6FF2E
:107840009307A11013570701E388F6CE83D70600EC
:1078500013960701135606419397170063540600C9
:10786000136717009397070193D707011376270033
:1078700093E51700E30E06FA2390B6006FF09FFB26
:107880001306C11093070112631207086382C70829
:1078900003570600130626006FF01FFF0326410260
:1078A00013078110930701120355070013072700E0
:1078B00013062600231FA6FEE318F7FE231E01125F
:1078C000130681101307C10E13054110035807005A
:1078D0001307270013062600231F06FFE318A7FE41
:1078E00003274102231001129308C10E1306C1138E
:1078F000035807001307270093882800239F08FFD9
:10790000E318C7FE231201106FF0DFBD13851600C8
:107910002315A1106FF05FC2032785008327C500E0
:107920000326050083264500130101FC1305010011
:10793000930541012324E1002326F100232E1102A7
:107940002320C1002322D100EFE05FBF83576102F3
:107950001305000093C7F7FF13971701631A070079
:1079600013054101EFD04FE1133515001305150044
:107970008320C10313010104678000001305050F74
:10798000678000003715008113058572678000004D
:10799000371500811305857267800000130101FF10
:1079A000232611002324810023229100630C060268
:1079B000B705008193854579130506001304060079
:1079C000EF101074B7040081631205021385047967
:1079D0008320C1000324810083244100130101019D
:1079E00067800000B70400816FF05FFE9385047923
:1079F00013050400EF10D070E30A05FCB705008101
:107A00009385853713050400EF10906FE30005FCA4
:107A1000130500006FF0DFFBB717008103C5077681
:107A2000678000003727008193070500032587BB87
:107A300013860500938507006FF05FF6130101F9C7
:107A400023248106138405008395E50023229106F3
:107A5000232021072326110693040600138906001C
:107A600063CA050413068100EF60404E63440504B9
:107A70000327C100B7F700008320C106B3F7E70072
:107A800037E7FFFFB387E7000324810693B71700AA
:107A90002320F9009307004023A0F40037150000CD
:107AA00083244106032901061305058013010107FC
:107AB000678000008357C4002320090093F707085C
:107AC000638407028320C106032481069307000410
:107AD00023A0F400032901068324410613050000B6
:107AE00013010107678000008320C106032481067B
:107AF0009307004023A0F4000329010683244106D4
:107B000013050000130101076780000083D7C5003B
:107B1000130101FE232C8100232E1100232A910042
:107B20002328210193F727001384050063880702A7
:107B30009387350423A0F50023A8F50093071000D0
:107B400023AAF5008320C10103248101832441017C
:107B50000329010113010102678000009306C1009F
:107B60001306810093040500EFF05FED832581008B
:107B70001309050013850400EF00400B8317C400B0
:107B800063080504374700801307874F23AEE402DC
:107B9000032781008326C10093E707082316F4001A
:107BA0002320A4002328A400232AE40063980604C9
:107BB000B3E727018320C1012316F40003248101C8
:107BC00083244101032901011301010267800000A0
:107BD00013F70720E31807F693F7C7FF93E727008B
:107BE000130734042316F400930710002320E40045
:107BF0002328E400232AF4006FF0DFF48315E40067
:107C000013850400EF609005631605008317C40018
:107C10006FF01FFA0357C4001377C7FF13671700ED
:107C20009317070193D707416FF09FF8130101FDE8
:107C3000232E3101232611022324810223229102C3
:107C400023202103232C4101232A510123286101F0
:107C50002326710123248101232291019387B500FA
:107C600013076001930905006366F7069307000197
:107C700063E6B71EEF00900B93040001130620008B
:107C800093078001371900811309497AB307F90076
:107C900003A44700138787FF630AE4208327440077
:107CA0008326C4000326840093F7C7FFB307F400BC
:107CB00003A747002326D60023A4C6001367170096
:107CC0001385090023A2E700EF0090061305840046
:107CD0006F00801993F487FF63C2071863E0B4183C
:107CE000EF00D0049307701F63F6974693D7940074
:107CF0006386071A13074000636CF73C93D7640050
:107D0000138697031385870393163600371900816E
:107D10001309497AB306D90003A44600938686FF67
:107D2000638686029305F0006F000001635C0732F2
:107D30000324C400638C86008327440093F7C7FFA5
:107D400033879740E3D4E5FE1306050003240901B9
:107D50009308890063081417032544009306F00074
:107D60001375C5FFB307954063CCF640232A19016C
:107D70002328190163D6073E9307F01F63EAA72E55
:107D8000937785FF9387870083254900B307F90020
:107D900083A6070013555500130710003317A700DB
:107DA0003367B700938587FF2326B4002324D400CC
:107DB0002322E90023A0870023A6860093572640AC
:107DC00093051000B395F5006368B710B3F7E500AD
:107DD00063940702939515001376C6FFB3F7E50089
:107DE00013064600639A070093951500B3F7E50064
:107DF00013064600E38A07FE1308F000131336004B
:107E000033036900130503008327C500130E060022
:107E10006302F52E03A747001384070083A7C7005A
:107E20001377C7FFB30697406342D82EE3C206FE1E
:107E30003307E400832647000326840013850900E6
:107E400093E616002322D7002326F60023A4C700BA
:107E5000EF00006E130584006F0000019307C0005F
:107E600023A0F900130500008320C102032481022E
:107E700083244102032901028329C101032A8101CC
:107E8000832A4101032B0101832BC100032C8100B4
:107E9000832C41001301010367800000930600203A
:107EA000130600041305F0036FF05FE603A4C70098
:107EB00013062600E39487DE032409019308890052
:107EC000E31C14E90327490093572640930510004B
:107ED000B395F500E37CB7EE03248900832A4400C0
:107EE00013FBCAFF63689B00B3079B401307F000B6
:107EF0006346F714B7270081B72C008183AA07C80F
:107F000003A7CCBB9307F0FF330A6401B38A540183
:107F1000630AF734B71700009387F700B38AFA00B3
:107F2000B7F7FFFFB3FAFA0093850A00138509003B
:107F3000EF1000689307F0FF930B0500630CF52822
:107F400063684529372C0081130C8CC483250C00F1
:107F5000B385BA002320BC00938705006304AA3AC6
:107F600083A6CCBB1307F0FF638CE63A338A4B4100
:107F7000B307FA002320FC0093FC7B0063860C30DF
:107F8000B7170000B38B9B4193858700938B8B00C1
:107F9000B3859541B38A5B019387F7FFB38555415C
:107FA00033FAF50093050A0013850900EF104060CD
:107FB0009307F0FF6300F53C33057541B30A4501B3
:107FC00083250C002324790193EA1A00B305BA0033
:107FD0002320BC0023A25B01630824359306F00034
:107FE00063F866350327440093074BFF93F787FF39
:107FF000137717003367F7002322E40013065000BD
:108000003307F4002322C7002324C70063EEF636AB
:1080100083AA4B0013840B00B727008103A7C7C7AF
:108020006374B70023AEB7C6B727008103A787C71D
:108030006376B71A23ACB7C66F00401A13E7140073
:108040002322E400B30494002324990093E717004B
:108050001385090023A2F400EF00804D130584006E
:108060006FF09FE08326C400032684006FF01FC4D6
:1080700093579500130740006372F71413074001EC
:10808000636AF7229386C7059385B70593963600F2
:10809000B306D90083A70600938686FF6388F61C83
:1080A00003A747001377C7FF6376E50083A7870020
:1080B000E398F6FE83A6C700032749002326D400D1
:1080C0002324F40023A4860023A687006FF01FCF8B
:1080D000130740016376F71213074005636AF71E22
:1080E00093D7C4001386F7061385E7069316360068
:1080F0006FF0DFC1130E1E0093773E00130585005D
:10810000638E07108327C5006FF09FD0032684007D
:1081100093E514002322B4002326F60023A4C7000D
:10812000B3049400232A99002328990093E71600AA
:1081300023A6140123A4140123A2F4003307E400AE
:10814000138509002320D700EF00803E130584002B
:108150006FF09FD113D63400938784006FF09FB2E5
:108160003307A400832747001385090093E717000E
:108170002322F700EF00C03B130584006FF0DFCE31
:1081800013E714002322E400B3049400232A990087
:108190002328990013E7170023A6140123A4140130
:1081A00023A2E4003305A4002320F5001385090071
:1081B000EF000038130584006FF01FCB9357650064
:1081C0009386970393858703939636006FF05FEC51
:1081D000630E241103248900832A440093FACAFF02
:1081E000B3879A4063E69A001307F000E348F7E488
:1081F00013850900EF00C033130500006FF0DFC6E0
:108200001386C7051385B705931636006FF01FB0A8
:10821000832783001306F6FF6392671C937736006B
:10822000130383FFE39607FE0327490093C7F5FF77
:10823000B3F7E7002322F90093951500E3EEB7C8E2
:10824000E38C05C833F7F500631A07009395150012
:1082500033F7F500130E4E00E30A07FE13060E0077
:108260006FF0DFB9938A0A016FF01FCC0325490034
:1082700093D52540130710003317B7003367A700C5
:108280002322E9006FF09FE3B3855B01B305B040A3
:108290009395450113DA450193050A0013850900FA
:1082A000EF1000319307F0FFE318F5D0130A000038
:1082B0006FF01FD1130740056362F7089357C5009D
:1082C0009386F7069385E706939636006FF05FDC9A
:1082D000130740156362F70893D7F40013868707E6
:1082E00013857707931636006FF05FA2372C008155
:1082F000130C8CC483270C00B387FA002320FC00E6
:108300006FF01FC613174A01E31C07C4032489003A
:10831000B30A5B0193EA1A00232254016FF0DFCF06
:1083200023AE7CBB6FF05FC513840B006FF0DFCE14
:108330009307100023A2FB006FF09FEB130740157B
:108340006362F7069357F50093868707938577074F
:10835000939636006FF0DFD3130740556362F7063C
:1083600093D724011386D7071385C70793163600C2
:108370006FF0DF99938C8CFFB38A9A01B38A7A41AC
:10838000130A00006FF0DFC3930584001385090012
:10839000EFC0CFE00324890083250C00832A44002A
:1083A0006FF09FC7130740556364F7029357250189
:1083B0009386D7079385C707939636006FF05FCDF6
:1083C0009306803F1306F0071305E0076FF01F9434
:1083D0009306803F9305E0076FF09FCB832749000A
:1083E0006FF09FE5B717008103A3C7716700030013
:1083F000638005026302060463880604834706005F
:1084000023A0F500034506003335A0006780000077
:10841000130101FF9305C10063040602638A06028B
:108420008347060023A0F500034506003335A0006E
:108430001301010167800000130500006780000040
:10844000130500006FF0DFFE1305E0FF67800000FA
:108450001305E0FF6FF0DFFD9377350093F6F50F1E
:10846000638A07029307F6FF630E06021306F0FF06
:108470006F0080011305150013773500630E0700A8
:108480009387F7FF6380C70203470500E314D7FE15
:108490006780000093070600130730006366F70249
:1084A000639607001305000067800000B307F5001E
:1084B0006F00C00013051500E386A7FE0347050003
:1084C000E31AD7FE67800000370701009398850004
:1084D0001307F7FFB3F8E80093F5F50FB3E5B8001D
:1084E00093980501B3E8B8003708FFFEB785808090
:1084F0001308F8EF938505081303300003270500E0
:1085000033C7E800330607011347F7FF3377E60068
:108510003377B700E31C07F89387C7FF13054500BF
:10852000E36EF3FCE39407F86FF0DFF76780000079
:10853000678000008327C504130101FF2324810005
:10854000232291002326110023202101130405007A
:1085500093840500638E070213952400B387A70058
:1085600003A50700630605040327050023A0E70011
:1085700023280500232605008320C1000324810051
:1085800083244100032901001301010167800000D9
:108590001306100293054000EF50C05A2326A4048E
:1085A00093070500E31A05FA130500006FF0DFFCDE
:1085B00013091000331999001306590013162600E9
:1085C0009305100013050400EF50C057E30E05FC9F
:1085D00023229500232425016FF09FF96380050273
:1085E00003A745008327C50413172700B387E700B7
:1085F00003A7070023A0E50023A0B70067800000C1
:10860000130101FE232A910083A405013703010011
:10861000232C81002328210123263101232E110040
:1086200023244101138905009309050013840600E2
:1086300013884501930800001303F3FF8327080004
:108640001308480093881800B3F66700B386C60283
:1086500093D70701B387C702B386860013DE0601EE
:1086600033F76600B386C701939706013387E700A7
:10867000232EE8FE13D40601E3C298FC6302040231
:108680008327890063D0F4049387440093972700DD
:10869000B307F90023A287009384140023289900CC
:1086A0008320C10103248101832441018329C10066
:1086B000032A8100130509000329010113010102A6
:1086C0006780000083254900138509009385150004
:1086D000EFF05FE603260901130A05009305C900C0
:1086E00013062600131626001305C500EF50D063AD
:1086F0000327490083A7C90413172700B387E7009E
:1087000003A707002320E90023A0270113090A007B
:108710006FF09FF7130101FE232C8100232A9100A3
:1087200023282101232631012324410113888600B7
:1087300093079000232E1100232251013348F802A1
:10874000938906001309050013840500130A060027
:108750009304070063D6D70C93071000930500001D
:108760009397170093851500E3CC07FF13050900C5
:10877000EFF05FDC930710002328F500232A950013
:10878000930790009305050063D64709930A940068
:1087900093840A003304440183C604001306A00036
:1087A00013050900938606FDEFF09FE593841400FE
:1087B00093050500E39284FE13048AFF33848A0044
:1087C00063563A03B3894941B3093401834604002F
:1087D0001306A00013050900938606FDEFF05FE283
:1087E0001304140093050500E39289FE8320C10160
:1087F0000324810183244101032901018329C1004C
:10880000032A8100832A4100138505001301010218
:10881000678000001304A400130A90006FF05FFA51
:10882000930500006FF09FF43707FFFF3377E500F3
:1088300093070500130500006316070093970701CF
:1088400013050001370700FF33F7E7006316070041
:108850001305850093978700370700F033F7E7008B
:10886000631607001305450093974700370700C0BC
:1088700033F7E700631607001305250093972700D9
:1088800063C807001397170013051500635407000A
:108890006780000013050002678000008327050041
:1088A0001307050093F677006384060293F617001A
:1088B00013050000639E060693F6270063800608F2
:1088C00093D717002320F7001305100067800000DE
:1088D0009396070193D606011305000063960600E0
:1088E00093D707011305000193F6F70F639606006F
:1088F0001305850093D7870093F6F700639606006B
:108900001305450093D7470093F63700639606009A
:108910001305250093D7270093F61700639C0600E4
:1089200093D717001305150063960700130500027F
:10893000678000002320F7006780000093D727009E
:108940002320F7001305200067800000130101FFBA
:1089500023248100138405009305100023261100B1
:10896000EFF05FBD8320C100232A8500032481002E
:10897000130710002328E5001301010167800000A0
:10898000130101FE232821012326310103A905013A
:1089900083290601232A910023244101232E11005B
:1089A000232C8100138A050093040600634C3901CF
:1089B000138709009384050093090900130A060030
:1089C0001309070083A7840083A544003384290189
:1089D000B3A78700B385F500EFF0DFB513034501BA
:1089E00093182400B308130193070300637813015D
:1089F00023A0070093874700E3EC17FF13084A0101
:108A0000131E2900938E440193952900330EC8014B
:108A1000B385BE006376C81393875401130F4000DB
:108A200063F0F516370601001306F6FF6F008001AC
:108A300093DF0F0163980F081308480013034300E6
:108A40006370C811832F0800B3F4CF00E38204FEE3
:108A50009303030093820E001309000003A7020092
:108A600083AF030093834300B376C700B3869602B7
:108A70009357070133F7CF0093DF0F019382420032
:108A8000B3879702B386E600B386260113D70601A3
:108A9000B3F6C600B387F701B387E7001397070162
:108AA000B366D70023AED3FE13D90701E3E8B2FAC9
:108AB000B307E30123A02701832F080093DF0F01F1
:108AC000E38C0FF6032703009302030093860E0046
:108AD000930407009303000083A7060093D90401C1
:108AE0003377C700B3F7C700B387F70383A4420007
:108AF000938242009386460033F9C400B38737015E
:108B0000B38777009393070133E7E30023AEE2FED8
:108B100003D7E6FF93D707013307F703330727018E
:108B20003307F70093530701E3E8B6FAB307E3010D
:108B300023A0E7001308480013034300E364C8F1CF
:108B4000634880006F0080011304F4FF6308040091
:108B500083A7C8FF9388C8FFE38807FE8320C1016D
:108B60002328850003248101832441010329010175
:108B70008329C100032A81001301010267800000DC
:108B8000338F9540130FBFFE137FCFFF130F4F009E
:108B90006FF05FE9130101FE232C810023263101D0
:108BA00023244101232E1100232A9100232821018F
:108BB000937736001304060093090500138A050015
:108BC0006394070C1354244013090A006308040635
:108BD00083A48904638E040C9377140013090A009C
:108BE0006390070213541440630A040403A50400AD
:108BF000630805069304050093771400E38407FED9
:108C0000138604009305090013850900EFF05FD770
:108C1000630809060327490083A7C90413541440B5
:108C200013172700B387E70003A707002320E900F5
:108C300023A0270113090500E31A04FA8320C101C8
:108C400003248101832441018329C100032A810077
:108C500013050900032901011301010267800000C7
:108C6000138604009385040013850900EFF05FD19B
:108C700023A0A40023200500930405006FF0DFF774
:108C8000130905006FF01FF69387F7FF3707008180
:108C90001307077A93972700B307F70003A6070087
:108CA00093060000EFF0DF95130A05006FF09FF1C7
:108CB0009305100013850900EFF0DF879307102755
:108CC000232AF500930710002328F50023A4A90404
:108CD00093040500232005006FF01FF0130101FE2F
:108CE0002324410103AA050183A78500232631011E
:108CF00093595640338A4901232C8100232A91003D
:108D00002328210123225101232E110013091A00C7
:108D1000938405001304060083A54500930A05000B
:108D200063D827019397170093851500E3CC27FF9D
:108D300013850A00EFF01F801308450163543003C8
:108D40009389590093992900330735019307080047
:108D50009387470023AE07FEE39CE7FE9389C9FE95
:108D60003308380103A70401938744011373F40106
:108D7000131627003386C700630C0308930500020F
:108D8000B3856540930808009306000003A7070019
:108D90009388480093874700331767003367D700ED
:108DA00023AEE8FE03A7C7FFB356B700E3E0C7FE54
:108DB00013875401930740006372E6083308F800F4
:108DC0002320D80063840600130A090003A7440087
:108DD00083A7CA048320C10113172700B387E700C4
:108DE00003A70700232845010324810123A0E400F1
:108DF00023A0970003290101832441018329C10095
:108E0000032A8100832A41001301010267800000C8
:108E100003A707009387470013084800232EE8FEA6
:108E2000E3F6C7FA03A70700938747001308480033
:108E3000232EE8FEE3EEC7FC6FF05FF9B307964020
:108E40009387B7FE93F7C7FF938747003308F8006F
:108E50002320D800E38C06F66FF01FF703270501E7
:108E600083A70501130805003305F7406314F704D1
:108E70009397270013084801938545013307F800AD
:108E8000B387F5006F0080006376E8028326C7FF92
:108E900003A6C7FF1307C7FF9387C7FFE386C6FE76
:108EA000B3B6C6003305D0401375E5FF13051500B2
:108EB000678000006780000083A705010327060183
:108EC000130101FE232C8100232A91002328210174
:108ED0002326310123244101232E1100138905008B
:108EE00093090600338AE740138445019304460141
:108EF0006398E70413172700B307E4003387E400FF
:108F00006F0080006370F41A03A8C7FF8326C7FFB1
:108F10009387C7FF1307C7FFE306D8FE6376D8021F
:108F20001307040093070900138404001389090040
:108F30009304070093890700130A10006F00C00014
:108F4000E3400AFE130A000083254900EFF08FDE9C
:108F5000032E090183AF090193024501931E2E00E0
:108F6000939F2F00B708010023264501B30ED401BB
:108F7000B38FF401138F020013880400130304005D
:108F8000930700009388F8FF032703008325080058
:108F9000130F4F00B3761701B386F600B3F7150130
:108FA000B386F64093D5050193570701B387B740C1
:108FB00013D70641B387E70013970701B3F61601ED
:108FC000B366D70013084800232EDFFE13034300C7
:108FD00093D70741E36AF8FB13C6F4FF3386CF004B
:108FE00093841400135626001307000063E49F00C7
:108FF000131726003387E2009305400063E69F00C5
:1090000013061600931526003304B400B382B20091
:10901000637ED405B708010013880200930504009D
:109020009388F8FF03A705001308480093854500BF
:10903000337617013306F60093560641935707011E
:10904000B387D7009396070133761601B3E6C600BF
:10905000232ED8FE93D70741E3E6D5FD1387FEFF05
:10906000330787401377C7FF3387E200639A060010
:109070008327C7FF130EFEFF1307C7FFE38A07FE10
:109080008320C101032481012328C50183244101D8
:10909000032901018329C100032A81001301010270
:1090A0006780000093050000EFF0CFC88320C10166
:1090B00003248101930710002328F500232A0500CB
:1090C00083244101032901018329C100032A81006E
:1090D0001301010267800000B707F07FB3F5B70006
:1090E000B707C0FCB385F5006358B00093070000D4
:1090F0001385070067800000B305B04093D5454154
:109100009307300163C8B700B7070800B3D5B7406D
:109110006FF0DFFD1387C5FE9306E00193050000A5
:1091200093071000E3C6E6FCB7070080B3D7E7005B
:109130001385070067800000130101FE232A9100B8
:1091400083240501232C81001304450193942400FA
:10915000B30494002328210103A9C4FF232631016D
:10916000232441011305090093890500232E1100D2
:10917000EFF08FEB13070002B307A74023A0F9001D
:109180009307A000138AC4FF63D0A708130555FFF7
:109190006370440583A784FF63000504B306A740FA
:1091A00033D7D7003319A9003369E900138684FF48
:1091B0003707F03F3367E900B397A7006372C40233
:1091C00003A644FFB356D600B3E7D7006F004001B3
:1091D00093070000631405063707F03F3367E90083
:1091E0008320C1010324810183244101032901015A
:1091F0008329C100032A8100138507009305070016
:1092000013010102678000009306B000B386A640F8
:10921000B707F03F3357D9003367F70093070000D3
:109220006376440183A784FFB3D7D70013055501A4
:109230003315A900B367F5006FF09FFA3315A90045
:109240003707F03F3367E500930700006FF05FF9E1
:10925000130101FD232A5101938A05009305100093
:109260002324810223229102232021039304060058
:10927000232E3101232C4101938906001309070095
:1092800023261102EFF00FAB13D74401370610006D
:109290009307F6FF9316570113040500B3F79700E1
:1092A000137AF77F63840600B3E7C7002326F10033
:1092B000638C0A061305810023245101EFF00FDEB1
:1092C0000327C100930705006316050A8326810062
:1092D000232AD400B334E00093841400232CE40048
:1092E0002328940063040A06130ADABC330AFA003E
:1092F0001305500323A04901B307F5402320F900CB
:109300008320C10213050400032481028324410247
:10931000032901028329C101032A8101832A410112
:1093200013010103678000001305C100EFF00FD7A0
:10933000930710002328F4008327C1009304100032
:10934000232AF40093070502E3100AFA1397240076
:109350003307E400032507019387E7BC23A0F90046
:10936000EFF08FCC93945400B384A4402320990051
:109370006FF01FF90326810093060002B386A64012
:10938000B316D700B3E6C6003357A700232AD4008C
:109390002326E1006FF01FF4130101FD23202103B8
:1093A00013890500930581002326110223248102DD
:1093B00023229102232E310193090500EFF0DFD71C
:1093C0009304050013840500130509009305C100EB
:1093D000EFF09FD68327090103A709018326C10067
:1093E0003307F7408327810013175700B387D7400F
:1093F000B307F70093060500635EF00293974701F9
:1094000033848700138606001385040093860500C5
:1094100093050400EF70407E8320C1020324810283
:1094200083244102032901028329C101130101039D
:109430006780000013974701B385E5406FF09FFCFC
:10944000130101FF23202101232611002324810081
:1094500023229100930770011309050063DAA70422
:1094600037170081832787028325C70237170081BA
:10947000032407038324470313850700130604000E
:1094800093860400EF7050651309F9FF93070500F8
:10949000E31409FE8320C1000324810083244100DA
:1094A00003290100138507001301010167800000F3
:1094B000B7070081131935009387077A338927018D
:1094C000832709018320C1000324810083254901EA
:1094D00083244100032901001385070013010101C2
:1094E00067800000832606019385F5FF93D55540DC
:1094F00093851500930746019396260093952500C2
:10950000B386D700B305B50063F8D702130705008B
:1095100003A807009387470013074700232E07FF80
:10952000E3E8D7FEB387C6409387B7FE93F7C7FF3C
:10953000938747003305F5006378B50013054500B0
:10954000232E05FEE36CB5FE6780000003270501AE
:1095500013D65540930645016352C702931727005F
:10956000B387F60063F2F60403A7C7FF9387C7FF2C
:10957000E30A07FE1305100067800000931726001A
:10958000B387F600E350E6FE93F5F501E38C05FCA6
:1095900003A60700130510003357B600B315B70034
:1095A000E302B6FC6780000013050000678000003E
:1095B000130101FF232481002322910013040500DD
:1095C000B7240081138505002326110023A804C6B3
:1095D000EF605FE39307F0FF630CF5008320C100A9
:1095E00003248100832441001301010167800000EE
:1095F00083A704C7E38407FE8320C1002320F4006F
:1096000003248100832441001301010167800000CD
:10961000130101FF23229100B7040080232481005D
:109620002326110093C4F4FF130406002320060030
:10963000B3F6B4003706F07F9387050013070500E3
:1096400063D0C606B3E8A600638C080433F6C500F1
:10965000138805009308000063120602B717008103
:1096600083A6C70303A68703EF70104713070500FF
:1096700013880500B3F6B4009308A0FC93D64641C6
:10968000B70710809387F7FF938626C03378F800DA
:10969000B3861601B707E03FB367F8002320D40074
:1096A0008320C100032481008324410013050700A7
:1096B000938507001301010167800000130101F683
:1096C000930EC108232AF10837030080B707FFFF74
:1096D000138E05001343F3FF2326D10893878720B9
:1096E0009305810093860E00232E1106232AF10094
:1096F0002328E108232C0109232E11092324C10169
:10970000232CC101232E6100232861002322D101D3
:10971000EF00005583278100238007008320C107C5
:109720001301010A67800000130E05003725008130
:10973000130101F6032585BB930E8108232AF10846
:1097400037030080B707FFFF1343F3FF2324C1084B
:109750002326D108938787201386050093860E0061
:1097600093058100232E1106232AF1002328E10806
:10977000232C0109232E11092324C101232CC1010B
:10978000232E6100232861002322D101EF00404DE8
:1097900083278100238007008320C1071301010A6A
:1097A00067800000130101FF23248100138405005A
:1097B0008395E50023261100EF40D07A634005022F
:1097C000832704058320C100B387A7002328F4045E
:1097D0000324810013010101678000008357C40046
:1097E00037F7FFFF1307F7FFB3F7E7008320C10048
:1097F0002316F40003248100130101016780000097
:1098000013050000678000008397C500130101FE67
:10981000232C8100232A91002328210123263101B2
:10982000232E110013F7071013840500930405007D
:109830008395E5001309060093890600631E07025D
:1098400037F7FFFF1307F7FFB3F7E7002316F4001E
:10985000032481018320C1019386090013060900B6
:109860008329C100032901011385040083244101D8
:10987000130101026F4040269306200013060000EA
:10988000EF40D0438317C4008315E4006FF05FFB03
:10989000130101FF23248100138405008395E50053
:1098A00023261100EF4090419307F0FF6304F50277
:1098B0008357C400371700008320C100B3E7E700D7
:1098C0002328A4042316F4000324810013010101BA
:1098D000678000008357C40037F7FFFF1307F7FFC7
:1098E000B3F7E7008320C1002316F40003248100AE
:1098F00013010101678000008395E5006F40802F10
:109900003367B5009303F0FF137737006310071038
:10991000B7877F7F9387F7F70326050083A60500A7
:10992000B372F6003363F600B382F200B3E2620072
:10993000639272106316D6080326450083A645007D
:10994000B372F6003363F600B382F200B3E2620052
:10995000639E720C6316D6060326850083A68500D7
:10996000B372F6003363F600B382F200B3E2620032
:109970006398720C6316D6040326C50083A6C5003F
:10998000B372F6003363F600B382F200B3E2620012
:109990006392720C6316D6020326050183A60501A5
:1099A000B372F6003363F600B382F200B3E26200F2
:1099B000639C720A1305450193854501E30ED6F4B5
:1099C0001317060193970601631EF700135706014C
:1099D00093D706013305F7409375F50F63900502A1
:1099E000678000001357070193D707013305F7403D
:1099F0009375F50F63940500678000001377F70FE8
:109A000093F7F70F3305F740678000000346050022
:109A100083C6050013051500938515006314D60051
:109A2000E31606FE3305D6406780000013054500A7
:109A300093854500E31CD6FC1305000067800000F9
:109A40001305850093858500E312D6FC13050000FD
:109A5000678000001305C5009385C500E318D6FA9A
:109A600013050000678000001305050193850501BB
:109A7000E31ED6F81305000067800000B367B50049
:109A800093F737006392070803A70500B7867F7F27
:109A90009386F6F7B377D700B387D700B3E7E7002D
:109AA000B3E7D7001306F0FF639EC7061306050051
:109AB0001308F0FF2320E60003A745009385450027
:109AC00013064600B377D700B387D700B3E7E700A4
:109AD000B3E7D700E38007FF83C7050003C715007E
:109AE00083C625002300F600638A0700A300E60072
:109AF000630607002301D600639406006780000018
:109B0000A3010600678000009307050003C7050056
:109B10009387170093851500A38FE7FEE31807FED0
:109B200067800000130605006FF01FFB9377350078
:109B300013070500639C0704B7867F7F9386F6F7BB
:109B40009305F0FF0326070013074700B377D600FD
:109B5000B387D700B3E7C700B3E7D700E384B7FE06
:109B60008346C7FF0346D7FF8347E7FF3307A74076
:109B700063800604630A06023335F0003305E5000E
:109B80001305E5FF67800000E38806FA83470700B6
:109B90001307170093763700E39807FE3307A740B3
:109BA0001305F7FF678000001305D7FF67800000EB
:109BB0001305C7FF67800000B3E7A50093F73700E0
:109BC00013070500639807069307300063F4C70680
:109BD0003703FFFEB78880801303F3EF93880808EC
:109BE000130E300083A60500B387660013C8F6FF86
:109BF000B3F70701B3F71701639E07022320D700CD
:109C00001306C6FF1307470093854500E36CCEFC9F
:109C100093851500930717006304060283C6F5FFBA
:109C20001308F6FFA38FD7FE638E06001387070085
:109C3000130608009385150093071700E31006FE2E
:109C4000678000003306C700630A08009387170087
:109C5000A38F07FEE39CC7FE6780000067800000BB
:109C6000130101E12326111E2320211F2324811D1E
:109C70002320A11D138C050013090600232AD100FF
:109C80002324811E2322911E232E311D232C411DAE
:109C9000232A511D2328611D2326711D2322911D76
:109CA000232EB11B130D0500EFD0DFCD8327050058
:109CB000138507002328F102EFF05FE70357CC007C
:109CC0002328010E232A010E232C010E232E010E20
:109CD000137707082326A1026308070003270C0156
:109CE000631407006F10C0569307C1103717008127
:109CF0002322F10E938807009307878C3717008182
:109D0000232CF100130B0900930747A42324F1002F
:109D100083470B002326010E2324010E232001027A
:109D2000232A0102232C0102232E010223240104F1
:109D300023260104232601006384072213040B0059
:109D4000930650026384D72C834714001304140035
:109D5000E39A07FEB3046441630464218326C10EC1
:109D60008327810E23A06801B3869600938717008E
:109D700023A298002326D10E2324F10E930670000F
:109D80009388880063CCF6280327C100834704002A
:109D9000330797002326E1006384071C83441400E3
:109DA000A303010C13041400930DF0FF93090000AA
:109DB000130A00001309A005930A9000930BA00258
:109DC000938C080013041400938704FE6364F90461
:109DD0000327810193972700B387E70083A7070034
:109DE0006780070093090000938604FD8344040004
:109DF00093972900B387370193971700B389F6002B
:109E0000938604FD13041400E3F2DAFE938704FE44
:109E1000E370F9FC93880C00638404142306911406
:109E2000A303010C930A1000930C1000130BC11430
:109E300023280100930D00002324010223220102A4
:109E4000232E0100937B2A0063840B00938A2A004F
:109E500013794A088327C10E6316090033885941D4
:109E6000E34C00638346710C638A06028326810EED
:109E70001306710C23A0C800938717001306100067
:109E80009386160023A2C8002326F10E2324D10EA8
:109E90001306700093888800634CD64C638A0B02CB
:109EA0008326810E1306810C23A0C8009387270008
:109EB000130620009386160023A2C8002326F10E65
:109EC0002324D10E1306700093888800E34CD66AD1
:109ED00093060008E300D942B38D9D41E34EB04D97
:109EE00093760A10E39A062C0327810EB387970115
:109EF00023A068011307170023A298012326F10E5F
:109F00002324E10E9306700063C0E65A938888000C
:109F1000137A4A0063060A00B38459416346905A93
:109F200063D4590193890A000327C100330737011D
:109F30002326E100E39C0752832701012324010E1D
:109F4000638807008325010113050D00EFA01FA5FD
:109F50009308C110130B040083470B00E39007DE46
:109F60008327C10E638407006F1050340357CC0061
:109F700013770704630407006F20803F8320C11E0E
:109F80000324811E0325C1008324411E0329011ED1
:109F90008329C11D032A811D832A411D032B011D15
:109FA000832BC11C032C811C832C411C032D011C01
:109FB000832DC11B1301011F6780000013050D00D5
:109FC000EFD05F9C83274500138507002326F1040B
:109FD000EFF0DFB59307050013050D00938407002C
:109FE0002324F104EFD01F9A83278500232EF1024A
:109FF000638404006F104016834404006FF09FDCFC
:10A0000083440400136A0A026FF0DFDBB304644187
:10A01000E31664D5834704006FF01FD81306410E82
:10A0200093050C0013050D00EF40D066E31005F416
:10A030009308C1106FF05FD593778A0093880C0066
:10A04000638407006F10800A832741011305010B09
:10A05000232891019387770093F787FF83A5070053
:10A0600003A6470093878700232AF100EFA0C030A2
:10A070008327010B832801012328F10E8327410B3D
:10A08000232AF10E8327810B232CF10E8327C10B8A
:10A09000232EF10E1305010F23281101EFD0DF87C6
:10A0A0002326A10C93072000832801016314F500E7
:10A0B0006F108065930710006314F5006F10500750
:10A0C000930710066394F4006F20C01993071004DF
:10A0D0006394F4006F10D05293FBF4FD9307F0FFEC
:10A0E000232A71056394FD006F10502193077004BB
:10A0F0006394FB006F20801E0323C10F23244103C0
:10A10000032E010F832E410F032F810F93670A1037
:10A11000635403006F20C039232C0104138A070005
:10A1200023280100930760046394FB006F10902BB9
:10A1300093075004232211056384FB006F10D03372
:10A1400013891D00930A010B930609001308C10D22
:10A150009307010D1307C10C1306200093850A0015
:10A1600013050D002328C10B2320C105232AD10B81
:10A170002322D103232CE10B2320E103232E610AA8
:10A18000232E6100EFC0CFCF0323C101032F0102B3
:10A19000832E4102032E010483284104130B050082
:10A1A00033092501930C010A93850C0013850A00DD
:10A1B000232E11012328C10B232AD10B232CE10BC1
:10A1C000232E610A2320010A2322010A2324010AE3
:10A1D0002326010AEF70806C8328C1011307090050
:10A1E000630205020327C10D637E27019306000366
:10A1F00093071700232EF10C2300D7000327C10D6E
:10A20000E36827FFB30767412320F1020327C10C4E
:10A2100093077004232EE100032741056314F70020
:10A220006F10501103274105930760046314F70072
:10A230006F10D0348327C101032741059305100413
:10A240009387F7FF2326F10C93F6F40F1306000013
:10A250006318B7009386F60093F6F60F1306100006
:10A26000230AD10C9306B00263DA07000327C10169
:10A27000930710009306D002B387E740A30AD10CDE
:10A280009306900063C4F6006F20400F1308310E50
:10A29000130508001306A000130E300633E7C702AB
:10A2A00093050500938607001305F5FF13070703C1
:10A2B000A38FE5FEB3C7C702E342DEFE9387070321
:10A2C00013F6F70FA30FC5FE9387E5FF63E40701BD
:10A2D0006F2080399306610D6F00800003C6070070
:10A2E0002380C6009387170093861600E39807FF24
:10A2F0009307510EB387B7401307610DB307F700FB
:10A300009306410DB387D740232CF10203270102A6
:10A310008326810393071000B30CD70063C4E700C2
:10A320006F2000238327C102B38CFC0083278102A6
:10A3300093CAFCFF93DAFA4113FAF7BF136A0A10C3
:10A34000B3FA5C012324010223220102232E01001F
:10A3500083278105639407006F1010059307D002CF
:10A36000A303F10C930D0000938A1A006FF09FADC8
:10A370001306410E93050C0013050D00EF409031BC
:10A38000E31005108327C10E9308C1106FF01FB1B1
:10A390008326810E938C1700832701021306100079
:10A3A00023A068019384160013898800E358F636C9
:10A3B0009307100023A2F8002326910F2324910E67
:10A3C00093077000E3C0974A8327C1020327010364
:10A3D00093841400B38CFC002322F9002320E900AD
:10A3E0002326910F2324910E9307700013098900EF
:10A3F000E3CC97488327010F138614009305010AC5
:10A400002328F10A8327410F1305010B232EC100D6
:10A41000232AF10A8327810F2320010A2322010A1C
:10A42000232CF10A8327C10F2324010A2326010AC2
:10A43000232EF10AEF7080460326C1018327010213
:10A440009308890093060600938DF7FFE30C052E11
:10A4500013071B00B38CBC012320E9002322B901A0
:10A460002326910F2324C10E9307700063D4C700E5
:10A470006F10800193070901938624001389080057
:10A4800093880700032681031307410D2320E90069
:10A49000B30796012322C9002326F10E2324D10EEF
:10A4A00013077000E356D7A61306410E93050C0060
:10A4B00013050D00EF40101E6314057C8327C10EA9
:10A4C0009308C1106FF0DFA4930600010327810EEB
:10A4D00063C496006F101012B7160081938E46A3C6
:10A4E00013090001130A7000138B0E006F00C000E7
:10A4F000938404FF63569904938707011307170099
:10A5000023A0680123A228012326F10E2324E10EB3
:10A5100093888800E35EEAFC1306410E93050C0065
:10A5200013050D00EF401017631C0574938404FF9E
:10A530008327C10E0327810E9308C110E34E99FAB9
:10A54000930E0B00B38797001307170023A0D801C1
:10A5500023A298002326F10E2324E10E9306700017
:10A56000E3D0E69C1306410E93050C0013050D0085
:10A57000EF405012631605708327C10E6FF05F9A8B
:10A5800083274101A303010C93880C0003AB070050
:10A5900013894700E3020B4E9307F0FF6394FD001D
:10A5A0006F10C01F13860D009305000013050B00EC
:10A5B000232A9101EFD05FEA2328A10083284101DB
:10A5C000631405006F10C07583270101232A210140
:10A5D00023280100B38C67418347710C93CAFCFFA9
:10A5E00093DAFA412324010223220102232E0100DF
:10A5F000B3FA5C01930D0000E3860784938A1A0086
:10A600006FF05F840327410193880C00A303010CC2
:10A610008327070013074700232AE1002306F114CC
:10A62000930A1000930C1000130BC1146FF05F809D
:10A6300083440400136A4A006FF0CFF88326410177
:10A6400093770A0293880C0003A7060093864600BE
:10A65000232AD100E390072893770A016384070037
:10A660006F10C01293770A04638407006F10803D57
:10A67000137A0A2063140A006F1040118327C10067
:10A68000130B04002300F7006FF01F8D83440400B8
:10A690009307C006E38EF438136A0A016FF08FF255
:10A6A00003274101B787FFFF93C707832314F10CEA
:10A6B00093074700232AF10003290700B707008109
:10A6C0009387473593880C00232AF102930C0000EE
:10A6D000936B2A009307200093048007A303010CC7
:10A6E0001307F0FF6386ED203367990113FAFBF738
:10A6F000631E071E63940D266390071C93FC1B00CA
:10A70000130B011BE3900C1C938A0C0063D4BC0157
:10A71000938A0D008347710C232801002324010232
:10A7200023220102232E0100E39A07EC6FF08FF140
:10A7300093880C00136A0A0193770A02E38C0706D8
:10A7400083274101138B7700137B8BFF03290B00B9
:10A75000832C4B0093078B00232AF100937BFABFD5
:10A76000930700006FF09FF783440400930780066F
:10A77000E388F42C136A0A046FF0CFE493880C008A
:10A78000936B0A0193F70B02E38C070483274101C3
:10A79000138B7700137B8BFF93078B00232AF10029
:10A7A00003290B00832C4B00930710006FF01FF35D
:10A7B00083440400136A8A006FF0CFE083274101CD
:10A7C0008344040083A9070093874700232AF100EC
:10A7D00063DA09DEB3093041136A4A006FF08FDE95
:10A7E00083440400136A1A006FF0CFDD8347710CB5
:10A7F00083440400639807DC93070002A303F10C71
:10A800006FF04FDC83440400136A0A086FF08FDB9B
:10A810008344040013071400639474016F10505FA5
:10A82000938604FD13040700930D000063EEDAD84D
:10A830008344040093972D00B387B70193971700C3
:10A84000B38DD700938604FD13041400E3F2DAFEFF
:10A850006FF08FD79307B00283440400A303F10C79
:10A860006FF04FD693880C00136A0A0193770A029F
:10A870006380077A83274101138B7700137B8BFF5B
:10A8800083274B0003290B0013078B00232AE100C9
:10A89000938C070063C6077A9307F0FF930B0A00B7
:10A8A0006384FD02B3679901937BFAF7639E070007
:10A8B00063920D02138A0B00930D0000930C0000AD
:10A8C000130B011B6FF05FE4E3960C4093079000BD
:10A8D000E3E2274113090903A307211B138A0B0095
:10A8E000930C1000130BF11A6FF01FE2930B0A0088
:10A8F00013071000E38AE7FC13072000638CE706C8
:10A90000130B011B1397DC0193777900135939005E
:10A91000938707033369270193DC3C00A30FFBFEF9
:10A920003367990113060B00130BFBFFE31C07FCB5
:10A9300093F61B00638A0606930600036386D70618
:10A940001306E6FF9307011BA30FDBFEB38CC74082
:10A95000138A0B00130B06006FF01FDB13071000A8
:10A960006394E7006F10101713072000930B0A0081
:10A97000E398E7F883264103130B011B9377F90053
:10A98000B387F60003C70700135949009397CC011A
:10A9900033E9270193DC4C00A30FEBFEB367990169
:10A9A000130BFBFFE39C07FC9307011BB38C674170
:10A9B000138A0B006FF05FD593065006E3DA969C7E
:10A9C0008326010F9305010A1305010B2328D10AE1
:10A9D0008326410F232211052320F104232AD10AC3
:10A9E0008326810F2320010A2322010A232CD10A66
:10A9F0008326C10F2324010A2326010A232ED10A0C
:10AA0000EF60D0698327010483284104631C053863
:10AA10000327810EB70600819386463823A0D8000D
:10AA200093871700930610001307170023A2D8007E
:10AA30002326F10E2324E10E9306700093888800EC
:10AA4000E3CCE6440327C10C832601026350D7669A
:10AA5000032701038326C1029388880023ACE8FE04
:10AA60000327810EB387D70023AED8FE1307170044
:10AA70002326F10E2324E10E9306700063CCE676C4
:10AA8000032701029304F7FF635490C89306000163
:10AA90000327810EE3D2964213090001930C700044
:10AAA0006F00C000938404FFE3589940832681001F
:10AAB000938707011307170023A0D80023A22801BA
:10AAC0002326F10E2324E10E93888800E3DCECFCBE
:10AAD0001306410E93050C0013050D00EF40803B5B
:10AAE0006310051A8327C10E0327810E9308C11036
:10AAF0006FF05FFB33895941635020BF130600019B
:10AB00008326810E63542607130E0001930B7000F9
:10AB10006F00C000130909FF635A2E050327810047
:10AB2000938707019386160023A0E80023A2C8019B
:10AB30002326F10E2324D10E93888800E3DCDBFC6E
:10AB40001306410E93050C0013050D00EF408034F1
:10AB500063180512130E0001130909FF8327C10EA4
:10AB60008326810E9308C110E34A2EFB0327810040
:10AB7000B38727019386160023A0E80023A22801AB
:10AB80002326F10E2324D10E13067000938888002B
:10AB90006354D6B41306410E93050C0013050D0043
:10ABA000EF40402F631E050CB38D9D418327C10EDE
:10ABB0009308C1106356B0B3130600018326810EBB
:10ABC0006352B607930B0001130970006F00C000B9
:10ABD000938D0DFF63D8BB05032781009387070181
:10ABE0009386160023A0E80023A278012326F10E05
:10ABF0002324D10E93888800E35CD9FC1306410E10
:10AC000093050C0013050D00EF40C028631A0506DC
:10AC1000938D0DFF8327C10E8326810E9308C110EB
:10AC2000E3CCBBFB03278100B387B70193861600F3
:10AC300023A0E80023A2B8012326F10E2324D10E7D
:10AC40001306700093888800635CD6A81306410E33
:10AC500093050C0013050D00EF40C023631205029D
:10AC60008327C10E9308C1106FF08FA71306410E02
:10AC700093050C0013050D00EF40C021630E05AADB
:10AC8000832B010163840BAE93850B0013050D002C
:10AC9000EF90DFD06FF08FAD371700811306000102
:10ACA0008326810E930E47A3635C0609232081044B
:10ACB0002322910413040D0093040C00130E0001D1
:10ACC00093027000130C0800138D0E006F00C0007B
:10ACD000130C0CFF635A8E059387070193861600A9
:10ACE00023A0A80123A2C8012326F10E2324D10EFC
:10ACF00093888800E3DED2FC1306410E938504009E
:10AD000013050400EF400019E3120516130E0001AD
:10AD1000130C0CFF8327C10E8326810E9308C110EC
:10AD200093027000E34A8EFB13080C00930E0D0093
:10AD3000138C0400130D0400832441040324010434
:10AD4000B38707019386160023A0D80123A2080128
:10AD50002326F10E2324D10E130670009388880059
:10AD60006352D6901306410E93050C0013050D0097
:10AD7000EF404012E31605F08327C10E9308C1107F
:10AD80006FF04F8E1306410E93050C0013050D0056
:10AD9000EF404010E31605EE8327C10E9308C11063
:10ADA0006FF00F938325C10C635CB07E0327C10154
:10ADB000832601029304070063C2E63C63569002B7
:10ADC0008326810EB387970023A06801938616001F
:10ADD00023A298002326F10E2324D10E130670001F
:10ADE00093888800E34CD64093C6F4FF0327C10143
:10ADF00093D6F641B3F4D400B3049740634E904821
:10AE00000327C10193760A40B30DEB00639A064E07
:10AE10008324C10C0327010263C6E40093761A0061
:10AE2000E3820640832601030327C1021306700054
:10AE300023A0D8008326810EB387E70023A2E80071
:10AE4000938616002326F10E2324D10E93888800C2
:10AE5000E344D66A832601023307DB00B3849640BD
:10AE60003307B7411389040063549700130907009F
:10AE7000635620030327810EB387270123A0B8015F
:10AE80001307170023A228012326F10E2324E10E25
:10AE90009306700093888800E3CAE66A1347F9FFB7
:10AEA0001357F7413377E900B384E44063449000DB
:10AEB0006FF00F86930600010327810E63DE967EF6
:10AEC00013090001930C70006F00C000938404FF0D
:10AED0006354997E83268100938707011307170027
:10AEE00023A0D80023A228012326F10E2324E10E5B
:10AEF00093888800E3DCECFC1306410E93050C00FC
:10AF000013050D00EF301079E31C05D68327C10E21
:10AF10000327810E9308C1106FF05FFB93771A002F
:10AF2000639807C823A2C8002326910F2324910EFB
:10AF30009307700063CA975493862600938808018C
:10AF40006FF04FD46350B0D5130700016344B701CD
:10AF50006F10806B130B7000930406006F000001EC
:10AF6000938D0DFFE35EB711938414008327810056
:10AF7000938C0C012322E9002320F9002326910F52
:10AF80002324910E13098900E35C9BFC1306410EF8
:10AF900093050C0013050D00EF30D06FE31205CEC2
:10AFA000832CC10E8324810E1309C11013070001E5
:10AFB0006FF01FFB8326410193770A011387460038
:10AFC0006394071893770A04E386071483274101E3
:10AFD000930C0000232AE10003D907006FF00FF85B
:10AFE0008326410193F70B011387460063940714EE
:10AFF00093F70B04E380071083274101930C0000B3
:10B00000232AE10003D90700930710006FF00FED2A
:10B010008326410193770A01138746006392071044
:10B0200093770A04E388070A83274101232AE10072
:10B0300003990700935CF94193870C00E3DE0784D2
:10B04000B3372001B30C9041B38CFC409307D0027E
:10B05000A303F10C33092041930B0A00930710005E
:10B060006FF00FE81306410E93050C0013050D0059
:10B07000EF305062E31605C0832CC10E8324810E8D
:10B080001309C1106FF04FB41306410E93050C0065
:10B0900013050D00EF301060E31405BE832CC10EC4
:10B0A0008324810E1309C1106FF0CFB413771A00F7
:10B0B000631407006FE0DFE56FF09F9993880C0041
:10B0C0006FF0CFFA93070003A307F11A130BF11ADD
:10B0D0006FF08FE38326C100130B040093D7F64172
:10B0E0002320D7002322F7006FE01FE70327410149
:10B0F0008327070013074700232AE10083A50700E1
:10B1000003A6470083A6870083A7C7002328B10EA4
:10B11000232AC10E232CD10E232EF10E6FE09FF7B0
:10B1200003A90600232AE100935CF94193870C00F0
:10B130006FF04FF603A90600930C0000232AE100EC
:10B14000930710006FF08FD903A90600930C00003D
:10B15000232AE1006FF08FE08327C10383440400BA
:10B16000639407006FE01FC683C70700639407005E
:10B170006FE05FC5136A0A406FE0DFC49384060086
:10B18000E34090C46FF05FC693880C00930B0A00F5
:10B190006FF04FDFB70700819387473593880C0026
:10B1A000232AF10293770A026380072C8327410147
:10B1B000138B7700137B8BFF03290B00832C4B0031
:10B1C00093078B00232AF10093771A00638E070000
:10B1D000B3679901638A0700930700032304F10C06
:10B1E000A304910C136A2A00937BFABF93072000F3
:10B1F0006FF0CFCE1306410E93050C0013050D0022
:10B20000EF305049E31E05A68327C10E9308C110F5
:10B210006FF01F87B70700819387873693880C00EC
:10B22000232AF1026FF01FF893880C006FF0CFD043
:10B2300083441400136A0A02130414006FE09FB8D9
:10B2400083441400136A0A20130414006FE09FB7AC
:10B250009305000413050D00EFC05F9D2320AC0093
:10B260002328AC00631405006F10C03C13070004D2
:10B27000232AEC006FE05FA793076000938C0D001A
:10B2800063EEB77937070081938A0C00232A2101E6
:10B29000130BC7376FE0DFB9130600018326810E59
:10B2A0006358966A930C0001930D70006F00C00004
:10B2B000938404FF63DE9C68032781009387070162
:10B2C0009386160023A0E80023A298012326F10EFE
:10B2D0002324D10E93888800E3DCDDFC1306410EA5
:10B2E00093050C0013050D00EF30D03AE31A0598D2
:10B2F0008327C10E8326810E9308C1106FF05FFB78
:10B3000003270102832C4102232E410123208104C3
:10B31000232231052322510383298102232461033F
:10B32000B30BEB000324C103032A8104832AC10465
:10B330009304700013090001130B0C0063880C08C0
:10B34000639809081304F4FF938CFCFF0327810E14
:10B35000B387470123A058011307170023A2480110
:10B360002326F10E2324E10E9388880063C4E4149D
:10B37000834604003386BB41138C06006354D60019
:10B38000130C0600635680038326810EB387870162
:10B3900023A0B8019386160023A288012326F10E6C
:10B3A0002324D10E63C0D4348346040093888800DC
:10B3B0001346FCFF1356F6413377CC00338CE6403E
:10B3C000634C8001B38DDD00E39C0CF6638C097245
:10B3D0009389F9FF6FF09FF78326810E63488901F7
:10B3E0006F008005130C0CFF63588905032781004B
:10B3F000938707019386160023A0E80023A2280163
:10B400002326F10E2324D10E93888800E3DCD4FC9C
:10B410001306410E93050B0013050D00EF30902726
:10B42000631C055A130C0CFF8327C10E8326810E63
:10B430009308C110E34C89FB03278100B387870180
:10B440009386160023A0E80023A288012326F10E8C
:10B450002324D10E63C4D4768346040093888800E5
:10B46000B38DDD006FF05FF68326410193770A010B
:10B47000138746006384072003A90600930C00008D
:10B48000232AE1006FF05FD41306410E93050C00F0
:10B4900013050D00EF301020631405FE8326810E86
:10B4A000832CC10E93084111938616001309C11015
:10B4B0006FE05FFD1306410E93050B0013050D00B1
:10B4C000EF30501D631A05508327C10E9308C11039
:10B4D0006FF01FEA130B011B930700002328810064
:10B4E000232E910013040B0023223103130B0C00B5
:10B4F0009304090093890C0013FA0B40832CC103B9
:10B50000930AF00F138C0800138907006F004002A4
:10B510001306A0009306000013850400938509001C
:10B52000EF4050696380094C93040500938905003E
:10B530001306A000930600001385040093850900FC
:10B54000EF50802A13050503A30FA4FE1309190069
:10B550001304F4FFE30E0AFA83C60C00E31AD9FAC7
:10B56000E30859FB639A09429307900063E6974208
:10B5700093080C009307011B130C0B00130B040022
:10B58000232E91038324C101832941020324010155
:10B5900023202103B38C6741138A0B006FF0CF96F1
:10B5A0008326810E370600811306463823A0C80083
:10B5B00093871700130610009386160023A2C80075
:10B5C0002326F10E2324D10E1306700093888800E1
:10B5D000634CD606639805200327010293761A0070
:10B5E000B3E6E600639406006FE09F9283260103B2
:10B5F0000327C1021306700023A0D8008326810E02
:10B60000B387E70023A2E800938616002326F10EF5
:10B610002324D10E634ED64A938888000327010263
:10B620009386160023A06801B387E70023A2E800F1
:10B630002326F10E2324D10E130770006344D70094
:10B640006FE0DF8C6FE05FE61306410E93050C00A0
:10B6500013050D00EF301004631405E28325C10CBF
:10B660008327C10E9308C1106FF0DFF6832B010111
:10B67000130D0400138C04006FF0CFE093770A04DD
:10B68000638C072283274101930C0000232AE100E9
:10B6900003D907006FF05FB31306410E93050C004A
:10B6A00013050D00EF30007F631C05DC8327C10EFE
:10B6B0009308C1106FF00FB983268100B3879700FC
:10B6C00023A2980023A0D800130717002326F10E09
:10B6D0002324E10E9306700063C4E6006FE01F832D
:10B6E0006FE09FDC1306410E93050B0013050D0060
:10B6F000EF30407A6312052E834604008327C10E83
:10B700009308C1106FF0DFCA8327010F9305010A68
:10B710001305010B2328F10A8327410F2320010A77
:10B720002322010A232AF10A8327810F2324010AF5
:10B730002326010A232CF10A8327C10F232EF10AA5
:10B74000EF60C03683280101634205528347710CC4
:10B7500013077004635E972837070081130B873443
:10B76000232801002324010223220102232E0100A9
:10B77000137AFAF7930A3000930C3000930D00000F
:10B78000638407006FE09FE76FE0CFEB8327C10082
:10B79000130B04002320F7006FE00FFC13050B00D0
:10B7A00023209105EFE08FB88347710C934AF5FF92
:10B7B00093DAFA41232A21012328010023240102DC
:10B7C00023220102232E010083280104930C05008B
:10B7D000B37A5501930D0000638407006FE01FE208
:10B7E0006FE04FE6832601030327C10213067000B2
:10B7F00023A0D8008326810EB387E70023A2E800A8
:10B80000938616002326F10E2324D10E93888800F8
:10B810006340D62CE3D405E0130600FFB304B04028
:10B82000E3D4C52613090001930C70006F00C0001B
:10B83000938404FFE35A9924032781009387070127
:10B840009386160023A0E80023A228012326F10EE8
:10B850002324D10E93888800E3DCDCFC1306410E20
:10B8600093050C0013050D00EF30C062631A05C08C
:10B870008327C10E8326810E9308C1106FF05FFBF2
:10B88000938614001307890083278100B38CBC01C1
:10B890002322B9012320F9002326910F2324D10E5E
:10B8A00093077000E3C2D7BE938616009308870003
:10B8B000130907006FE01FBD93770A20638E071CF2
:10B8C00083274101930C0000232AE10003C90700EC
:10B8D0006FF09F8F93770A206384071A83274101B3
:10B8E000232AE10003890700935CF94193870C0048
:10B8F0006FE05FFA93F70B206388071683274101F7
:10B90000930C0000232AE10003C9070093071000ED
:10B910006FE0DFDC93770A20638E071283274101F3
:10B92000930C0000232AE10003C907006FE01FE326
:10B930008327C10F63C807188347710C130770046E
:10B94000635C974637070081130B07356FF05FE1A3
:10B9500003278100B38797009386160023A0E80091
:10B9600023A298002326F10E2324D10E1306700083
:10B97000938888006356D6C81306410E93050C00C1
:10B9800013050D00EF300051631C05AE8327C10E77
:10B990009308C1106FF0CFC6832781048325C104AB
:10B9A000130900003304F440138607001305040054
:10B9B000EFE08FA083C51C001306A00093060000D3
:10B9C0003338B0001385040093850900B38C0C0153
:10B9D000EF40501E6FF05FB5832B0101130C0B007D
:10B9E0006FF04FAA93079000E3E097B46FF05FB851
:10B9F00037070081130B47346FF09FD61306410EB3
:10BA000093050C0013050D00EF30C048631A05A61E
:10BA10008327C10E9308C1106FF00FBD930C600017
:10BA20006FF05F86832601023307DB00B384964004
:10BA30003308B74113890400635298C613090800FC
:10BA40006FF0CFC58327C100130B04002310F7004C
:10BA50006FE08FD083274101930C0000232AE1007F
:10BA600003A907006FE09FCF83274101930C0000DB
:10BA7000232AE10003A90700930710006FE01FC607
:10BA800083274101232AE10003A90700935CF941C0
:10BA900093870C006FE01FE083274101930C0000A7
:10BAA000232AE10003A907006FF00FF21306410EED
:10BAB00093050C0013050D00EF30C03D0357CC007B
:10BAC0006FE00FCB9307D002A303F10C6FF01FE7D9
:10BAD0001306410E93050C0013050D00EF30803B5B
:10BAE0006310059A8325C10C8327C10E8326810E1E
:10BAF0009308C110E3D405B26FF01FD2930D60001C
:10BB00006FE08FDF03270102130C0B00032B810270
:10BB1000232E8102032AC101B306EB000324010492
:10BB200083294104832A410263F4B6AF938D060052
:10BB30006FF00FAE0327C1019307D0FF6344F700F6
:10BB400063DAED009384E4FF93F7F4FD232AF10414
:10BB50006FE04FEE832701020327C1016344F726FC
:10BB600083278102930C070093F717006386070071
:10BB70008327C102B30CF7008327810293F70740A4
:10BB8000638607008327C101E34AF01293CAFCFFD2
:10BB900093DAFA41B3FA5C0193047006232401029C
:10BBA000232201026FE0CFFA8347710C930D00004E
:10BBB000638407006FE09FA46FE0CFA81306410ED7
:10BBC00093050B0013050D00EF30C02CE31605E0C4
:10BBD000834604008327C10E9308C110B38DDD0096
:10BBE0006FF08FFE930A010B1308C10D9307010D2F
:10BBF0001307C10C93860D001306300093850A00CD
:10BC000013050D00232211052328C10B2320C10594
:10BC1000232AD10B2322D103232CE10B2320E10380
:10BC2000232E610A232E6100EFA09FA50323C101EB
:10BC3000032F0102832E4102032E010483284104B5
:10BC4000130B0500930760043309BB01639AFB6281
:10BC500083460B0093070003E386F610930C010A5A
:10BC60008327C10C3309F9006FE00FD49307D0028A
:10BC7000A303F10C6FF0DFAD930A010B9307010DE5
:10BC80001308C10D1307C10C93860D001306200085
:10BC900093850A0013050D002328C10B2320C1053D
:10BCA000232AD10B2322D103232CE10B2320E103F0
:10BCB000232E610A232E6100EFA09F9C930770043E
:10BCC0000323C101032F0102832E4102032E01042D
:10BCD00083284104130B0500E396FBF683278102BA
:10BCE00093F7170063980758930770040327C10D53
:10BCF000232AF1046FE00FD11306410E93050C00C7
:10BD000013050D00EF300019630405006FE05FF7C5
:10BD10008324C10C8327C10E9308C1106FF08F9349
:10BD20008347710C232A21012324010223220102CB
:10BD3000232E0100938A0D00938C0D00930D0000BB
:10BD4000638407006FE09F8B6FE0CF8F1306410E77
:10BD500093050C0013050D00EF30C01363040500BC
:10BD60006FE01FF28324C10C032701028327C10E59
:10BD70009308C110B30497406FF04F92832781025C
:10BD80000327C10193F71700B3E7B701E354E004B9
:10BD90006396077A832CC10193046006832781028E
:10BDA00093F70740639E077093CAFCFF93DAFA414A
:10BDB000B3FA5C016FF09FDE37070081130BC734C5
:10BDC0006FF01F9A832701020327C10293047006B4
:10BDD000B38CE7008327C101E342F0FCB38CFC4045
:10BDE000938C1C0093CAFCFF93DAFA41B3FA5C010E
:10BDF0006FF0DFDAB7160081938E46A36FE08FF401
:10BE0000930700032304F10C9307800513672A00AE
:10BE1000A304F10C2324E102930730062328010038
:10BE2000130BC11463CEB7410323C10F93FBF4FD81
:10BE3000232A7105232C0104032E010F832E410FA9
:10BE4000032F810F136A2A106342033893071006E9
:10BE5000638EF454930710046384F4006FE08FAC96
:10BE6000930A010B13850A00232811052328C10B0F
:10BE7000232AD10B232CE10B232E610AEF80006FC4
:10BE80001306C10CEFD0CFF813860500930505000B
:10BE900013850A00EF80404E8327010B930C010AA3
:10BEA000130901092328F1088327410B1306010810
:10BEB00093050900232AF1088327810B13850C00C1
:10BEC0002320C104232CF1088327C10B2320010860
:10BED00023220108232EF108B707FC3F2326F1088F
:10BEE00023240108EF50D0500328010A032E410AF1
:10BEF000832E810A032FC10A93850C0013850A0043
:10BF00002328010B23220105232AC10B2322C1036D
:10BF1000232CD10B2320D103232EE10B232EE1016F
:10BF20002320010A2322010A2324010A2326010ACD
:10BF3000EF50D016032FC101832E0102032E4102C0
:10BF400003284104832801056316050093071000A8
:10BF50002326F10CB7070081938787362322F1024D
:10BF60009386FDFF232E4105232291062326B10748
:10BF7000232AA107232C8107930B0B002320810682
:10BF80002324310723281107138C0600232E610771
:10BF9000130D0800930D0E0093840E00130A0F007A
:10BFA0006F00800493850C0013850A002320C102D2
:10BFB000232EF101232CF10B232EC10A2328610B20
:10BFC000232A310B2320010A2322010A2324010AF8
:10BFD0002326010AEF50900C832FC1010326010292
:10BFE000130CFCFF6302050EB7070340130609009C
:10BFF00093850C0013850A00232EF1082320A10B42
:10C000002322B10B2324910A2326410B2328010864
:10C01000232A0108232C0108EF50903D13850A00C4
:10C02000EF80400F930505001304050013850A00F7
:10C030008329010B8324410B032B810B032AC10BA2
:10C04000EF80801E0327010B0326010493050900DE
:10C050002320E1080327410B13850C002328310915
:10C060002322E1080327810B232A9108232C61094D
:10C070002324E1080327C10B232E41092326E108CD
:10C08000EF60503783274102032B010A8329410ABD
:10C090003387870003470700832F810A0326C10ADD
:10C0A000232871052380EB00232281059307F0FFED
:10C0B000938B1B00130D0B00938D090093840F00CD
:10C0C000130A0600E310FCEE8328010793030B001C
:10C0D000938209003709FE3F93850C0013850A00FF
:10C0E00023201103232E8100032AC1058324410646
:10C0F000032401062328710A23227106232A510AE8
:10C1000023205106232CF10B232EF105232EC10AE7
:10C110002320C1042320010A2322010A2324010A27
:10C120002326210BEF505004832DC106032D410718
:10C13000032C8107032BC107832981068328010271
:10C140006340A00A8323410683220106832FC10591
:10C150000326010493850C0013850A002328710A25
:10C16000232A510A232CF10B232EC10A2320010A72
:10C170002322010A2324010A2326210BEF500072F7
:10C1800083280102631805008327C10193FC17006F
:10C1900063980C0483274104130600039386170059
:10C1A000B386DB0063C80700938B1B00A38FCBFE15
:10C1B000E39CDBFEB3876B412320F1026FE00F8528
:10C1C0002324410323280100130A0900B707008034
:10C1D00033C367009307D002232CF1046FF01FC70D
:10C1E0008327010593860B00232EF10C8327410240
:10C1F00003C6FBFF83C5F7006310B60213050003F7
:10C20000A38FA6FE8326C10D9387F6FF232EF10C84
:10C2100003C6F6FFE386C5FE9305160013059003DB
:10C2200093F5F50F6306A600A38FB6FE6FF09FF897
:10C230008327410283C5A700A38FB6FE6FF09FF747
:10C2400093851D0013050D0023281101EFB01F9EDB
:10C2500083280101130B05006308053E2328A10074
:10C260006FF09FBC930700032304F10C9307800732
:10C270006FF0DFB9930770043309BB01232AF1047F
:10C28000930C010A6FD05FF203278100B3879700F8
:10C290009386160023A0E80023A298002326F10E1F
:10C2A0002324D10E130670006358D6B61306410E30
:10C2B00093050C0013050D00EF20D03D630405002D
:10C2C0006FE01F9C8327C10E8326810E9308C11047
:10C2D0006FF0CFB4930B0A006FE0CFDF63940D00D3
:10C2E000930D10000323C10F032E010F832E410F66
:10C2F000032F810F13690A10E34403EC930A010B27
:10C300001308C10D9307010D1307C10C93860D008F
:10C310001306200093850A0013050D002322110542
:10C320002328C10B2320C105232AD10B2322D103AB
:10C33000232CE10B2320E103232E610A232E61002D
:10C34000EFA00FB40323C10123244103032F0102F3
:10C35000832E4102032E010483284104130B0500A0
:10C36000130A090023280100232C01046FF01F97F2
:10C370009307F0FF2326F1006FD05FC09306610D95
:10C380006318060093060003230BD10C9306710D6E
:10C390001307011B938707033386E6402380F600CB
:10C3A0009307D60D232CF1026FD05FF6930A010B91
:10C3B00013850A00232811052328C10B232AD10B3A
:10C3C000232CE10B232E610AEF80401A1306C10CC7
:10C3D000EFD00FA4138605009305050013850A000E
:10C3E000EF7090798327010B930C010A130901095F
:10C3F0002328F1088327410B130601089305090040
:10C40000232AF1088327810B13850C002320C10404
:10C41000232CF1088327C10B2320010823220108C4
:10C42000232EF108B707FC3F2326F1082324010837
:10C43000EF50007C0328010A032E410A832E810A53
:10C44000032FC10A93850C0013850A002328010BD2
:10C4500023220105232AC10B2322C103232CD10B44
:10C460002320D103232EE10B232EE1012320010AF7
:10C470002322010A2324010A2326010AEF50004245
:10C48000032FC101832E0102032E41020328410420
:10C490008328010563160500930710002326F10C7D
:10C4A000B7070081938747352322F1026FF05FAB16
:10C4B00023280100138A07006FF05FD193047006F0
:10C4C0000326C1039306F00F834706006388D7183D
:10C4D0000327C101130500009305000063DEE70098
:10C4E0003307F740834716006384070493851500DC
:10C4F00013061600E394D7FE232EC102232EE1007B
:10C500002322B1022324A1020327810283274102AF
:10C51000B387E70003278104B387E702B38C970151
:10C5200093CAFCFF93DAFA41B3FA5C016FD05FE281
:10C5300083470600130515006FF0DFFB8327C10258
:10C5400093046006B30CF700B38CBC016FF01F8539
:10C550008327810293F71700639407006FD01FDDD4
:10C560006FD05FDC930C010A93850C0013850A00E1
:10C57000232211052328C10B2320C105232AD10B17
:10C580002322D103232CE10B2320E103232E610A74
:10C59000232E61002320010A2322010A2324010AF9
:10C5A0002326010AEF50802F0323C101032F01022C
:10C5B000832E4102032E010483284104630205EA0D
:10C5C00093071000B387B7412326F10C3309F90014
:10C5D0006FD09FBD639A0700930A10009304600612
:10C5E000930C10006FF08FDB8327C1029304600669
:10C5F000938C1700B38CBC0193CAFCFF93DAFA4109
:10C60000B3FA5C016FF08FD9138708006FF0CFA7E2
:10C610008327410183AD07009387470063D40D0052
:10C62000930DF0FF83441400232AF1001304070044
:10C630006FD04FF99307C0002320FD009307F0FF50
:10C640002326F1006FD09F930357CC009367070414
:10C65000138707002316FC006FD09F91232401024B
:10C66000232201026FF05FEA93072000232CF102DE
:10C670006FD0DFC983A74506130101FD232861019F
:10C680002326110223248102232291022320210345
:10C69000232E3101232C4101232A5101232671012C
:10C6A0002324810113972701130B06006358070AFF
:10C6B00083278600832B0600138905009309050054
:10C6C000930AF0FF6388070803AC4B0003A40B0038
:10C6D000135A2C0063060A06930400006F00C00082
:10C6E00013044400630C9A04832504001306090014
:10C6F00013850900EF10C07A93841400E31255FFEC
:10C700001305F0FF8320C1020324810223240B00C0
:10C7100023220B0083244102032901028329C10142
:10C72000032A8101832A4101032B0101832BC100CC
:10C73000032C8100130101036780000083278B0015
:10C74000137CCCFFB38787412324FB00938B8B00A2
:10C75000E39C07F6130500006FF0DFFAEF10900579
:10C760006FF05FFA03278600630407006FF09FF005
:10C77000232206001305000067800000130101ED6D
:10C78000232E3111232C411123267111232611123E
:10C79000232481122322911223202113232A5111B1
:10C7A0002328611123248111232291112320A11117
:10C7B000232EB10F2328D100130A05009389050009
:10C7C000930B06006306050083278503638E075ECF
:10C7D0000397C900931707019316270193D7070101
:10C7E00063CA0602B727000083A64906B367F700AD
:10C7F0009397070137E7FFFF93D707411307F7FF29
:10C8000033F7E6002396F9009397070123A2E90680
:10C8100093D7070113F787006300074003A70901B7
:10C82000630C073E93F7A7011307A0006386E74058
:10C83000B7170081938747A5371B00819304C10474
:10C84000232AF1003719008193070BBC138C0B00CE
:10C85000232091042324010423220104232C01001A
:10C86000232E01002322010223200102232601009E
:10C870002324F100130909BD938B040083470C00A6
:10C880006388072613040C0013075002638EE742E7
:10C890008347140013041400E39A07FEB30C844189
:10C8A00063088425032781048327410423A08B0187
:10C8B0003387EC009387170023A29B012324E10414
:10C8C0002322F10493067000938B8B0063D0F60251
:10C8D000E30A073A130601049385090013050A00C9
:10C8E000EFF05FD9631A0520938B04000327C10082
:10C8F00083470400330797012326E100638A071E5C
:10C9000003471400130C1400A30D0102930AF0FF57
:10C9100023220100130B0000930CA005130D9000BF
:10C920001306A002130C1C00930707FE63E8FC0427
:10C930008326410193972700B387D70083A7070079
:10C940006780070023220100930707FD832541002C
:10C9500003470C00130C1C0093962500B386B60009
:10C9600093961600B387D7002322F100930707FDA3
:10C97000E37EFDFC930707FEE3FCFCFA630A07165F
:10C980002306E108A30D0102930C1000130D100003
:10C990001304C108930A0000937F2B0063840F00E7
:10C9A000938C2C0003274104137F4B0883278104B9
:10C9B000930617001386060063180F0083254100B5
:10C9C000B38D9541E342B0098345B10393868B0053
:10C9D000638C05021307B1039387170023A0EB00B4
:10C9E0001307100023A2EB002324F1042322C10427
:10C9F000130770006340C77E13070600938B060081
:10CA00001306160093868600638E0F041307C10376
:10CA10009387270023A0EB001307200023A2EB003D
:10CA20002324F1042322C10413077000E350C7003C
:10CA3000E384072A130601049385090013050A00FD
:10CA40002324E103EFF01FC36318050A0327410401
:10CA500083278104032F81029306410513061700E3
:10CA6000938B0400930500086306BF5AB38AAA415A
:10CA700063425069B307FD0023A08B0023A2AB01E2
:10CA80002324F1042322C104130770006352C70258
:10CA9000E38E070A130601049385090013050A00B3
:10CAA000EFF05FBD631A05048327810493860400B9
:10CAB00013734B006308030003274100B30B974136
:10CAC000E344700B032441006354940113840C006D
:10CAD0000327C100330787002326E1006398076C12
:10CAE00083470C0023220104938B0400E39C07D8A6
:10CAF00083278104E39A076483D7C90093F7070467
:10CB0000E39207688320C112032481120325C10028
:10CB100083244112032901128329C111032A81119F
:10CB2000832A4111032B0111832BC110032C811087
:10CB3000832C4110032D0110832DC10F130101130C
:10CB40006780000013050A00EFA0DFE3832745009C
:10CB5000138507002320F102EFC05FFD9307050056
:10CB600013050A00138407002322F102EFA09FE1BE
:10CB7000832785001306A002232EF100E318042A60
:10CB800003470C006FF01FDA03470C00136B0B0216
:10CB90006FF05FD9136B0B0193770B026384071659
:10CBA000832701019387770093F787FF03A7470047
:10CBB00003AD0700938787002328F100930C07003B
:10CBC000634A07161307F0FF930D0B006388EA0012
:10CBD00033679D01937DFBF7E30C070AE3960C1680
:10CBE00013079000E362A71793070D03A307F10E45
:10CBF000138B0D00130D10001304F10E938C0A001B
:10CC000063D4AA01930C0D008347B103B337F0003E
:10CC1000B38CFC006FF05FD89385090013050A0000
:10CC2000EF70CFACE310055683D7C9001307A000FF
:10CC300093F7A701E39EE7BE8397E900E3CA07BE27
:10CC40008326010113860B009385090013050A0052
:10CC5000EF00D0582326A1006FF0DFEA136B0B0121
:10CC600093770B02638A0706832701019387770076
:10CC700093F787FF03AD070083AC470093878700D6
:10CC80002328F100937DFBBF13070000A30D0102D1
:10CC90009306F0FF6384DA0CB3669D0113FBFDF786
:10CCA0006390065A639C0A306318077E13FD1D00CB
:10CCB0001304010FE3040DF493070003A307F10E1F
:10CCC0001304F10E6FF09FF3B30C8441E31C84BD99
:10CCD000834704006FF09FC28326010193770B0105
:10CCE00013874600E39C071693770B04E388073805
:10CCF00083270101930C00002328E10003DD0700D6
:10CD00006FF05FF88326010193770B0113874600CC
:10CD1000E394071093770B04E38207328327010122
:10CD20002328E100039D0700935CFD4113870C005D
:10CD3000E35A07E83337A001B30E9041B38CEE40BD
:10CD40001307D002A30DE1029306F0FF330DA041BB
:10CD5000930D0B0013071000E390DAF49306100014
:10CD6000E30ED7E6930620006304D7261304010FD1
:10CD70009397DC0113777D00135D3D0013070703D4
:10CD800033EDA70193DC3C00A30FE4FEB3679D01E4
:10CD9000130604001304F4FFE39C07FC93F71D0043
:10CDA0006382072693070003630EF7241306E6FF4A
:10CDB000A30FF4FE9307010F338DC740138B0D00B3
:10CDC000130406006FF09FE3EF70DFA46FF05FA025
:10CDD00083270101A30D010203A40700938D4700DF
:10CDE000E30004229307F0FFE388FA1213860A0097
:10CDF0009305000013050400EFB00FE6E3000536CD
:10CE0000330D85402328B101930A00006FF01FDF26
:10CE100003270101A30D0102930C100083270700D3
:10CE2000130747002328E1002306F108130D100023
:10CE30001304C1086FF01FB6832701013787FFFF76
:10CE40001347078303AD0700938747002328F100AA
:10CE5000B707008193874735231EE102930C00003A
:10CE6000936D2B00232CF100130720006FF01FE2BD
:10CE700003470C009307C006E306F716136B0B017C
:10CE80006FF05FAA03470C0093078006E304F714D2
:10CE9000136B0B046FF01FA9936D0B0193F70D0239
:10CEA00063840760832701011307100093877700CD
:10CEB00093F787FF03AD070083AC47009387870094
:10CEC0002328F1006FF09FDC03470C00136B0B0865
:10CED0006FF05FA58326010103470C0083A70600BE
:10CEE000938646002328D1002322F100E3DC07A229
:10CEF000B307F0402322F100136B4B006FF09FA2A9
:10CF000003470C00136B1B006FF0DFA18347B103D5
:10CF100003470C00E39807A093070002A30DF1025A
:10CF20006FF05FA003470C00136B4B006FF09F9FE7
:10CF30009307B00203470C00A30DF1026FF09F9E10
:10CF400003470C0093061C00E30AC724930707FD60
:10CF5000138C0600930A0000E368FD9C03470C0055
:10CF600093962A00B38A5601939A1A00B38AFA005C
:10CF7000930707FD130C1C00E372FDFE6FF0DF9AB0
:10CF80008326010193770B0203A7060093864600D0
:10CF90002328D100639A076A93770B01E39C070467
:10CFA00093770B04E390071413730B20E30403043B
:10CFB0008327C1002300F7006FF05F8C93061000F9
:10CFC000E30ED71A93062000930D0B00E310D7DA77
:10CFD000832681011304010F9377FD00B387F600C8
:10CFE00003C70700135D4D009397CC0133EDA701F4
:10CFF00093DC4C00A30FE4FEB3679D011304F4FF20
:10D00000E39C07FC9307010F338D8740138B0D00C2
:10D010006FF0DFBE83254100B38D9541E358B0A585
:10D0200093050001E3D6B517930E0001130F7000AE
:10D030006F00800113062700938B8B001387060077
:10D04000938D0DFF63DCBE059387070193061700E0
:10D0500023A02B0123A2DB012324F1042322D104EA
:10D06000E35ADFFC63800716130601049385090069
:10D0700013050A00EFF00FE0E31005A803274104B1
:10D08000930E0001938D0DFF83278104938B040081
:10D0900013061700130F7000E3C8BEFB93050600CC
:10D0A00013858B00B387B70123A02B0123A2BB01FB
:10D0B0002324F1042322B10413077000635AB752EA
:10D0C0006386077E130601049385090013050A0091
:10D0D000EFF04FDAE31205A203274104B38AAA4115
:10D0E000832781049306410513061700938B0400E0
:10D0F000E35250999305000163D0557B93080001DA
:10D10000930D70006F00800113062700938B8B0036
:10D1100013870600938A0AFF63DA5805938707018D
:10D120009306170023A02B0123A21B012324F10443
:10D130002322D104E3DADDFC63820706130601042F
:10D140009385090013050A00EFF0CFD2E316059A84
:10D150000327410493080001938A0AFF832781046F
:10D16000938B040013061700E3CA58FB93858B00CA
:10D17000B387570123A02B0123A25B012324F104D1
:10D180002322C104130770006346C72C1306160040
:10D1900093868500938B05006FF0DF8D13061000DA
:10D1A00013070000938B04006FF0DFF613060104F1
:10D1B0009385090013050A00EFF0CFCBE302059237
:10D1C0006FF09F931306100013070000938B040069
:10D1D0006FF01FE7638C0730130601049385090085
:10D1E00013050A002326E1032324F103EFF08FC87F
:10D1F000E31405900327410483278104032FC10210
:10D20000832F81029306410513061700938B0400B8
:10D210006FF08FFF9307C1032326F10493072000CB
:10D220002328F10413061000930641051307060096
:10D23000938B06001306170093868B006FF09F8276
:10D24000930D0B006FF09FB1130600016350B6738E
:10D2500013860B00930E0001930B040093027000E1
:10D26000138409002324F10393890D00930D0C000E
:10D27000138C0A00930A0F006F00C00113052700EA
:10D280001306860013870600938909FF63DE3E05B7
:10D290009306170083258100938707012322D60177
:10D2A0002320B6002324F1042322D104E3D8D2FCA6
:10D2B00063860708130601049305040013050A009A
:10D2C000EFF04FBB6316054C03274104930E00019A
:10D2D000938909FF8327810413860400130517002F
:10D2E00093027000E3C63EFB832F8102138F0A0076
:10D2F00093050500930A0C00138C0D00938D090013
:10D300009309040013840B00930B0600032781008C
:10D31000B387B70123A2BB0123A0EB002324F104B0
:10D320002322B104130770006342B71E938B8B0056
:10D3300013861500138705006FF00FE9130700002F
:10D3400013051000138604006FF01FF4232201045C
:10D3500013734B006302030E03274100B30B974185
:10D36000635C700D938604001307000103264104DB
:10D3700063527761130D0001930D70006F008001FF
:10D38000130526009386860013060700938B0BFF78
:10D39000635A7D05832581009387070113071600D3
:10D3A00023A0B60023A2A6012324F1042322E10432
:10D3B000E3D8EDFC638A0706130601049385090090
:10D3C00013050A00EFF00FAB631805F203264104C2
:10D3D000938B0BFF832781049386040013051600AB
:10D3E000E34A7DFB9305050003278100B38777019E
:10D3F00023A2760123A0E6002324F1042322B10412
:10D40000130770006350B7EC63880702130601042A
:10D410009385090013050A00EFF0CFA5631E05EC04
:10D42000832781046FF00FEA130510001306000034
:10D43000938604006FF09FF5032441006354940128
:10D4400013840C008327C100B38787002326F100D3
:10D450006FF00FE963820734130601049385090016
:10D4600013050A00EFF00FA1631805E80326410435
:10D47000832781049306410513061600938B04004D
:10D480006FF04FDF23220104938B04006FF00FC66F
:10D49000639C0AF4138B0D00930A0000130D000027
:10D4A0001304010F6FF08FF58326010193F70D012F
:10D4B000138746006398071493F70D046380073AB7
:10D4C00083270101930C00002328E10003DD0700FE
:10D4D000130710006FF08FFB930641051306100031
:10D4E00013070000938B04006FF0CFD763800F18F1
:10D4F0009307C1032326F104930720002328F10496
:10D5000013071000930B41056FF0DFD263820722EF
:10D51000130601049385090013050A002326E1037D
:10D520002324F103EFF00F95631805DC0327410472
:10D5300083278104032FC102832F8102938B040070
:10D54000130617006FF04FC893F70D4023244103D3
:10D5500023263103138A0C0093090D00130B0000DE
:10D56000032DC1011304010F938C07006F004002CB
:10D570001306A000930600001385090093050A0016
:10D58000EF205063630E0A3093090500138A0500EB
:10D590001306A000930600001385090093050A00F6
:10D5A000EF30802413050503A30FA4FE130B1B000B
:10D5B0001304F4FFE38E0CFA83460D00E39A66FB36
:10D5C0009307F00FE306FBFA63140A189307900021
:10D5D00063E037199307010F232EA101032A81026B
:10D5E0008329C102338D8740138B0D006FF00FE14B
:10D5F000138615009306850013870500930B05001D
:10D600006FF0CFC62328E10003AD0600930C0000A5
:10D61000130710006FF08FE703AD06002328E10029
:10D62000935CFD4113870C006FF08FD98327C101F4
:10D6300003470C00638807AE83C70700638407AE07
:10D64000136B0B406FF00FAE8326C10093D7F641EA
:10D650002320D7002322F7006FF04FA203AD06006E
:10D66000930C00002328E1006FF0CFE113070000C6
:10D670009306410513061000938B04006FF08FBED4
:10D68000930D0B006FF09F81B7070081938787365A
:10D69000232CF10093770B02638007068327010197
:10D6A0009387770093F787FF03AD070083AC4700AC
:10D6B000938787002328F10093761B00638E060072
:10D6C000B3669D01638A060093060003230ED10210
:10D6D000A30EE102136B2B00937DFBBF1307200009
:10D6E0006FF0CFDAB707008193874735232CF1001D
:10D6F00093770B02E39407FA0326010193770B015A
:10D7000093064600638A070A032D0600930C000067
:10D710002328D1006FF05FFA13050400EFC00FC19A
:10D72000130D05002328B101930A00006FF00FCDFF
:10D730000347B103631A0718E39E0FAC13070000F9
:10D740001306100093064105938B04006FF08FB110
:10D750008327410283250102130B00003304F440A8
:10D760001386070013050400EFC00FC583451D0095
:10D770001306A000930600003337B000138509009C
:10D7800093050A00330DED00EF20D0426FF0DFDF8C
:10D79000930904006FF04FB61307100093070D00B4
:10D7A000232681042328A1052324A1052322E104A3
:10D7B000930641056FF0CFAF93770B0463820706A2
:10D7C00083270101930C00002328D10003DD07000B
:10D7D0006FF09FEE03471C00136B0B20130C1C0013
:10D7E0006FF04F9403471C00136B0B02130C1C00CB
:10D7F0006FF04F938327C1002320F7006FF00F884D
:10D8000093076000138D0A0063EC570B370E0081FD
:10D81000930C0D002328B1011304CE376FF08F97BE
:10D8200093770B206388071083270101930C000076
:10D830002328D10003CD07006FF01FE893770B205A
:10D84000638E070C832701012328E100038D070065
:10D85000935CFD4113870C006FF08FB693F70D209A
:10D860006382070A83270101930C00002328E1004B
:10D8700003CD0700130710006FF04FC193770B2003
:10D880006388070683270101930C00002328E10029
:10D8900003CD07006FF00FBF938506006FF05F8D1B
:10D8A00093079000E3E237CF6FF0DFD29306410594
:10D8B0001306100013070000938B04006FF00F9BFA
:10D8C000130D60006FF09FF49307B1032326F1045A
:10D8D000930710002328F104130610009306410556
:10D8E0006FF08F918327C1002310F7006FE01FF9BD
:10D8F00083270101930C00002328E10003AD0700FA
:10D900006FF04FB883270101930C00002328E1003A
:10D9100003AD0700130710006FF04FB78327010115
:10D920002328E10003AD0700935CFD4113870C0041
:10D930006FF00FA983270101930C00002328D10069
:10D9400003AD07006FF05FD713060104938509004C
:10D9500013050A00EFE01FD26FF00F9A138D0A0033
:10D960002328B101930A00006FF04FA993850600A8
:10D970006FF0DF99930516006FF01FA7930D0B0052
:10D980006FF08FA69307F0FF2326F1006FF08F97BB
:10D9900013850600930506006FF0CFF08327010181
:10D9A00083AA07009387470063D40A00930AF0FF15
:10D9B00003471C002328F100138C06006FE09FF63C
:10D9C0003727008193070500032587BB93060600D0
:10D9D00013860500938507006FE05FDA83D7C500E3
:10D9E00003AE450603D3E50083A8C50103A845029D
:10D9F000130101B893F7D7FF13070040232C81468A
:10DA0000231AF10013840500930701079305810091
:10DA1000232A914623282147232E11461309050066
:10DA20002326C107231B61002322110323260103A0
:10DA30002324F100232CF1002328E100232EE10010
:10DA400023200102EFE09FD393040500635C0502ED
:10DA50008357410193F70704638807008357C40085
:10DA600093E707042316F4008320C147032481476A
:10DA7000032901471385040083244147130101480A
:10DA8000678000009305810013050900EF60DF9DAA
:10DA9000E30005FC9304F0FF6FF09FFBB7170081D4
:10DAA00003A3877167000300638405029307F00FE7
:10DAB00063E8C7002380C5001305100067800000DD
:10DAC0009307A0082320F5001305F0FF67800000EE
:10DAD0001305000067800000130101FF1387050094
:10DAE00023248100232291009305060013040500DE
:10DAF000B7240081138606001305070023261100B2
:10DB000023A804C6EF201F869307F0FF630CF500DF
:10DB10008320C100032481008324410013010101FB
:10DB20006780000083A704C7E38407FE8320C10049
:10DB30002320F40003248100832441001301010108
:10DB400067800000B385C502130101FF2324810013
:10DB500023261100EFA08F8D130405006308050232
:10DB60000326C5FF130740021376C6FF1306C6FF40
:10DB70006360C706930630019307050063E2C6029F
:10DB800023A0070023A2070023A407008320C100CD
:10DB900013050400032481001301010167800000C4
:10DBA00023200500232205009307B00163F0C7047A
:10DBB000232405002326050093070501E312E6FC54
:10DBC0002328050093078501232A05006FF05FFBDA
:10DBD00093050000EF300FE48320C100130504001B
:10DBE0000324810013010101678000009307850071
:10DBF0006FF01FF9130101FF2324810023229100FC
:10DC000013040500B72400811385050023261100A5
:10DC100023A804C6EF200FE49307F0FF630CF50080
:10DC20008320C100032481008324410013010101EA
:10DC30006780000083A704C7E38407FE8320C10038
:10DC40002320F400032481008324410013010101F7
:10DC500067800000130101FF2326110023248100A7
:10DC600023229100232021016380050213840500F3
:10DC7000930405006306050083278503638C070A68
:10DC80008317C400639207028320C100032481002C
:10DC90001309000083244100130509000329010032
:10DCA000130101016780000093050400138504003F
:10DCB000EF60CFD58327C40213090500638A0700EC
:10DCC0008325C40113850400E7800700634C050623
:10DCD0008357C40093F70708639E07068325040350
:10DCE000638C0500930704046386F5001385040024
:10DCF000EF60DFCA232804028325440463880500FB
:10DD000013850400EF609FC923220404EF609FB1D4
:10DD100023160400EF605FB18320C100032481005B
:10DD200083244100130509000329010013010101A7
:10DD300067800000EF601FAE8317C400E38607F41E
:10DD40006FF09FF68357C4001309F0FF93F707089D
:10DD5000E38607F88325040113850400EF601FC4E0
:10DD60006FF0DFF7B72700819305050003A587BB98
:10DD70006FF05FEE130101FD23248102232E310198
:10DD8000232861012326110223229102232021034B
:10DD9000232C4101232A5101130B0500938905000F
:10DDA00013040600EF905FC7930710006310F5029D
:10DDB0009387F9FF1307E00F636AF70013F7F90F72
:10DDC0002306E100130910006F00C0029306C4058A
:10DDD000138609009305C10013050B00EF20C04C0A
:10DDE0009307F0FF130905006304F50A630E0508A5
:10DDF0000347C10093040000130AF0FF930AA00038
:10DE00006F00800283270400938617002320D4002C
:10DE10002380E700938414009307C100B387970021
:10DE200063F4240703C70700832784009387F7FF61
:10DE30002324F400E3D807FC83268401930507001C
:10DE40001306040013050B0063C4D700E31C57FB43
:10DE5000EF20C02BE31045FD1309F0FF8320C10222
:10DE600003248102832441028329C101032A810101
:10DE7000832A4101032B0101130509000329010233
:10DE80001301010367800000138909006FF01FFD73
:10DE90008357C40093E707042316F4006FF01FFCB8
:10DEA0008317C6001397270163400702032746061E
:10DEB000B7260000B3E7D700B72600003367D700C6
:10DEC0002316F6002322E6066FF0DFEA130101FEB7
:10DED000B7270081232C810003A487BB232E1100C8
:10DEE0001386050093050500630604008327840359
:10DEF000638007048317C600139727016340070256
:10DF000003274606B7260000B3E7D700B726000070
:10DF10003367D7002316F6002322E6061305040014
:10DF2000032481018320C101130101026FF09FE4EA
:10DF30002324A100130504002326C100EF609F8D58
:10DF40000326C100832581006FF0DFFA130101FF72
:10DF50001387050023248100232291001304050068
:10DF6000B72400819305060013050700232611003E
:10DF700023A804C6EF200FB19307F0FF630CF50050
:10DF80008320C10003248100832441001301010187
:10DF90006780000083A704C7E38407FE8320C100D5
:10DFA0002320F40003248100832441001301010194
:10DFB0006780000083278600638E073283D7C50001
:10DFC000130101FD23248102232C4101232A510145
:10DFD000232611022322910223202103232E310123
:10DFE0002328610123267101232481012322910129
:10DFF0002320A10113F78700130A0600930A0500E6
:10E00000138405006306070803A7050163020708D8
:10E0100013F7270083240A00630C070883274402B0
:10E020008325C401370B0080930900001309000009
:10E03000134B0BC01386090013850A006302090401
:10E040009306090063742B0193060B00E780070019
:10E050006358A02883278A00B389A9003309A940FF
:10E060003385A7402324AA00630A0520832744029E
:10E070008325C4011386090013850A00E31209FCF5
:10E0800083A9040003A94400938484006FF09FFADD
:10E090009305040013850A00EF505FE5631C053A01
:10E0A0008357C40083240A0013F72700E31807F6F8
:10E0B00013F7170063140724832C8400032504003E
:10E0C000370B0080934BEBFF130C0000130900008B
:10E0D000134BFBFF630E090E13F70720630C072495
:10E0E000138D0C006362992F13F70748630A070822
:10E0F000832944018325040113071900939619000D
:10E10000B386360193D9F601330DB540B389D900F2
:10E1100093D919403307A7011386090063F6E90074
:10E12000930907001306070093F707406384072E3F
:10E130009305060013850A00EF905FAF930C05006E
:10E14000630205308325040113060D00EF00C03D76
:10E150008357C40093F7F7B793E707082316F40033
:10E160003385AC01B387A941232894012320A4005F
:10E17000232A3401930C09002324F400130D090011
:10E1800013060D0093050C00EF00C04B032784001D
:10E190008327040093090900B30C9741B387A701B3
:10E1A000232494012320F4001309000003268A008D
:10E1B000330C3C01B309364123243A016380090C36
:10E1C000832C8400032504008357C400E31609F060
:10E1D00003AC040003A94400938484006FF09FEF14
:10E1E00083A9440003AC040093848400E38A09FEFD
:10E1F000138609009305A00013050C00EFA0CFA51E
:10E200006304051213051500330B854193070B00BA
:10E21000938B090063F43701938B070003250400F7
:10E22000832704018326440163F8A700032984009F
:10E23000338926016342790963C8DB1A83274402C4
:10E240008325C40113060C0013850A00E78007002C
:10E25000130905006356A008330B2B41130510006A
:10E26000630A0B1603268A00330C2C01B38929415B
:10E270003309264123242A01631A090813050000E3
:10E280008320C10203248102832441020329010265
:10E290008329C101032A8101832A4101032B010142
:10E2A000832BC100032C8100832C4100032D01002E
:10E2B000130101036780000093050C001306090099
:10E2C000EF004038832704009305040013850A00FB
:10E2D000B38727012320F400EF600F99E30E05F6C2
:10E2E0008317C40093E707042316F4001305F0FF17
:10E2F0006FF01FF91305000067800000130B00008A
:10E3000013050000130C000093090000E38A09ECD8
:10E31000E31E05EE138609009305A00013050C000B
:10E32000EFA08F93E31005EE93871900138B07007E
:10E330006FF01FEE8327040163E2A70483274401E3
:10E34000636EF9029306090063F42B0193060B0038
:10E35000B3C6F602032744028325C40113060C004A
:10E3600013850A00B386F602E7000700930905004B
:10E37000E358A0F6330939416FF05FE393890C004D
:10E3800063749901930909001386090093050C0031
:10E39000EF00402B8327840003270400B387374115
:10E3A000330737012324F4002320E400E39407FC1F
:10E3B0009305040013850A00EF600F8BE31205F24A
:10E3C000330939416FF09FDE930C0900130D0900EA
:10E3D0006FF01FDB9305040013850A00EF60CF8800
:10E3E000E30205E86FF0DFEF13860B0093050C00E6
:10E3F000EF004025832784000326040013890B00C7
:10E40000B3877741330676012324F4002320C40028
:10E410006FF09FE413850A00EF00803B930C05002A
:10E42000E31005D48325040113850A00EF600FD79C
:10E430008317C4001307C00023A0EA0093F7F7F77F
:10E440006FF05FEA1307C0008317C40023A0EA003F
:10E450006FF05FE91305F0FF6FF09FE2130101FF1A
:10E46000232481002322910013040500B724008196
:10E47000138505002326110023A804C6EF101FE50D
:10E480009307F0FF630CF5008320C1000324810093
:10E4900083244100130101016780000083A704C7A2
:10E4A000E38407FE8320C1002320F40003248100BD
:10E4B000832441001301010167800000130101FF63
:10E4C0001387050023248100232291009305060071
:10E4D00013040500B7240081138606001305070006
:10E4E0002326110023A804C6EF10DFE19307F0FFF5
:10E4F000630CF5008320C1000324810083244100C4
:10E50000130101016780000083A704C7E38407FEAD
:10E510008320C1002320F4000324810083244100D0
:10E520001301010167800000B3C7A50093F737000E
:10E53000B308C500639207069307300063FEC70463
:10E5400093773500130705006398070613F6C8FF95
:10E55000930706FE636CF708637CC7029386050089
:10E560009307070003A80600938747009386460099
:10E5700023AE07FFE3E8C7FE9307F6FFB387E74044
:10E5800093F7C7FF938747003307F700B385F5007C
:10E59000636817016780000013070500E37C15FF1F
:10E5A00083C705001307170093851500A30FF7FE17
:10E5B000E36817FF6780000083C605001307170094
:10E5C00093773700A30FD7FE93851500E38007F8F4
:10E5D00083C605001307170093773700A30FD7FEF4
:10E5E00093851500E39A07FC6FF05FF683A645005C
:10E5F00083A2050083AF850003AFC50083AE05018C
:10E6000003AE450103A3850103A8C5012322D7005A
:10E6100083A60502232057002324F7012326E701C0
:10E620002328D701232AC701232C6700232E0701A3
:10E630002320D7021307470293854502E368F7FAC0
:10E640006FF09FF163F6A502B387C5006372F50210
:10E650003307C500630A060E83C6F7FF9387F7FFEB
:10E660001307F7FF2300D700E398F5FE678000004B
:10E670009307F00063E8C702930705009306F6FFCF
:10E68000630C060C93861600B386D70003C70500FB
:10E690009387170093851500A38FE7FEE398D7FEB5
:10E6A00067800000B3E7A50093F737006390070A7F
:10E6B000930806FF93F808FF9388080133081501B3
:10E6C000138705009307050083260700130707013A
:10E6D0009387070123A8D7FE832647FF23AAD7FEE7
:10E6E000832687FF23ACD7FE8326C7FF23AED7FE42
:10E6F000E31CF8FC1377C600B38515011378F60008
:10E70000630E07041387050093880700130E30007B
:10E710000323070013074700B306E84023A068005F
:10E72000B386D50093884800E364DEFE1307C8FF74
:10E730001377C7FF1307470013763600B387E70048
:10E74000B385E5006FF09FF3678000009306F6FF46
:10E75000930705006FF01FF36780000013060800A1
:10E760006FF0DFF1130101FF1387050023248100FF
:10E77000232291009305060013040500B7240081AD
:10E7800013860600130507002326110023A804C6DC
:10E79000EF105FBA9307F0FF630CF5008320C10010
:10E7A00003248100832441001301010167800000DC
:10E7B00083A704C7E38407FE8320C1002320F4005D
:10E7C00003248100832441001301010167800000BC
:10E7D000130101FD2320210323261102232481029A
:10E7E00023229102232E3101232C4101232A51019E
:10E7F00023286101232671012324810113090600C6
:10E80000638405221384050093090500EF901FD24D
:10E810009304B9009307600163FE970E93F484FF9D
:10E820001387040063CE040E63EC240F8327C4FF18
:10E83000930A84FF13FAC7FF338B4A01635CEA181B
:10E84000B7160081938B467A03A68B0083264B0074
:10E85000630E662313F6E6FF3306CB00032646005D
:10E86000137616006314061A93F6C6FF3306DA0011
:10E87000635EE63293F7170063940702032C84FF6C
:10E88000338C8A4183274C0093F7C7FFB386D700A8
:10E89000B38B460163DAEB34B30BFA0063D2EB0CB3
:10E8A0009305090013850900EF904FB8130905007F
:10E8B000630C05048327C4FF130785FF93F7E7FF65
:10E8C000B387FA006382E7301306CAFF930740025A
:10E8D00063E6C7301307300183260400636CC72644
:10E8E000930705001307040023A0D70083264700E1
:10E8F00023A2D7000327870023A4E7009305040081
:10E9000013850900EF608F8913850900EF905FC2BE
:10E910006F00C0019304000113070001E3F824F124
:10E920009307C00023A0F900130900008320C1024F
:10E9300003248102832441028329C101032A810126
:10E94000832A4101032B0101832BC100032C810089
:10E950001305090003290102130101036780000068
:10E960008327CC0003278C001306CAFF93064002BE
:10E970002326F70023A4E70013098C00330B7C0146
:10E9800063E4C62E930530010327040093070900B2
:10E9900063F2C5022324EC00032744009307B0016F
:10E9A0002326EC0063E2C7300327840093070C01A1
:10E9B0001304840023A0E70003274400138A0B00FC
:10E9C000930A0C0023A2E700032784001304090024
:10E9D00023A4E70083A74A0033079A409306F00078
:10E9E00093F7170063ECE606B367FA0023A2FA0078
:10E9F00083274B0093E717002322FB0013850900B0
:10EA0000EF901FB3130904006FF05FF293F7170044
:10EA1000E39807E8032C84FF338C8A4183274C005A
:10EA200093F7C7FF6FF05FE7032481028320C102E1
:10EA300083244102032901028329C101032A8101A0
:10EA4000832A4101032B0101832BC100032C810088
:10EA500093050600130101036F904F9DB3E79700E4
:10EA600023A2FA00B3859A001367170023A2E500DA
:10EA700083274B00938585001385090093E71700D2
:10EA80002322FB00EF509FF16FF05FF793F6C6FF74
:10EA90003306DA00938504016350B60E93F717002E
:10EAA000E39007E0032C84FF338C8A4183274C00DA
:10EAB00093F7C7FFB386D700338B4601E34EBBDC29
:10EAC0008327CC0003278C001306CAFF930640025D
:10EAD0002326F70023A4E70013098C0063EEC62069
:10EAE00093053001032704009307090063F2C50270
:10EAF0002324EC00032744009307B0012326EC00F5
:10EB000063E4C7200327840093070C0113048400E7
:10EB100023A0E7000327440023A2E7000327840083
:10EB200023A4E70033079C00B3079B4023A4EB001A
:10EB300093E717002322F70083274C001385090071
:10EB400093F71700B3E4970023229C00EF905F9E99
:10EB50006FF0DFDD2320D500832644001307B001CA
:10EB60002322D5006360C712832684001307840024
:10EB7000930785006FF05FD7B38A9A00B30796407A
:10EB800023A45B0193E7170023A2FA008327C4FFA5
:10EB9000138509001309040093F71700B3E49700E5
:10EBA000232E94FEEF90DF986FF05FD88327CB0081
:10EBB00003278B00130A0600338BCA002326F700B5
:10EBC00023A4E7006FF01FE18327C5FF93F7C7FF7A
:10EBD000330AFA00338B4A016FF0DFDF930504003C
:10EBE000EFF05FA66FF09FD18327CB0003278B0048
:10EBF0001306CAFF930640022326F70023A4E7006A
:10EC000003278C008327CC0013098C00330B7C0175
:10EC10002326F70023A4E70063E8C6049306300127
:10EC20000327040093070900E3F6C6D82324EC0069
:10EC3000032744009307B0012326EC000327840038
:10EC4000E3F6C7D62328EC000327C400930740024D
:10EC5000232AEC00032704016304F60693078C01C2
:10EC6000130404016FF01FD5930504001305090078
:10EC7000EFF05F9D13040900138A0B00930A0C0048
:10EC80006FF05FD5032784002324E5000327C40029
:10EC90002326E500832604016302F604130704011A
:10ECA000930705016FF05FC4832784002328FC00CD
:10ECB0008327C400232AFC0003270401E310D6FAAB
:10ECC000232CEC000327440193070C021304840156
:10ECD000232EEC00032704006FF0DFCD2328D5009E
:10ECE000832644011307840193078501232AD50055
:10ECF000832684016FF05FBF9305040013050900AC
:10ED0000EFF05F946FF01FE2832784002328FC005C
:10ED10008327C400232AFC00032704016308D600CC
:10ED200093078C01130404016FF09FDE232CEC0089
:10ED30000327440193070C0213048401232EEC00E3
:10ED4000032704006FF0DFDC130101FF232481009F
:10ED50001384050083A505002322910023261100BA
:10ED60009304050063840500EFF01FFE9305040083
:10ED7000032481008320C100138504008324410003
:10ED8000130101016F509FC1B727008183A787BB83
:10ED90006380A7108325C504130101FE232A910077
:10EDA000232E1100232C8100232821012326310149
:10EDB000930405006380050413090000930900080B
:10EDC000B387250103A40700630E04009305040024
:10EDD0000324040013850400EF505FBCE31804FE15
:10EDE00083A5C40413094900E31C39FD13850400FD
:10EDF000EF50DFBA83A50404638605001385040081
:10EE0000EF50DFB903A48414630004021389C4140F
:10EE1000630C2401930504000324040013850400FB
:10EE2000EF50DFB7E31889FE83A54405638605002C
:10EE300013850400EF509FB683A78403638C0702F9
:10EE400083A7C40313850400E780070083A5042E6D
:10EE500063820502032481018320C101032901018A
:10EE60008329C10013850400832441011301010299
:10EE70006FF09FED8320C1010324810183244101B0
:10EE8000032901018329C1001301010267800000E9
:10EE90006780000083278600130101FD232A5101AA
:10EEA00023261102232481022322910223202103FD
:10EEB000232E3101232C41012328610123267101D6
:10EEC00023248101930A060063880714130B0500AD
:10EED0008329060003A5050083A48500138405008B
:10EEE0006F00400D8357C40013F70748630A0708F3
:10EEF0008326440183250401130719009394160007
:10EF0000B386D40093D4F601330AB540B384D40059
:10EF100093D41440330747011386040063F6E400DA
:10EF2000930407001306070093F707406386070A58
:10EF30009305060013050B00EF805FCF130C05004F
:10EF4000630A050A8325040113060A00EFF0CFDDEA
:10EF50008357C40093F7F7B793E707082316F40025
:10EF600033054C01338A4441232A9400232444016D
:10EF7000232884012320A40093040900130A090014
:10EF800013060A0093850B00EFF0CFEB03278400F4
:10EF90000325040083A78A00B30497403305450185
:10EFA000232494002320A4003389274123A42A0189
:10EFB0006304090603A9490083AB0900138A04000E
:10EFC00093898900E30809FEE37E99F09304090020
:10EFD000130A09006FF0DFFA13050B00EFF04FFF83
:10EFE000130C0500E31E05F68325040113050B0031
:10EFF000EF50DF9A9307C0002320FB008357C40023
:10F000001305F0FF93E707042316F40023A40A0076
:10F0100023A20A006F00C00023A20A00130500000B
:10F020008320C102032481028324410203290102B7
:10F030008329C101032A8101832A4101032B010194
:10F04000832BC100032C81001301010367800000A2
:10F0500083D7C500130101ED232C41112328611131
:10F060002320A1112326111223248112232291127D
:10F0700023202113232E3111232A5111232671110C
:10F080002324811123229111232EB10F93F7070816
:10F090002326D100138A0500130B0500130D06006B
:10F0A0006386070083A70501E384075EB717008125
:10F0B000930AC104938747CEB71B0081B714008120
:10F0C00093090D0023205105232401042322010468
:10F0D000232A0100232C010023200102232E0100FA
:10F0E000232401002328F100938B0BE5938404E68D
:10F0F000138D0A0083C70900638C0720138409005D
:10F10000930650026388D72A83471400130414001F
:10F11000E39A07FE330C3441630C341F83268104C9
:10F120008327410423203D01B3868601938717007E
:10F1300023228D012324D1042322F104930670009D
:10F14000130D8D0063C0F628032781008347040058
:10F15000330787012324E100638C071A9308F0FF2B
:10F160008346140093091400A30D01022322010019
:10F1700013090000130CA005930C90009305A00246
:10F180001384080093891900938706FE6368FC04C2
:10F190000327010193972700B387E70083A70700A0
:10F1A0006780070023220100938706FD03264100A4
:10F1B00083C6090093891900131726003307C70077
:10F1C00013171700B387E7002322F100938706FD8A
:10F1D000E3FEFCFC938706FEE37CFCFA638A0612DE
:10F1E0002306D108A30D0102130C1000930C10008C
:10F1F0001304C10893080000137F290063040F0063
:10F20000130C2C00937E49088327810403264104B4
:10F2100063980E0003274100B30D8741634AB07B1A
:10F220000345B1039305160093068D0063000504A2
:10F230001305B103938717002320AD0013051000B9
:10F240002322AD002324F1042322B104130570000E
:10F25000E340B50A930F260013050D011386050040
:10F26000138D060093850F0093060500630C0F02B3
:10F270001306C103938727002320CD001306200027
:10F280002322CD002324F1042322B10413077000AC
:10F29000E342B70A13860500138D06009385150017
:10F2A0009386860013050008638CAE54B38D984195
:10F2B0006344B063B387FC0023208D0023229D01AB
:10F2C0002324F1042322B104130770006342B76CB6
:10F2D000137349006308030003274100B30C8741FF
:10F2E000E3489009032441006354840113040C0093
:10F2F00003278100330787002324E100639A076A0C
:10F3000083C7090023220104138D0A00E39807DE56
:10F3100083278104E39E07568357CA0093F70704A7
:10F32000E394075A8320C11203248112032581002C
:10F3300083244112032901128329C111032A811157
:10F34000832A4111032B0111832BC110032C81103F
:10F35000832C4110032D0110832DC10F13010113C4
:10F360006780000013050B00EF80CFE18327450085
:10F3700013850700232EF100EFA04FFB9307050034
:10F3800013050B00938D07002320F102EF808FDF20
:10F39000832785009305A002232CF100E3980D1E1E
:10F3A00083C609006FF01FDE83C6090013690902D6
:10F3B0006FF05FDD330C3441E31234D78347040030
:10F3C0006FF09FD91306010493050A0013050B0083
:10F3D000EFF05FACE31205F4138D0A006FF0DFD697
:10F3E0008327C10093080400A30D010203A40700B2
:10F3F000938D4700E30404389307F0FFE38EF8266B
:10F40000138608009305000013050400232611014C
:10F41000EF908F848328C100E3060548B30C854034
:10F420002326B101930800006F0040090327C100A3
:10F43000A30D0102130C10008327070013074700D8
:10F440002326E1002306F108930C10001304C108E1
:10F450006FF05FDA9377090293080400638E070E5A
:10F460008327C1009387770093F787FF83A6470020
:10F4700083AC0700938787002326F100138C0600D6
:10F4800063C406109306F0FF930D09006388D8004B
:10F49000B3E68C01937DF9F7638E0676E31C0C00CE
:10F4A00093069000E3E8960193870C03A307F10EFF
:10F4B00013890D00930C10001304F10E138C080037
:10F4C00063D49801138C0C008347B103B337F00069
:10F4D000330CFC006FF05FD293080400136909013C
:10F4E00093770902638407748327C10093877700A9
:10F4F00093F787FF83AC070003AC4700938787002F
:10F500002326F100937DF9BF93060000A30D0102AD
:10F510001306F0FF638EC80833E68C0113F9FDF77C
:10F520006314064A63920828639A066E93FC1D00D2
:10F530001304010FE3840CF893070003A307F10EF3
:10F540001304F10E6FF09FF7136909019377090215
:10F5500093080400E39607F00327C100937709019D
:10F5600093064700E392070493770904E38607268E
:10F570008327C1002326D100839C070013DCFC41B4
:10F5800093060C00E3D006F0B3369001B30E804131
:10F59000338CDE409306D002A30DD1021306F0FF98
:10F5A000B30C9041930D090093061000E396C8F642
:10F5B00013061000E384C6EE130620006380C62005
:10F5C0001304010F9317DC0193F67C0093DC3C00DD
:10F5D00093860603B3EC9701135C3C00A30FD4FEA3
:10F5E000B3E78C01930504001304F4FFE39C07FCCC
:10F5F00093F71D00638E071E93070003638AF61EB0
:10F600009385E5FFA30FF4FE9307010FB38CB7407A
:10F6100013890D00138405006FF05FEA930804005E
:10F62000936D090193F70D02638807628327C10078
:10F630009306100013897700137989FF93078900D7
:10F64000832C0900032C49002326F1006FF01FECE6
:10F650008327C100B786FFFF93C6068383AC0700EC
:10F66000938747002326F100B7070081938747352A
:10F67000231ED10293080400130C0000936D29008F
:10F68000232AF100930620006FF05FE883C609008B
:10F69000136909086FF01FAF83C6090013871900AB
:10F6A000E38AB622938706FD93090700130400003E
:10F6B000E3ECFCAC83C6090013172400B3088700F1
:10F6C000939818003384F800938706FD93891900F6
:10F6D000E3F2FCFE6FF05FAB83C6090013694900DB
:10F6E0006FF05FAA9307B00283C60900A30DF10271
:10F6F0006FF05FA90327C10083C6090083270700B5
:10F70000130747002326E1002322F100E3DC07A6CC
:10F71000B307F0402322F100136949006FF09FA660
:10F7200083C60900136919006FF0DFA58347B10391
:10F7300083C60900E39807A493070002A30DF10212
:10F740006FF05FA483C6090093078006638EF67E80
:10F75000136909046FF01FA30327C10093770902FF
:10F7600083260700130747002326E100639C075EFA
:10F7700093770901639E077E93770904E39407104A
:10F78000137309206306037E832781002380F6001C
:10F790006FF05F9683C609009307C006638EF67A02
:10F7A000136909016FF01F9E13061000E384C61051
:10F7B00013062000930D0900E394C6E0832641015F
:10F7C0001304010F93F7FC00B387F60003C707008B
:10F7D00093DC4C009317CC01B3EC9701135C4C0005
:10F7E000A30FE4FEB3E78C011304F4FFE39C07FCD2
:10F7F0009307010FB38C874013890D006FF01FCC66
:10F8000003274100B30D8741E352B0AB130500015C
:10F81000E356B50B232281029306000113040A006C
:10F82000930E7000138A0D00938D090093890800D0
:10F830006F00C000130A0AFF63DA460593870701C9
:10F840001306160023209D002322DD002324F1044B
:10F850002322C104130D8D00E3DECEFC1306010448
:10F860009305040013050B00EFF0CFE2631E056E55
:10F8700093060001130A0AFF83278104032641042B
:10F88000138D0A00930E7000E3CA46FB93880900AB
:10F8900093890D00930D0A00130A0400032441020A
:10F8A0001306160013058D00B387B70123209D00B2
:10F8B0002322BD012324F1042322C1041307700075
:10F8C000634AC764B38D984193051600930685007B
:10F8D000130D0500E350B09F13050001635EB5737F
:10F8E00093060001930870006F00C000938D0DFF18
:10F8F00063DAB605938707011306160023209D00DF
:10F900002322DD002324F1042322C104130D8D00E2
:10F91000E3DEC8FC1306010493050A0013050B007F
:10F92000EFF04FD7E31A059E93060001938D0DFF6C
:10F930008327810403264104138D0A009308700075
:10F94000E3CAB6FB9305160013068D00B387B70113
:10F9500023209D002322BD012324F1042322B1048E
:10F96000130770006342B732130D0600938515002C
:10F97000B387FC0023208D0023229D012324F10462
:10F980002322B1041307700093068600E352B79454
:10F990001306010493050A0013050B00EFF08FCF47
:10F9A000E31C05968327810493860A006FF05F921B
:10F9B0001306010493050A0013050B00EFF08FCD29
:10F9C000E30005946FF05F95930D09006FF05FBE43
:10F9D0009306000163DEB60B13070D00930F700052
:10F9E000130D0C002322E103130C09002324D1037F
:10F9F00013090A00138A09009309040013840D00F7
:10FA0000938D0C00938C08006F00C000130404FF5A
:10FA100063DA860493870701130616002320770113
:10FA20002322D7002324F1042322C10413078700D3
:10FA3000E3DECFFC130601049305090013050B0058
:10FA4000EFF04FC56316054A93060001130404FF47
:10FA5000832781040326410413870A00930F700053
:10FA6000E3CA86FA032F4102832E810293880C0099
:10FA7000938C0D00930D04001384090093090A0070
:10FA8000130A090013090C00130C0D00130D0700D5
:10FA9000B387B7011306160023207D012322BD0181
:10FAA0002324F1042322C10493067000130D8D005A
:10FAB00063D8C6F61306010493050A0013050B006C
:10FAC000232611032324D1032322E103EFF08FBC6B
:10FAD000E314058483278104032641048328C1029B
:10FAE000832E8102032F4102138D0A006FF04FF322
:10FAF0001306010493050A0013050B0023261103C6
:10FB00002324D1032322E103EFF0CFB8E3160580CD
:10FB100003264104832781048328C102832E8102A6
:10FB2000032F41029306410593051600138D0A0029
:10FB30006FF0CFF31306010493050A0013050B00C1
:10FB4000232411032322D103EFF0CFB4631605FC65
:10FB5000032641048327810483288102832E4102E6
:10FB60009306410593051600138D0A006FF08FF37D
:10FB7000130600010327410463509607930D00010B
:10FB8000130470006F00C000938C0CFF63D69D05BA
:10FB9000938707011307170023A0760123A2B6015C
:10FBA0002324F1042322E10493868600E35EE4FC2F
:10FBB0001306010493050A0013050B00EFF08FAD47
:10FBC000631C05F4938C0CFF8327810403274104F5
:10FBD00093860A00E3CE9DFBB387970113071700B6
:10FBE00023A0760123A296012324F1042322E10419
:10FBF0009306700063D8E6EE1306010493050A002D
:10FC000013050B00EFF00FA9631805F0832781049B
:10FC10006FF04FEDE39A088813890D0093080000F8
:10FC2000930C00001304010F6FF05F890327C100DC
:10FC300093770901930647006392071893770904A5
:10FC4000638E07368327C100130C00002326D100E2
:10FC500083DC07006FF01F8B0327C10093F70D01B2
:10FC600093064700639A071093F70D0463860738DD
:10FC70008327C100130C00002326D10083DC07007A
:10FC8000930610006FF09F881306010493050A0085
:10FC900013050B00EFF00FA0631005E88325410466
:10FCA000832781049306410593851500138D0A006F
:10FCB0006FF04FE093F70D402324410323263103D7
:10FCC000130A0C0093890C0013090000832C810196
:10FCD0001304010F23221103138C07006F0040024D
:10FCE0001306A000930600001385090093050A007F
:10FCF000EF00406C63060A3293090500138A050081
:10FD00001306A000930600001385090093050A005E
:10FD1000EF00902D13050503A30FA4FE130919008E
:10FD20001304F4FFE30E0CFA83C60C00E39A26FBDF
:10FD30009307F00FE306F9FA631C0A169307900085
:10FD400063E837179307010F232C910183284102A1
:10FD5000032A81028329C102B38C874013890D00D5
:10FD60006FF0CFF5032781009357F74123A0E600FA
:10FD700023A2F6006FF00FB82326D100832C0700D2
:10FD8000130C0000930610006FF04FF883278101D9
:10FD900083C60900638807BE83C70700638407BE64
:10FDA000136909406FF00FBE832C07002326D10092
:10FDB00013DCFC4193060C006FF08FEC832C0700E2
:10FDC000130C00002326D1006FF0CFF3B70700819A
:10FDD00093878736232AF10093770902930804005A
:10FDE000638C07068327C1009387770093F787FF0B
:10FDF00083AC070003AC4700938787002326F100FC
:10FE000013761900630E060033E68C01630A0600C0
:10FE100013060003230EC102A30ED10213692900A9
:10FE2000937DF9BF930620006FF04FEE9308040016
:10FE3000930D09006FF00FFF930804006FF04FEA75
:10FE4000B707008193874735232AF100937709028A
:10FE500093080400E39807F80327C100937709018A
:10FE600013064700638A0708832C0700130C000061
:10FE70002326C1006FF0DFF813050400EF901FCBBD
:10FE8000930C05002326B101930800006FF00FE3E7
:10FE900093050004EF709FD92320AA002328AA000D
:10FEA000630C052493070004232AFA006FF00FA0C7
:10FEB000832701028325C101130900003304F440A4
:10FEC0001386070013050400EF901FCF83C51C00A5
:10FED0001306A000930600003338B0001385090014
:10FEE00093050A00B38C0C01EF00C04C6FF0DFE00B
:10FEF000130A09006FF04FC2937709046382070A5F
:10FF00008327C100130C00002326C10083DC0700F7
:10FF10006FF01FEF1306010493050A0013050B0091
:10FF200023221103EFE01FF7631805BE03264104E7
:10FF30008327810483284102930641059305160017
:10FF4000138D0A006FF08FB683C61900136909205C
:10FF5000938919006FF00FA383C619001369090272
:10FF6000938919006FF00FA2130A04006FF0CFBA43
:10FF70008327810023A0F6006FF0CF9793076000DE
:10FF8000938C080063F41701930C6000370E008116
:10FF9000138C0C002326B1011304CE376FF08FA50C
:10FFA000937709206386070C8327C100130C000098
:10FFB0002326C10083CC07006FF09FE493770920CC
:10FFC000638E07088327C100130C00002326D1008D
:10FFD00083CC07006FF00FD3937709206384070663
:10FFE0008327C1002326D100838C070013DCFC414A
:10FFF00093060C006FF0CFC893F70D2063880702BB
:02000004800179
:100000008327C100130C00002326D10083CC0700F6
:10001000930610006FF08FCF138606006FF01F93CA
:1000200093079000E3EA37CD6FF0DFD18327C1005B
:10003000130C00002326D10083AC070093061000A8
:100040006FF0CFCC8327C1002326D10083AC0700FB
:1000500013DCFC4193060C006FF08FC28327C100B4
:10006000130C00002326D10083AC07006FF08FC96A
:100070008327C100130C00002326C10083AC0700B6
:100080006FF01FD8832781002390F6006FF08F86D2
:100090001306010493050A0013050B00EFE09FDF30
:1000A0006FF08FA7938C08002326B10193080000FE
:1000B0006FF0CFC0930D09006FF00FBF13850600DE
:1000C000138605006FF04FFE9307F0FF2324F10025
:1000D0006FF04FA58327C10003A407009387470053
:1000E000635404001304F0FF83C619002326F100B3
:1000F000930907006FF00F899307C0002320FB00CE
:100100009307F0FF2324F1006FF0CFA1130101FE4C
:10011000232C8100232A910023282101232E110062
:1001200023263101130905009384050013040600FA
:100130006306050083278503638807140317C4003B
:1001400083268401937787002324D4009316070124
:1001500093D606016382070883270401638E07068E
:100160001396260193F9F40F93F4F40F635E0608D7
:100170000327040083264401B307F74063DED70A50
:1001800083268400130617002320C4009386F6FFFD
:100190002324D40023003701032744019387170049
:1001A0006308F70C8357C40093F7170063860700B2
:1001B0009307A000638EF40A8320C1010324810108
:1001C000032901018329C10013850400832441010F
:1001D0001301010267800000930504001305090064
:1001E000EF30DFD0631E05080317C40093F9F40F46
:1001F000832704019316070193D60601139626015F
:1002000093F4F40FE34606F68326440637260000EF
:100210003367C70037E6FFFF1306F6FFB3F6C600E5
:100220002316E400032704002322D4068326440176
:10023000B307F740E3C6D7F493050400130509009C
:10024000EF408FA2631E050203270400832684006B
:1002500093071000130617009386F6FF2320C400AF
:100260002324D4002300370103274401E31CF7F2C1
:100270009305040013050900EF400F9FE30E05F2FC
:100280009304F0FF6FF05FF3EF40CFD86FF01FEBF8
:100290003727008193070500032587BB13860500D8
:1002A000938507006FF09FE6130101FE232C810068
:1002B000232A9100B7170081232E110083A787718D
:1002C000130405009384060063820502E78007009B
:1002D0009307F0FF6306F5028320C1010324810127
:1002E000832441011301010267800000130600000E
:1002F00093054100E78007009307F0FFE31EF5FC3C
:1003000023A004009307A0088320C1012320F40048
:10031000032481018324410113010102678000004D
:10032000130101FEB7270081232C8100232A9100AD
:10033000232E110083A487BBB717008183A7877181
:1003400013040600630A05021386050093060400E1
:100350009305050013850400E78007009307F0FF6D
:10036000630AF5028320C101032481018324410132
:100370001301010267800000930606009305410007
:100380001306000013850400E78007009307F0FFC1
:10039000E31AF5FC232004008320C101032481011A
:1003A0009307A00823A0F400832441011301010254
:1003B0006780000093080500938705001308060076
:1003C000138506001383080063940628B71600817E
:1003D000938646F263F6C50E370701006378E60C94
:1003E0001307F00F3337C700131737003355E600F4
:1003F000B386A60083C60600130500023387E60015
:10040000B306E540630CE500B397D70033D7E800A7
:100410003318D600B365F7003393D800935808011A
:10042000B3D715031316080113560601135703011A
:10043000B3F6150313850700B305F602939606017C
:1004400033E7E600637EB700330707011385F7FF44
:10045000636807016376B7001385E7FF3307070179
:100460003307B740B3771703131303011353030183
:10047000335717039397070133E36700B306E60288
:1004800013060700637CD300330368001306F7FFED
:10049000636603016374D3001306E7FF13150501B8
:1004A0003365C500930500006F00400E370500015D
:1004B00013070001E36CA6F2130780016FF01FF32E
:1004C00063160600130710003358C70237070100F0
:1004D0006370E80C1307F00F6374070113058000C5
:1004E0003357A800B386E60003C7060013060002D0
:1004F0003307A700B306E6406316E60AB387074151
:1005000093051000935808011316080113560601AD
:1005100013570301B3F61703B3D7170393960601D6
:1005200033E7E600330EF60213850700637EC7014A
:10053000330707011385F7FF636807016376C70177
:100540001385E7FF330707013307C741B377170365
:100550001313030113530301335717039397070131
:1005600033E36700B306E60213060700637CD3009B
:10057000330368001306F7FF636603016374D30057
:100580001306E7FF131505013365C50067800000FA
:100590003707000113050001E364E8F41305800147
:1005A0006FF01FF43318D800B3D5E7003393D800A9
:1005B000B397D70033D7E800935808013366F700A4
:1005C00033F715039317080193D707011355060155
:1005D000B3D51503131707013367A700B386B70216
:1005E00013850500637ED700330707011385F5FFE8
:1005F000636807016376D7001385E5FF33070701BA
:10060000B306D74033F71603131606011356060137
:10061000B3D6160313170701B388D702B367C70011
:100620001387060063FE1701B38707011387F6FFE0
:1006300063E8070163F617011387E6FFB387070135
:1006400093150501B3871741B3E5E5006FF09FEB04
:1006500063E6D5183707010063F4E6041307F00FCB
:10066000B335D700939535003717008133D5B600E1
:10067000130747F23307A7000347070013050002DB
:100680003307B700B305E5406316E5021305100014
:10069000E3EEF6EE33B5C800134515006FF01FEF1B
:1006A0003707000193050001E3E0E6FC93058001B4
:1006B0006FF09FFB3353E600B396B6003363D3006D
:1006C00013550301B31EB60033D6E700B376A60276
:1006D000B397B70033D7E8003368F70093170301E7
:1006E00093D70701135708013356A60293960601C4
:1006F00033E7E600338FC702130E0600637EE7017F
:1007000033076700130EF6FF636867006376E7013F
:10071000130EE6FF330767003307E741B376A702FE
:100720003357A702939606013386E7029317080111
:1007300093D70701B3E7F6009306070063FEC700EF
:10074000B38767009306F7FF63E8670063F6C700A7
:100750009306E7FFB387670013150E01370E0100FC
:100760003365D5009306FEFF3378D500B387C740C5
:10077000B3F6DE001356050193DE0E013303D802F3
:10078000B306D602135703013308D8033308D80041
:10079000330707013306D6036374D7003306C60157
:1007A000935607013386C60063E6C702E39CC7CEB3
:1007B000B70701009387F7FF3377F7001317070197
:1007C0003373F300B398B800330767009305000054
:1007D000E3FEE8DA1305F5FF6FF0DFCC93050000C8
:1007E000130500006FF09FDA9308060013870600D8
:1007F0009307050013880500639C0622B716008145
:10080000938646F263FCC50C37030100637E660ADB
:100810001303F00F6374C300130780003353E60023
:10082000B386660003CE0600330EEE001307000207
:100830003303C741630CC701B3956500335EC5013F
:10084000B31866003368BE00B317650013D60801FD
:100850003377C802139508011355050193D6070194
:100860003358C80213170701B366D70033080503CE
:1008700063FA0601B386160163E6160163F4060106
:10088000B3861601B386064133F7C6029397070174
:1008900093D70701B3D6C602B306D50213150701D5
:1008A000B367F50063FAD700B387170163E6170152
:1008B00063F4D700B3871701B387D74033D56700F8
:1008C0009305000067800000370300011307000153
:1008D000E36666F4130780016FF05FF463160600A9
:1008E00013061000B35816033706010063F2C80A56
:1008F0001306F00F637416011307800033D6E80067
:10090000B386C60003CE0600330EEE0013070002C6
:100910003303C7416318C709B385154113D70801CD
:10092000139508011355050113D60701B3F6E50227
:10093000B3D5E50293960601B3E6C600B305B5024A
:1009400063FAB600B386160163E6160163F4B600D7
:10095000B3861601B385B640B3F6E5029397070157
:1009600093D70701B3D5E502B305B5021395060188
:10097000B367F50063FAB700B387170163E61701A1
:1009800063F4B700B3871701B387B7406FF01FF365
:100990003706000113070001E3E2C8F613078001E0
:1009A0006FF0DFF5B398680033D7C501B317650062
:1009B000335EC50113D50801B376A702B395650070
:1009C000336EBE009395080193D5050113560E01B1
:1009D0003357A70293960601B3E6C6003387E502B4
:1009E00063FAE600B386160163E6160163F4E600D7
:1009F000B38616013386E640B376A602131E0E01B7
:100A0000135E0E013356A602939606013386C50285
:100A1000B3E5C60163FAC500B385150163E61501A8
:100A200063F4C500B3851501B385C5406FF01FEFB2
:100A3000E3EAD5E83707010063FCE604130EF00F84
:100A40003337DE0013173700B718008133D3E600C1
:100A5000938848F2B388680003CE0800330EEE0096
:100A6000130700023303C741631EC70363E4B600E4
:100A7000636AC500B307C540B385D5403335F5007B
:100A80003388A54013850700930508006FF09FE3A6
:100A9000B708000113070001E3E816FB1307800104
:100AA0006FF09FFA3357C601B3966600336FD700D5
:100AB000B3D7C50113570F01B3F8E702B39565002B
:100AC0003358C5013368B80093150F0193D505015C
:100AD000935608013316660033156500B3D7E70255
:100AE00093980801B3E6D800B38EF5029388070007
:100AF00063FED601B386E6019388F7FF63E8E6015B
:100B000063F6D6019388E7FFB386E601B386D64144
:100B1000B3FEE6021318080113580801B3D6E60223
:100B2000939E0E01B3EE0E01B385D50293870600A6
:100B300063FEBE00B38EEE019387F6FF63E8EE011D
:100B400063F6BE009387E6FFB38EEE01B385BE4029
:100B500093980801B70E0100B3E8F8009387FEFFF1
:100B600033F8F8009356060193D80801B377F600DE
:100B70003307F802B387F8023308D802B388D802E3
:100B80003308F80093560701B386060163F4F600B4
:100B9000B388D801B70701009387F7FF13D8060180
:100BA000B3F6F600939606013377F700B308180101
:100BB0003387E60063E61501639E1501637CE5005B
:100BC0003306C7403337C7003307E701B388E8402F
:100BD000130706003307E5403335E500B3851541BB
:100BE000B385A540B397C5013357670033E5E700E8
:100BF000B3D565006FF01FCD130101FD93D74501FB
:100C00002322910223202103232C41012328610167
:100C1000232481019394C5002326110223248102F9
:100C2000232E3101232A51012326710113975701E5
:100C300013090500130B0600138C060093D4C4009F
:100C400013DAF5016304070A93FAF77F9307F07F3D
:100C50006380FA109359D50193943400B3E499005A
:100C6000B7098000B3E9340113143500938A1AC020
:100C7000930B000093574C011315CC0013975701A9
:100C80009354C50093F5F77F135CFC0163000710D4
:100C90009307F07F6382F516139534009357DB01B9
:100CA00033E5A700B7048000B3649500931F3B00B1
:100CB000138515C01306000093972B00B3E7C700F8
:100CC0009387F7FF1307E000B3468A01B385AA4074
:100CD0006360F7163717008193972700130707E71C
:100CE000B387E70083A7070067800700B3E9A40084
:100CF000638E09066380040413850400EF30D03B43
:100D0000930755FF1307C001634CF7029309D00105
:100D1000130485FFB389F940B3948400B3593901B2
:100D2000B3E99900331489009305D0C0B38AA54074
:100D30006FF01FF4EF305038130505026FF05FFCC1
:100D4000930485FDB3199900130400006FF0DFFDD3
:100D5000B3E9A40063840902130405009389040025
:100D6000930AF07F930B30006FF0DFF01304000064
:100D7000930A0000930B10006FF0DFEF13040000E4
:100D8000930AF07F930B20006FF0DFEEB3EF640166
:100D900063800F086382040413850400EF30D031B0
:100DA00093050500938755FF1307C001634EF702B3
:100DB0009306D001938F85FFB386F6403395F401F7
:100DC000B356DB00B3E4A600B31FFB011307D0C08A
:100DD0003305B7406FF01FEE13050B00EF30D02D39
:100DE000930505026FF01FFC138585FDB314AB005E
:100DF000930F00006FF09FFDB3EF640163820F0259
:100E0000930F0B001305F07F130630006FF0DFEA3D
:100E10009304000013050000130610006FF0DFE9D3
:100E2000930400001305F07F130620006FF0DFE845
:100E300063E63401639C9934636AF4351396F901CF
:100E4000135714009317F40193D919003364E60083
:100E50001395840093D88F01B3E8A80013550501BA
:100E600033D8A902939E080193DE0E0113570401A3
:100E700013938F00B3F4A902930F080033860E0377
:100E80009399040133673701637EC7003307170165
:100E9000930FF8FF636817016376C700930FE8FFAD
:100EA000330717013307C740335EA7021314040149
:100EB000135404013377A70213060E003388CE03C0
:100EC000131707013367E400637E07013307170137
:100ED0001306FEFF63681701637607011306EEFF32
:100EE0003307170133040741939F0F0137080100AF
:100EF000B3EFCF00130EF8FF13D60F0133F7CF0176
:100F0000135F0301337EC301B303EE02B304C603D0
:100F10003307EF02B302E6033306970013D703014A
:100F20003307C70063749700B382020113560701A9
:100F300033065600B70201009382F2FF3378570060
:100F400013180801B3F35300330878006368C40032
:100F500093840F006314C40463F20705B38767002A
:100F600033B76700330717013304E4009384FFFFAE
:100F700063E688006394880263E267026366C400E4
:100F8000631E860063FC0701B387670033B7670001
:100F9000330717019384EFFF3304E40033880741DC
:100FA0003304C440B3B707013304F440930FF0FF98
:100FB00063848812B35FA402135708013374A40238
:100FC00013860F00B387FE031314040133648700F4
:100FD000637EF400330414011386FFFF6368140179
:100FE0006376F4001386EFFF330414013304F440F6
:100FF0003357A40213180801135808013374A402CC
:1010000093070700B38EEE021314040133648800C3
:10101000637ED401330414019307F7FF636814015E
:101020006376D4019307E7FF330414011316060116
:101030003366F6009317060193D70701135706018D
:101040003308EF023304D441330FFF02B38EC703DA
:10105000330EC70393D70E01330FCF01B387E701D8
:1010600063F6C701370701003308E80013D707010B
:1010700033070701370801001308F8FF33F50701AC
:1010800013150501B3FE0E013305D5016368E400B5
:101090006310E424930F0600630005043384880082
:1010A000930FF6FF636414036366E4006310E422A5
:1010B0006370A3029317130033B36700B3081301DF
:1010C000930FE6FF33041401138307006314E40055
:1010D0006304650093EF1F009387F53F6358F0109A
:1010E00013F77F006300070213F7FF0013064000A9
:1010F000630AC70013864F00B33FF601B384F401BF
:10110000930F060013977400635A0700B70700FF98
:101110009387F7FFB3F4F400938705401307E07F4C
:101120006340F70A93DF3F001397D4013367F70159
:1011300013D53400939747013706F07F1315C50088
:101140008320C10203248102B3F7C7001355C500F1
:1011500033E5A7009396F601B367D50083244102D7
:10116000032901028329C101032A8101832A410144
:10117000032B0101832BC100032C81001305070001
:101180009385070013010103678000009385F5FF35
:10119000930700006FF0DFCB93060A0093840900E9
:1011A000930F040013860B00930730006308F60EBC
:1011B00093071000630EF60E93072000E31EF6F06F
:1011C00013050000130700009307F07F6FF09FF6F0
:1011D00093060C006FF05FFDB7040800930F00004A
:1011E00093060000130630006FF01FFC130510007B
:1011F0003305F54013078003634CA70A1307F0017A
:101200006344A7069385E541B397B40033D7AF0095
:10121000B395BF00B3E7E700B335B000B3E7B7005D
:1012200033D5A40013F777006300070213F7F70024
:1012300013064000630AC70013874700B337F7005F
:101240003305F50093070700131785006348070669
:101250001317D50193D737003367F70013553500BF
:10126000930700006FF01FED130710FEB307F74060
:1012700013060002B3D7F400130700006306C5008D
:101280009385E5433397B400B36FF701B33FF001A3
:10129000B3E7F701130500006FF0DFF8370508002A
:1012A000130700009307F07F930600006FF09FE89C
:1012B00013050000130700006FF09FFA13050000EC
:1012C00013070000930710006FF0DFE613860F008E
:1012D000930F06006FF01FE0130101FD93D7450146
:1012E0002324810223229102232E3101232C410148
:1012F000232A51019394C5002326110223202103A0
:101300002328610123267101139757011304050057
:1013100093090600938A060093D4C40013DAF501FA
:101320006306070A13FBF77F9307F07F6302FB1046
:101330009357D50193943400B3E49700B707800026
:10134000B3E4F40013193500130B1BC0930B00001A
:1013500093D74A011394CA00139757011354C4003A
:1013600013F5F77F93DAFA01630007109307F07F14
:101370006300F51693D7D9011314340033E48700C2
:10138000B70780003364F400130515C09397390044
:101390001307000093962B00B3E6E6003305AB007D
:1013A0009386F6FF1308E00033465A0193051500B3
:1013B000636CD81437150081939626001305C5EA8F
:1013C000B386A60083A606006780060033E9A40062
:1013D000630C09066380040413850400EF30C04DDC
:1013E000130755FF9307C00163CCE7029307D001B1
:1013F000130985FFB387E740B3942401B357F40082
:10140000B3E4970033192401130BD0C0330BAB4066
:101410006FF0DFF3EF30404A130505026FF05FFC19
:10142000930485FDB3149400130900006FF0DFFDF1
:1014300033E9A4006302090213090500130BF07FCE
:10144000930B30006FF0DFF093040000130B0000EB
:10145000930B10006FF0DFEF93040000130BF07F8D
:10146000930B20006FF0DFEEB3673401638E070645
:101470006300040413050400EF300044930655FF95
:101480009307C00163CED7021307D001930785FFEE
:101490003307D7403314F40033D7E90033648700AF
:1014A000B397F9001307D0C03305A7406FF05FEE84
:1014B00013850900EF304040130505026FF01FFC53
:1014C000130485FD33948900930700006FF09FFD9E
:1014D000B367340163820702938709001305F07F25
:1014E000130730006FF01FEB13040000130500001A
:1014F000130710006FF01FEA130400001305F07FBC
:10150000130720006FF01FE9370F01001307FFFFDB
:101510009356090113D307013379E900B3F7E700C4
:10152000B30823033308F902B38FF602B38EF80130
:1015300093580801B388D801338E660263F4F8012A
:10154000330EEE0193D20801B3F8E8003378E800D7
:10155000135F0401939808013374E400B388080111
:10156000338786023308890233092F03B30EE9005B
:10157000135908013309D901B386E6036376E900FC
:1015800037070100B386E600935E0901B38EDE00E3
:10159000B7060100938FF6FF3379F9013378F8012C
:1015A00013D7040113190901B3F4F401B3839702AB
:1015B00033090901B382220133089302B307F7020A
:1015C000B30FE3023303F80013D8030133086800B4
:1015D0006374F800B38FDF0093570801B70601006A
:1015E000B38FF7019387F6FF3378F800B3F7F30072
:1015F000B3039402131808013308F8003304870278
:10160000B3049F023303EF02B384840013D70301B2
:10161000B304970063F484003303D300B7070100D9
:101620009387F7FFB3F6F40093960601B3F7F30040
:10163000330E5E00B386F60033392E01B386D60131
:1016400033872601330E0E0133380E01330FF701B5
:10165000B3020F01B3B6D6013337270133E7E600F3
:1016600033B8020193D40401B33FFF01330797005D
:1016700033E80F0193179E00330707013307670014
:10168000B3E7170113179700B337F000135E7E011D
:1016900013D47201B3E7C7019392920093167700B7
:1016A00033648700B3E7570063D4061013D71700DD
:1016B00093F71700B367F7001317F401B3E7E700D8
:1016C000135414009386F53F6358D00E13F7770038
:1016D0006300070213F7F70013054000630AA70031
:1016E00013874700B337F7003304F400930707006C
:1016F00013177400635A0700370700FF1307F7FF3B
:101700003374E400938605401307E07F6348D716DF
:1017100013D737009317D401B3E7E700135434000D
:10172000139746011314C400B706F07F3377D70030
:101730001354C400336487001316F6018320C102DA
:101740003367C40003248102832441020329010278
:101750008329C101032A8101832A4101032B01014D
:10176000832BC100138507009305070013010103B4
:101770006780000013060A00138404009307090021
:1017800013870B0093062000630AD70E93063000E0
:10179000630CD70C93061000E316D7F21304000075
:1017A000930700006F00800813860A006FF09FFD0A
:1017B000930505006FF01FF1130510003305D540A8
:1017C00013078003E34CA7FC1307F0016344A7064B
:1017D0009385E5413317B400B3D6A700B397B7009C
:1017E0003367D700B337F000B367F7003354A40072
:1017F00013F777006300070213F7F7009306400022
:10180000630AD70013874700B337F7003304F400A7
:101810009307070013178400634A07061317D401C0
:1018200093D73700B367F7001354340093060000D2
:101830006FF01FEF130710FE3307D74013080002A5
:101840003357E40093060000630605019385E543E2
:10185000B316B400B3E7F600B337F000B367F70090
:10186000130400006FF0DFF837040800930700004E
:101870009306F07F130600006FF09FEA1304000048
:10188000930700009306F07F6FF09FE913040000B8
:1018900093070000930610006FF09FE88327C500B0
:1018A00003AF050083AF450083A2850083A5C50073
:1018B0003787000093D607011307F7FF1398070136
:1018C000939E050113D6F701B3F6E60093D7050101
:1018D0008328050003234500032E8500130101FF23
:1018E0001358080193DE0E01B3F7E70093D5F50115
:1018F0006390E60233E768003367C7013367070187
:1019000013051000631A07046398D7046F00800062
:10191000639CE7003367FF01336757003367D701E4
:1019200013051000631A0702130510006396D7020F
:101930006394E8036312F30363105E02631ED8012D
:101940006300B602639A070033E568003365C5019A
:10195000336505013335A0001301010167800000E4
:10196000130500006FF05FFF832F0500032845007B
:10197000032E85000325C50083A6C500B787000098
:10198000135605019387F7FF1393060113D706013A
:1019900083A2050083A8450083AE85003376F60058
:1019A00093150501130101FF93D505011355F501A9
:1019B000135303013377F70093D6F601631EF60045
:1019C000B3E70F01B3E7C701B3E7B7006388070CBC
:1019D0001305E0FF6F004006631AF700B3E712013A
:1019E000B3E7D701B3E76700E39407FE631A060A7B
:1019F000B3E70F01B3E7C701B3E7B70093B7170029
:101A0000631A070033EF1201336FDF01336F6F008A
:101A1000630A0F06639C07006394A6006352C70223
:101A2000630E05041305F0FF6F0000011305F0FFBE
:101A3000638406001385060013010101678000001E
:101A40006356E600E31A05FE6FF0DFFDE36AB3FCC0
:101A5000639E6502E3E6CEFD631EDE03E3E208FD5E
:101A600063141801E3EEF2FBE36E18FD6314180132
:101A7000E3EA5FFC130500006FF01FFC1305100084
:101A80006FF09FFBE39807FE6FF09FF9E3EC65FAB8
:101A90006FF05FFEE368DEFB6FF0DFFDE300C7F48D
:101AA000E31C07F6930700006FF0DFF5832F0500B6
:101AB00003284500032E85000325C50083A6C50025
:101AC000B7870000135605019387F7FF13930601AC
:101AD00013D7060183A2050083A8450083AE8500C5
:101AE0003376F60093150501130101FF93D5050127
:101AF0001355F501135303013377F70093D6F6011D
:101B0000631EF600B3E70F01B3E7C701B3E7B70001
:101B10006388070C130520006F004006631AF70066
:101B2000B3E71201B3E7D701B3E76700E39407FE19
:101B3000631A060AB3E70F01B3E7C701B3E7B700BB
:101B400093B71700631A070033EF1201336FDF01F9
:101B5000336F6F00630A0F06639C07006394A6004F
:101B60006352C702630E05041305F0FF6F00000106
:101B70001305F0FF638406001385060013010101BD
:101B8000678000006356E600E31A05FE6FF0DFFD94
:101B9000E36AB3FC639E6502E3E6CEFD631EDE03EB
:101BA000E3E208FD63141801E3EEF2FBE36E18FDB7
:101BB00063141801E3EA5FFC130500006FF01FFCDB
:101BC000130510006FF09FFBE39807FE6FF09FF97D
:101BD000E3EC65FA6FF05FFEE368DEFB6FF0DFFDBC
:101BE000E300C7F4E31C07F6930700006FF0DFF58E
:101BF000130101F4232A910A83A4C50083A60500DA
